Component: Arm Compiler for Embedded 6.19 Tool: armlink [5e73cb00]

==============================================================================

Section Cross References

    hal_entry.o(.text.getSystemTicks) refers to hal_entry.o(.bss.SysTickms) for SysTickms
    hal_entry.o(.ARM.exidx.text.getSystemTicks) refers to hal_entry.o(.text.getSystemTicks) for [Anonymous Symbol]
    hal_entry.o(.text.SystickInit) refers to bsp_clocks.o(.text.R_BSP_SourceClockHzGet) for R_BSP_SourceClockHzGet
    hal_entry.o(.ARM.exidx.text.SystickInit) refers to hal_entry.o(.text.SystickInit) for [Anonymous Symbol]
    hal_entry.o(.text.SysTick_Handler) refers to hal_entry.o(.bss.SysTickms) for SysTickms
    hal_entry.o(.ARM.exidx.text.SysTick_Handler) refers to hal_entry.o(.text.SysTick_Handler) for [Anonymous Symbol]
    hal_entry.o(.text.read_button_GPIO) refers to common_data.o(.bss.g_ioport_ctrl) for g_ioport_ctrl
    hal_entry.o(.text.read_button_GPIO) refers to r_ioport.o(.text.R_IOPORT_PinRead) for R_IOPORT_PinRead
    hal_entry.o(.ARM.exidx.text.read_button_GPIO) refers to hal_entry.o(.text.read_button_GPIO) for [Anonymous Symbol]
    hal_entry.o(.text.Callback_btn_Handler) refers to hal_entry.o(.bss.SysTickms) for SysTickms
    hal_entry.o(.text.Callback_btn_Handler) refers to log.o(.text.logWrite) for logWrite
    hal_entry.o(.text.Callback_btn_Handler) refers to hal_entry.o(.rodata.str1.1) for [Anonymous Symbol]
    hal_entry.o(.ARM.exidx.text.Callback_btn_Handler) refers to hal_entry.o(.text.Callback_btn_Handler) for [Anonymous Symbol]
    hal_entry.o(.text.DAC_SetVoltage) refers to hal_data.o(.rodata.g_dac0) for g_dac0
    hal_entry.o(.ARM.exidx.text.DAC_SetVoltage) refers to hal_entry.o(.text.DAC_SetVoltage) for [Anonymous Symbol]
    hal_entry.o(.text.GPT2_PWMA_SetDuty) refers to hal_data.o(.rodata.g_timer0) for g_timer0
    hal_entry.o(.text.GPT2_PWMA_SetDuty) refers to hal_data.o(.rodata.g_timer2) for g_timer2
    hal_entry.o(.text.GPT2_PWMA_SetDuty) refers to uldiv.o(.text) for __aeabi_uldivmod
    hal_entry.o(.ARM.exidx.text.GPT2_PWMA_SetDuty) refers to hal_entry.o(.text.GPT2_PWMA_SetDuty) for [Anonymous Symbol]
    hal_entry.o(.ARM.exidx.text.dwt_timestamp_init) refers to hal_entry.o(.text.dwt_timestamp_init) for [Anonymous Symbol]
    hal_entry.o(.text.hal_entry) refers to bsp_clocks.o(.text.R_BSP_SourceClockHzGet) for R_BSP_SourceClockHzGet
    hal_entry.o(.text.hal_entry) refers to hal_data.o(.rodata.g_uart9) for g_uart9
    hal_entry.o(.text.hal_entry) refers to hal_entry.o(.bss.buff) for buff
    hal_entry.o(.text.hal_entry) refers to hal_entry.o(.bss.buff_data) for buff_data
    hal_entry.o(.text.hal_entry) refers to lwrb.o(.text.lwrb_init) for lwrb_init
    hal_entry.o(.text.hal_entry) refers to shell_port_1.o(.text.userShellInit) for userShellInit
    hal_entry.o(.text.hal_entry) refers to hal_entry.o(.bss.SysTickms) for SysTickms
    hal_entry.o(.text.hal_entry) refers to hal_entry.o(.rodata.str1.1) for .L__FUNCTION__.hal_entry
    hal_entry.o(.text.hal_entry) refers to log.o(.text.logWrite) for logWrite
    hal_entry.o(.text.hal_entry) refers to hal_data.o(.rodata.g_adc0) for g_adc0
    hal_entry.o(.text.hal_entry) refers to hal_data.o(.rodata.g_dac0) for g_dac0
    hal_entry.o(.text.hal_entry) refers to hal_data.o(.rodata.g_timer0) for g_timer0
    hal_entry.o(.text.hal_entry) refers to hal_data.o(.rodata.g_timer2) for g_timer2
    hal_entry.o(.text.hal_entry) refers to hal_entry.o(.data.gpt2_pwma_duty) for gpt2_pwma_duty
    hal_entry.o(.text.hal_entry) refers to uldiv.o(.text) for __aeabi_uldivmod
    hal_entry.o(.text.hal_entry) refers to hal_data.o(.rodata.g_timer5) for g_timer5
    hal_entry.o(.text.hal_entry) refers to hal_entry.o(.bss.info) for info
    hal_entry.o(.text.hal_entry) refers to hal_entry.o(.bss.period) for period
    hal_entry.o(.text.hal_entry) refers to hal_entry.o(.bss.btn) for btn
    hal_entry.o(.text.hal_entry) refers to hal_entry.o(.text.read_button_GPIO) for read_button_GPIO
    hal_entry.o(.text.hal_entry) refers to hal_entry.o(.text.Callback_btn_Handler) for Callback_btn_Handler
    hal_entry.o(.text.hal_entry) refers to multi_button.o(.text.button_init) for button_init
    hal_entry.o(.text.hal_entry) refers to multi_button.o(.text.button_attach) for button_attach
    hal_entry.o(.text.hal_entry) refers to multi_button.o(.text.button_start) for button_start
    hal_entry.o(.text.hal_entry) refers to common_data.o(.rodata.g_ioport) for g_ioport
    hal_entry.o(.text.hal_entry) refers to multi_button.o(.text.button_ticks) for button_ticks
    hal_entry.o(.text.hal_entry) refers to lwrb.o(.text.lwrb_get_full) for lwrb_get_full
    hal_entry.o(.text.hal_entry) refers to lwrb.o(.text.lwrb_read) for lwrb_read
    hal_entry.o(.text.hal_entry) refers to shell_port_1.o(.bss.shell) for shell
    hal_entry.o(.text.hal_entry) refers to shell.o(.text.shellHandler) for shellHandler
    hal_entry.o(.text.hal_entry) refers to r_adc.o(.text.get_adc_scan_status) for get_adc_scan_status
    hal_entry.o(.text.hal_entry) refers to hal_entry.o(.bss.adc_val) for adc_val
    hal_entry.o(.text.hal_entry) refers to hal_data.o(.bss.g_adc0_ctrl) for g_adc0_ctrl
    hal_entry.o(.text.hal_entry) refers to r_adc.o(.text.R_ADC_InfoGet) for R_ADC_InfoGet
    hal_entry.o(.text.hal_entry) refers to hal_entry.o(.bss.temperature) for temperature
    hal_entry.o(.text.hal_entry) refers to hal_entry.o(.bss.gi_temperature) for gi_temperature
    hal_entry.o(.text.hal_entry) refers to r_adc.o(.text.reset_adc_scan_state) for reset_adc_scan_state
    hal_entry.o(.text.hal_entry) refers to hal_entry.o(.rodata.sindata) for sindata
    hal_entry.o(.text.hal_entry) refers to hal_entry.o(.bss.pwm_high_level_time) for pwm_high_level_time
    hal_entry.o(.text.hal_entry) refers to hal_entry.o(.bss.pwm_period) for pwm_period
    hal_entry.o(.text.hal_entry) refers to hal_entry.o(.bss.pwm_freq) for pwm_freq
    hal_entry.o(.text.hal_entry) refers to hal_entry.o(.bss.pwm_duty) for pwm_duty
    hal_entry.o(.text.hal_entry) refers to bsp_common.o(.text.__aeabi_assert) for __aeabi_assert
    hal_entry.o(.ARM.exidx.text.hal_entry) refers to hal_entry.o(.text.hal_entry) for [Anonymous Symbol]
    hal_entry.o(.text.R_BSP_WarmStart) refers to common_data.o(.bss.g_ioport_ctrl) for g_ioport_ctrl
    hal_entry.o(.text.R_BSP_WarmStart) refers to pin_data.o(.rodata.g_bsp_pin_cfg) for g_bsp_pin_cfg
    hal_entry.o(.text.R_BSP_WarmStart) refers to r_ioport.o(.text.R_IOPORT_Open) for R_IOPORT_Open
    hal_entry.o(.ARM.exidx.text.R_BSP_WarmStart) refers to hal_entry.o(.text.R_BSP_WarmStart) for [Anonymous Symbol]
    hal_entry.o(.text.user_timer0_callback) refers to common_data.o(.rodata.g_ioport) for g_ioport
    hal_entry.o(.text.user_timer0_callback) refers to hal_entry.o(.data.user_timer0_callback.level_led3) for user_timer0_callback.level_led3
    hal_entry.o(.ARM.exidx.text.user_timer0_callback) refers to hal_entry.o(.text.user_timer0_callback) for [Anonymous Symbol]
    hal_entry.o(.text.user_timer5_callback) refers to hal_entry.o(.bss.user_timer5_callback.one_period_flag) for user_timer5_callback.one_period_flag
    hal_entry.o(.text.user_timer5_callback) refers to hal_entry.o(.bss.user_timer5_callback.overflow_times) for user_timer5_callback.overflow_times
    hal_entry.o(.text.user_timer5_callback) refers to hal_entry.o(.bss.period) for period
    hal_entry.o(.text.user_timer5_callback) refers to hal_entry.o(.bss.user_timer5_callback.a_time) for user_timer5_callback.a_time
    hal_entry.o(.text.user_timer5_callback) refers to hal_entry.o(.bss.pwm_period) for pwm_period
    hal_entry.o(.text.user_timer5_callback) refers to hal_entry.o(.bss.pwm_high_level_time) for pwm_high_level_time
    hal_entry.o(.ARM.exidx.text.user_timer5_callback) refers to hal_entry.o(.text.user_timer5_callback) for [Anonymous Symbol]
    hal_entry.o(shellCommand) refers to hal_entry.o(.rodata.shellCmdgettemperature) for shellCmdgettemperature
    hal_entry.o(shellCommand) refers to hal_entry.o(.bss.gi_temperature) for gi_temperature
    hal_entry.o(shellCommand) refers to hal_entry.o(.rodata.shellDescgettemperature) for shellDescgettemperature
    hal_entry.o(shellCommand) refers to hal_entry.o(.rodata.shellCmdvarPwm) for shellCmdvarPwm
    hal_entry.o(shellCommand) refers to hal_entry.o(.data.gpt2_pwma_duty) for gpt2_pwma_duty
    hal_entry.o(shellCommand) refers to hal_entry.o(.rodata.shellDescvarPwm) for shellDescvarPwm
    shell.o(.text.shellInit) refers to shell.o(.bss.shellList) for shellList
    shell.o(.text.shellInit) refers to shell.o(.rodata.shellCmdDefaultUser) for shellCmdDefaultUser
    shell.o(.text.shellInit) refers to shell.o(.text.shellSeekCommand) for shellSeekCommand
    shell.o(.text.shellInit) refers to shell.o(.text.shellSetUser) for shellSetUser
    shell.o(.text.shellInit) refers to shell.o(.text.shellWritePrompt) for shellWritePrompt
    shell.o(.ARM.exidx.text.shellInit) refers to shell.o(.text.shellInit) for [Anonymous Symbol]
    shell.o(.text.shellSetUser) refers to strcmp.o(.text) for strcmp
    shell.o(.text.shellSetUser) refers to shell.o(.rodata.str1.1) for .L.str.21
    shell.o(.ARM.exidx.text.shellSetUser) refers to shell.o(.text.shellSetUser) for [Anonymous Symbol]
    shell.o(.text.shellSeekCommand) refers to shell.o(.text.shellCheckPermission) for shellCheckPermission
    shell.o(.text.shellSeekCommand) refers to shell.o(.text.shellGetCommandName) for shellGetCommandName
    shell.o(.text.shellSeekCommand) refers to strncmp.o(.text) for strncmp
    shell.o(.text.shellSeekCommand) refers to strcmp.o(.text) for strcmp
    shell.o(.ARM.exidx.text.shellSeekCommand) refers to shell.o(.text.shellSeekCommand) for [Anonymous Symbol]
    shell.o(.text.shellWritePrompt) refers to shell.o(.rodata.str1.1) for .L.str.2
    shell.o(.ARM.exidx.text.shellWritePrompt) refers to shell.o(.text.shellWritePrompt) for [Anonymous Symbol]
    shell.o(.text.shellRemove) refers to shell.o(.bss.shellList) for shellList
    shell.o(.ARM.exidx.text.shellRemove) refers to shell.o(.text.shellRemove) for [Anonymous Symbol]
    shell.o(.text.shellGetCurrent) refers to shell.o(.bss.shellList) for shellList
    shell.o(.ARM.exidx.text.shellGetCurrent) refers to shell.o(.text.shellGetCurrent) for [Anonymous Symbol]
    shell.o(.ARM.exidx.text.shellWriteString) refers to shell.o(.text.shellWriteString) for [Anonymous Symbol]
    shell.o(.text.shellPrint) refers to printfa.o(i.__0vsnprintf) for vsnprintf
    shell.o(.ARM.exidx.text.shellPrint) refers to shell.o(.text.shellPrint) for [Anonymous Symbol]
    shell.o(.ARM.exidx.text.shellCheckPermission) refers to shell.o(.text.shellCheckPermission) for [Anonymous Symbol]
    shell.o(.ARM.exidx.text.shellToHex) refers to shell.o(.text.shellToHex) for [Anonymous Symbol]
    shell.o(.ARM.exidx.text.shellToDec) refers to shell.o(.text.shellToDec) for [Anonymous Symbol]
    shell.o(.text.shellListItem) refers to shell.o(.text.shellGetCommandName) for shellGetCommandName
    shell.o(.text.shellListItem) refers to shell.o(.rodata.str1.1) for .L.str.1
    shell.o(.ARM.exidx.text.shellListItem) refers to shell.o(.text.shellListItem) for [Anonymous Symbol]
    shell.o(.text.shellGetCommandName) refers to shell.o(.bss.shellGetCommandName.buffer) for shellGetCommandName.buffer
    shell.o(.ARM.exidx.text.shellGetCommandName) refers to shell.o(.text.shellGetCommandName) for [Anonymous Symbol]
    shell.o(.text.shellListCommand) refers to shell.o(.text.shellCheckPermission) for shellCheckPermission
    shell.o(.text.shellListCommand) refers to shell.o(.text.shellListItem) for shellListItem
    shell.o(.ARM.exidx.text.shellListCommand) refers to shell.o(.text.shellListCommand) for [Anonymous Symbol]
    shell.o(.text.shellListVar) refers to shell.o(.text.shellCheckPermission) for shellCheckPermission
    shell.o(.text.shellListVar) refers to shell.o(.text.shellListItem) for shellListItem
    shell.o(.ARM.exidx.text.shellListVar) refers to shell.o(.text.shellListVar) for [Anonymous Symbol]
    shell.o(.text.shellListUser) refers to shell.o(.text.shellCheckPermission) for shellCheckPermission
    shell.o(.text.shellListUser) refers to shell.o(.text.shellListItem) for shellListItem
    shell.o(.ARM.exidx.text.shellListUser) refers to shell.o(.text.shellListUser) for [Anonymous Symbol]
    shell.o(.text.shellListKey) refers to shell.o(.text.shellCheckPermission) for shellCheckPermission
    shell.o(.text.shellListKey) refers to shell.o(.text.shellListItem) for shellListItem
    shell.o(.ARM.exidx.text.shellListKey) refers to shell.o(.text.shellListKey) for [Anonymous Symbol]
    shell.o(.text.shellListAll) refers to shell.o(.text.shellListCommand) for shellListCommand
    shell.o(.ARM.exidx.text.shellListAll) refers to shell.o(.text.shellListAll) for [Anonymous Symbol]
    shell.o(.text.shellDeleteCommandLine) refers to shell.o(.rodata.str1.1) for .L.str.3
    shell.o(.ARM.exidx.text.shellDeleteCommandLine) refers to shell.o(.text.shellDeleteCommandLine) for [Anonymous Symbol]
    shell.o(.text.shellClearCommandLine) refers to shell.o(.rodata.str1.1) for .L.str.3
    shell.o(.ARM.exidx.text.shellClearCommandLine) refers to shell.o(.text.shellClearCommandLine) for [Anonymous Symbol]
    shell.o(.text.shellInsertByte) refers to shell.o(.rodata.str1.1) for .L.str.8
    shell.o(.text.shellInsertByte) refers to shell.o(.text.shellWritePrompt) for shellWritePrompt
    shell.o(.ARM.exidx.text.shellInsertByte) refers to shell.o(.text.shellInsertByte) for [Anonymous Symbol]
    shell.o(.text.shellDeleteByte) refers to shell.o(.rodata.str1.1) for .L.str.3
    shell.o(.ARM.exidx.text.shellDeleteByte) refers to shell.o(.text.shellDeleteByte) for [Anonymous Symbol]
    shell.o(.text.shellSplit) refers to memseta.o(.text) for __aeabi_memclr4
    shell.o(.text.shellSplit) refers to shell.o(.data.pairedChars) for pairedChars
    shell.o(.ARM.exidx.text.shellSplit) refers to shell.o(.text.shellSplit) for [Anonymous Symbol]
    shell.o(.ARM.exidx.text.shellGetVarValue) refers to shell.o(.text.shellGetVarValue) for [Anonymous Symbol]
    shell.o(.text.shellSetVarValue) refers to shell.o(.text.shellShowVar) for shellShowVar
    shell.o(.ARM.exidx.text.shellSetVarValue) refers to shell.o(.text.shellSetVarValue) for [Anonymous Symbol]
    shell.o(.text.shellShowVar) refers to shell.o(.rodata.str1.4) for .L__const.shellWriteReturnValue.buffer
    shell.o(.text.shellShowVar) refers to shell.o(.text.shellGetVarValue) for shellGetVarValue
    shell.o(.text.shellShowVar) refers to shell.o(.rodata.str1.1) for .L.str.30
    shell.o(.text.shellShowVar) refers to shell.o(.text.shellToDec) for shellToDec
    shell.o(.ARM.exidx.text.shellShowVar) refers to shell.o(.text.shellShowVar) for [Anonymous Symbol]
    shell.o(.text.shellSetVar) refers to shell.o(.bss.shellList) for shellList
    shell.o(.text.shellSetVar) refers to shell.o(.text.shellSeekCommand) for shellSeekCommand
    shell.o(.text.shellSetVar) refers to shell.o(.text.shellSetVarValue) for shellSetVarValue
    shell.o(.ARM.exidx.text.shellSetVar) refers to shell.o(.text.shellSetVar) for [Anonymous Symbol]
    shell.o(.text.shellRunCommand) refers to strlen.o(.text) for strlen
    shell.o(.text.shellRunCommand) refers to shell_ext.o(.text.shellExtRun) for shellExtRun
    shell.o(.text.shellRunCommand) refers to shell.o(.text.shellWriteReturnValue) for shellWriteReturnValue
    shell.o(.text.shellRunCommand) refers to shell.o(.text.shellShowVar) for shellShowVar
    shell.o(.text.shellRunCommand) refers to shell.o(.text.shellSetUser) for shellSetUser
    shell.o(.ARM.exidx.text.shellRunCommand) refers to shell.o(.text.shellRunCommand) for [Anonymous Symbol]
    shell.o(.text.shellWriteReturnValue) refers to shell.o(.rodata.str1.4) for .L__const.shellWriteReturnValue.buffer
    shell.o(.text.shellWriteReturnValue) refers to shell.o(.text.shellToDec) for shellToDec
    shell.o(.text.shellWriteReturnValue) refers to shell.o(.rodata.str1.1) for .L.str.31
    shell.o(.ARM.exidx.text.shellWriteReturnValue) refers to shell.o(.text.shellWriteReturnValue) for [Anonymous Symbol]
    shell.o(.text.shellNormalInput) refers to shell.o(.text.shellInsertByte) for shellInsertByte
    shell.o(.ARM.exidx.text.shellNormalInput) refers to shell.o(.text.shellNormalInput) for [Anonymous Symbol]
    shell.o(.text.shellExec) refers to strcmp.o(.text) for strcmp
    shell.o(.text.shellExec) refers to shell.o(.rodata.str1.1) for .L.str.7
    shell.o(.text.shellExec) refers to shell.o(.text.shellSplit) for shellSplit
    shell.o(.text.shellExec) refers to shell.o(.text.shellSeekCommand) for shellSeekCommand
    shell.o(.text.shellExec) refers to shell.o(.text.shellRunCommand) for shellRunCommand
    shell.o(.ARM.exidx.text.shellExec) refers to shell.o(.text.shellExec) for [Anonymous Symbol]
    shell.o(.text.shellUp) refers to shell.o(.text.shellHistory) for shellHistory
    shell.o(.ARM.exidx.text.shellUp) refers to shell.o(.text.shellUp) for [Anonymous Symbol]
    shell.o(.text.shellHistory) refers to shell.o(.text.shellClearCommandLine) for shellClearCommandLine
    shell.o(.ARM.exidx.text.shellHistory) refers to shell.o(.text.shellHistory) for [Anonymous Symbol]
    shell.o(.text.shellDown) refers to shell.o(.text.shellHistory) for shellHistory
    shell.o(.ARM.exidx.text.shellDown) refers to shell.o(.text.shellDown) for [Anonymous Symbol]
    shell.o(.ARM.exidx.text.shellRight) refers to shell.o(.text.shellRight) for [Anonymous Symbol]
    shell.o(.ARM.exidx.text.shellLeft) refers to shell.o(.text.shellLeft) for [Anonymous Symbol]
    shell.o(.text.shellTab) refers to shell.o(.text.shellCheckPermission) for shellCheckPermission
    shell.o(.text.shellTab) refers to shell.o(.text.shellGetCommandName) for shellGetCommandName
    shell.o(.text.shellTab) refers to shell.o(.rodata.str1.1) for .L.str.2
    shell.o(.text.shellTab) refers to shell.o(.text.shellListItem) for shellListItem
    shell.o(.text.shellTab) refers to shell.o(.text.shellClearCommandLine) for shellClearCommandLine
    shell.o(.text.shellTab) refers to shell.o(.text.shellListCommand) for shellListCommand
    shell.o(.text.shellTab) refers to shell.o(.text.shellWritePrompt) for shellWritePrompt
    shell.o(.ARM.exidx.text.shellTab) refers to shell.o(.text.shellTab) for [Anonymous Symbol]
    shell.o(.text.shellBackspace) refers to shell.o(.text.shellDeleteByte) for shellDeleteByte
    shell.o(.ARM.exidx.text.shellBackspace) refers to shell.o(.text.shellBackspace) for [Anonymous Symbol]
    shell.o(.text.shellDelete) refers to shell.o(.text.shellDeleteByte) for shellDeleteByte
    shell.o(.ARM.exidx.text.shellDelete) refers to shell.o(.text.shellDelete) for [Anonymous Symbol]
    shell.o(.text.shellEnter) refers to shell.o(.text.shellExec) for shellExec
    shell.o(.text.shellEnter) refers to shell.o(.text.shellWritePrompt) for shellWritePrompt
    shell.o(.ARM.exidx.text.shellEnter) refers to shell.o(.text.shellEnter) for [Anonymous Symbol]
    shell.o(.text.shellHelp) refers to shell.o(.bss.shellList) for shellList
    shell.o(.text.shellHelp) refers to shell.o(.text.shellListCommand) for shellListCommand
    shell.o(.text.shellHelp) refers to shell.o(.text.shellSeekCommand) for shellSeekCommand
    shell.o(.text.shellHelp) refers to shell.o(.text.shellGetCommandName) for shellGetCommandName
    shell.o(.text.shellHelp) refers to shell.o(.rodata.str1.1) for .L.str.13
    shell.o(.ARM.exidx.text.shellHelp) refers to shell.o(.text.shellHelp) for [Anonymous Symbol]
    shell.o(.text.shellHandler) refers to shell.o(.text.shellCheckPermission) for shellCheckPermission
    shell.o(.text.shellHandler) refers to shell.o(.text.shellInsertByte) for shellInsertByte
    shell.o(.ARM.exidx.text.shellHandler) refers to shell.o(.text.shellHandler) for [Anonymous Symbol]
    shell.o(.text.shellWriteEndLine) refers to shell.o(.text.shellWritePrompt) for shellWritePrompt
    shell.o(.ARM.exidx.text.shellWriteEndLine) refers to shell.o(.text.shellWriteEndLine) for [Anonymous Symbol]
    shell.o(.text.shellTask) refers to shell.o(.text.shellHandler) for shellHandler
    shell.o(.ARM.exidx.text.shellTask) refers to shell.o(.text.shellTask) for [Anonymous Symbol]
    shell.o(.text.shellUsers) refers to shell.o(.bss.shellList) for shellList
    shell.o(.text.shellUsers) refers to shell.o(.text.shellListUser) for shellListUser
    shell.o(.ARM.exidx.text.shellUsers) refers to shell.o(.text.shellUsers) for [Anonymous Symbol]
    shell.o(.text.shellCmds) refers to shell.o(.bss.shellList) for shellList
    shell.o(.text.shellCmds) refers to shell.o(.text.shellListCommand) for shellListCommand
    shell.o(.ARM.exidx.text.shellCmds) refers to shell.o(.text.shellCmds) for [Anonymous Symbol]
    shell.o(.text.shellVars) refers to shell.o(.bss.shellList) for shellList
    shell.o(.text.shellVars) refers to shell.o(.text.shellListVar) for shellListVar
    shell.o(.ARM.exidx.text.shellVars) refers to shell.o(.text.shellVars) for [Anonymous Symbol]
    shell.o(.text.shellKeys) refers to shell.o(.bss.shellList) for shellList
    shell.o(.text.shellKeys) refers to shell.o(.text.shellListKey) for shellListKey
    shell.o(.ARM.exidx.text.shellKeys) refers to shell.o(.text.shellKeys) for [Anonymous Symbol]
    shell.o(.text.shellClear) refers to shell.o(.bss.shellList) for shellList
    shell.o(.text.shellClear) refers to shell.o(.rodata.str1.1) for .L.str.21
    shell.o(.ARM.exidx.text.shellClear) refers to shell.o(.text.shellClear) for [Anonymous Symbol]
    shell.o(.text.shellRun) refers to strlen.o(.text) for strlen
    shell.o(.text.shellRun) refers to shell.o(.rodata.str1.1) for .L.str.8
    shell.o(.text.shellRun) refers to shell.o(.text.shellExec) for shellExec
    shell.o(.ARM.exidx.text.shellRun) refers to shell.o(.text.shellRun) for [Anonymous Symbol]
    shell.o(shellCommand) refers to shell.o(.rodata.shellCmdDefaultUser) for shellCmdDefaultUser
    shell.o(shellCommand) refers to shell.o(.rodata.shellPasswordDefaultUser) for shellPasswordDefaultUser
    shell.o(shellCommand) refers to shell.o(.rodata.shellDesDefaultUser) for shellDesDefaultUser
    shell.o(shellCommand) refers to shell.o(.rodata.shellCmdsetVar) for shellCmdsetVar
    shell.o(shellCommand) refers to shell.o(.text.shellSetVar) for shellSetVar
    shell.o(shellCommand) refers to shell.o(.rodata.shellDescsetVar) for shellDescsetVar
    shell.o(shellCommand) refers to shell.o(.text.shellUp) for shellUp
    shell.o(shellCommand) refers to shell.o(.rodata.shellDesc0x1B5B4100) for shellDesc0x1B5B4100
    shell.o(shellCommand) refers to shell.o(.text.shellDown) for shellDown
    shell.o(shellCommand) refers to shell.o(.rodata.shellDesc0x1B5B4200) for shellDesc0x1B5B4200
    shell.o(shellCommand) refers to shell.o(.text.shellRight) for shellRight
    shell.o(shellCommand) refers to shell.o(.rodata.shellDesc0x1B5B4300) for shellDesc0x1B5B4300
    shell.o(shellCommand) refers to shell.o(.text.shellLeft) for shellLeft
    shell.o(shellCommand) refers to shell.o(.rodata.shellDesc0x1B5B4400) for shellDesc0x1B5B4400
    shell.o(shellCommand) refers to shell.o(.text.shellTab) for shellTab
    shell.o(shellCommand) refers to shell.o(.rodata.shellDesc0x09000000) for shellDesc0x09000000
    shell.o(shellCommand) refers to shell.o(.text.shellBackspace) for shellBackspace
    shell.o(shellCommand) refers to shell.o(.rodata.shellDesc0x08000000) for shellDesc0x08000000
    shell.o(shellCommand) refers to shell.o(.text.shellBackspace) for shellBackspace
    shell.o(shellCommand) refers to shell.o(.rodata.shellDesc0x7F000000) for shellDesc0x7F000000
    shell.o(shellCommand) refers to shell.o(.text.shellDelete) for shellDelete
    shell.o(shellCommand) refers to shell.o(.rodata.shellDesc0x1B5B337E) for shellDesc0x1B5B337E
    shell.o(shellCommand) refers to shell.o(.text.shellEnter) for shellEnter
    shell.o(shellCommand) refers to shell.o(.rodata.shellDesc0x0A000000) for shellDesc0x0A000000
    shell.o(shellCommand) refers to shell.o(.text.shellEnter) for shellEnter
    shell.o(shellCommand) refers to shell.o(.rodata.shellDesc0x0D000000) for shellDesc0x0D000000
    shell.o(shellCommand) refers to shell.o(.rodata.shellCmdhelp) for shellCmdhelp
    shell.o(shellCommand) refers to shell.o(.text.shellHelp) for shellHelp
    shell.o(shellCommand) refers to shell.o(.rodata.shellDeschelp) for shellDeschelp
    shell.o(shellCommand) refers to shell.o(.rodata.shellCmdusers) for shellCmdusers
    shell.o(shellCommand) refers to shell.o(.text.shellUsers) for shellUsers
    shell.o(shellCommand) refers to shell.o(.rodata.shellDescusers) for shellDescusers
    shell.o(shellCommand) refers to shell.o(.rodata.shellCmdcmds) for shellCmdcmds
    shell.o(shellCommand) refers to shell.o(.text.shellCmds) for shellCmds
    shell.o(shellCommand) refers to shell.o(.rodata.shellDesccmds) for shellDesccmds
    shell.o(shellCommand) refers to shell.o(.rodata.shellCmdvars) for shellCmdvars
    shell.o(shellCommand) refers to shell.o(.text.shellVars) for shellVars
    shell.o(shellCommand) refers to shell.o(.rodata.shellDescvars) for shellDescvars
    shell.o(shellCommand) refers to shell.o(.rodata.shellCmdkeys) for shellCmdkeys
    shell.o(shellCommand) refers to shell.o(.text.shellKeys) for shellKeys
    shell.o(shellCommand) refers to shell.o(.rodata.shellDesckeys) for shellDesckeys
    shell.o(shellCommand) refers to shell.o(.rodata.shellCmdclear) for shellCmdclear
    shell.o(shellCommand) refers to shell.o(.text.shellClear) for shellClear
    shell.o(shellCommand) refers to shell.o(.rodata.shellDescclear) for shellDescclear
    shell_companion.o(.ARM.exidx.text.shellCompanionAdd) refers to shell_companion.o(.text.shellCompanionAdd) for [Anonymous Symbol]
    shell_companion.o(.ARM.exidx.text.shellCompanionDel) refers to shell_companion.o(.text.shellCompanionDel) for [Anonymous Symbol]
    shell_companion.o(.ARM.exidx.text.shellCompanionGet) refers to shell_companion.o(.text.shellCompanionGet) for [Anonymous Symbol]
    shell_ext.o(.text.shellExtParsePara) refers to shell.o(.text.shellSeekCommand) for shellSeekCommand
    shell_ext.o(.text.shellExtParsePara) refers to shell.o(.text.shellGetVarValue) for shellGetVarValue
    shell_ext.o(.text.shellExtParsePara) refers to shell_ext.o(.text.shellExtParseChar) for shellExtParseChar
    shell_ext.o(.ARM.exidx.text.shellExtParsePara) refers to shell_ext.o(.text.shellExtParsePara) for [Anonymous Symbol]
    shell_ext.o(.ARM.exidx.text.shellExtParseChar) refers to shell_ext.o(.text.shellExtParseChar) for [Anonymous Symbol]
    shell_ext.o(.text.shellExtRun) refers to memseta.o(.text) for __aeabi_memclr4
    shell_ext.o(.text.shellExtRun) refers to shell_ext.o(.text.shellExtParsePara) for shellExtParsePara
    shell_ext.o(.ARM.exidx.text.shellExtRun) refers to shell_ext.o(.text.shellExtRun) for [Anonymous Symbol]
    shell_port_1.o(.text.userShellWrite) refers to hal_data.o(.rodata.g_uart9) for g_uart9
    shell_port_1.o(.text.userShellWrite) refers to r_sci_uart.o(.text.uart9_wait_for_tx) for uart9_wait_for_tx
    shell_port_1.o(.ARM.exidx.text.userShellWrite) refers to shell_port_1.o(.text.userShellWrite) for [Anonymous Symbol]
    shell_port_1.o(.ARM.exidx.text.userShellRead) refers to shell_port_1.o(.text.userShellRead) for [Anonymous Symbol]
    shell_port_1.o(.ARM.exidx.text.userShellLock) refers to shell_port_1.o(.text.userShellLock) for [Anonymous Symbol]
    shell_port_1.o(.ARM.exidx.text.userShellUnlock) refers to shell_port_1.o(.text.userShellUnlock) for [Anonymous Symbol]
    shell_port_1.o(.text.uartLogWrite) refers to shell_port_1.o(.data.uartLog) for uartLog
    shell_port_1.o(.text.uartLogWrite) refers to shell.o(.text.shellWriteEndLine) for shellWriteEndLine
    shell_port_1.o(.ARM.exidx.text.uartLogWrite) refers to shell_port_1.o(.text.uartLogWrite) for [Anonymous Symbol]
    shell_port_1.o(.text.userShellInit) refers to shell_port_1.o(.bss.shell) for shell
    shell_port_1.o(.text.userShellInit) refers to shell_port_1.o(.text.userShellWrite) for userShellWrite
    shell_port_1.o(.text.userShellInit) refers to shell_port_1.o(.bss.shellBuffer) for shellBuffer
    shell_port_1.o(.text.userShellInit) refers to shell.o(.text.shellInit) for shellInit
    shell_port_1.o(.text.userShellInit) refers to shell_port_1.o(.data.uartLog) for uartLog
    shell_port_1.o(.text.userShellInit) refers to log.o(.text.logRegister) for logRegister
    shell_port_1.o(.ARM.exidx.text.userShellInit) refers to shell_port_1.o(.text.userShellInit) for [Anonymous Symbol]
    shell_port_1.o(.data.uartLog) refers to shell_port_1.o(.text.uartLogWrite) for uartLogWrite
    shell_cmds.o(.text) refers (Special) to _scanf_int.o(.text) for _scanf_int
    shell_cmds.o(.text.cmd_rd) refers (Special) to _scanf_int.o(.text) for _scanf_int
    shell_cmds.o(.text.cmd_rd) refers to shell_port_1.o(.bss.shell) for shell
    shell_cmds.o(.text.cmd_rd) refers to shell.o(.text.shellPrint) for shellPrint
    shell_cmds.o(.text.cmd_rd) refers to shell_cmds.o(.rodata.str1.1) for .L.str.2
    shell_cmds.o(.text.cmd_rd) refers to __0sscanf.o(.text) for __0sscanf
    shell_cmds.o(.text.cmd_rd) refers to puts.o(i.puts) for puts
    shell_cmds.o(.ARM.exidx.text.cmd_rd) refers (Special) to _scanf_int.o(.text) for _scanf_int
    shell_cmds.o(.ARM.exidx.text.cmd_rd) refers to shell_cmds.o(.text.cmd_rd) for [Anonymous Symbol]
    shell_cmds.o(.text.cmd_wr) refers (Special) to _scanf_int.o(.text) for _scanf_int
    shell_cmds.o(.text.cmd_wr) refers to shell_port_1.o(.bss.shell) for shell
    shell_cmds.o(.text.cmd_wr) refers to shell_cmds.o(.rodata.str1.1) for .L.str.15
    shell_cmds.o(.text.cmd_wr) refers to shell.o(.text.shellPrint) for shellPrint
    shell_cmds.o(.text.cmd_wr) refers to __0sscanf.o(.text) for __0sscanf
    shell_cmds.o(.ARM.exidx.text.cmd_wr) refers (Special) to _scanf_int.o(.text) for _scanf_int
    shell_cmds.o(.ARM.exidx.text.cmd_wr) refers to shell_cmds.o(.text.cmd_wr) for [Anonymous Symbol]
    shell_cmds.o(.text.cmd_hex2dec) refers (Special) to _scanf_int.o(.text) for _scanf_int
    shell_cmds.o(.text.cmd_hex2dec) refers to shell_port_1.o(.bss.shell) for shell
    shell_cmds.o(.text.cmd_hex2dec) refers to shell_cmds.o(.rodata.str1.1) for .L.str.2
    shell_cmds.o(.text.cmd_hex2dec) refers to __0sscanf.o(.text) for __0sscanf
    shell_cmds.o(.text.cmd_hex2dec) refers to shell.o(.text.shellPrint) for shellPrint
    shell_cmds.o(.ARM.exidx.text.cmd_hex2dec) refers (Special) to _scanf_int.o(.text) for _scanf_int
    shell_cmds.o(.ARM.exidx.text.cmd_hex2dec) refers to shell_cmds.o(.text.cmd_hex2dec) for [Anonymous Symbol]
    shell_cmds.o(.text.cmd_time) refers (Special) to _scanf_int.o(.text) for _scanf_int
    shell_cmds.o(.text.cmd_time) refers to shell_port_1.o(.bss.shell) for shell
    shell_cmds.o(.text.cmd_time) refers to shell_cmds.o(.rodata.str1.1) for .L.str.27
    shell_cmds.o(.text.cmd_time) refers to shell.o(.text.shellPrint) for shellPrint
    shell_cmds.o(.text.cmd_time) refers to shell.o(.text.shellSeekCommand) for shellSeekCommand
    shell_cmds.o(.text.cmd_time) refers to shell_cmds.o(.bss.shell_get_ts_ns.cyc) for shell_get_ts_ns.cyc
    shell_cmds.o(.text.cmd_time) refers to uldiv.o(.text) for __aeabi_uldivmod
    shell_cmds.o(.ARM.exidx.text.cmd_time) refers (Special) to _scanf_int.o(.text) for _scanf_int
    shell_cmds.o(.ARM.exidx.text.cmd_time) refers to shell_cmds.o(.text.cmd_time) for [Anonymous Symbol]
    shell_cmds.o(.rodata.str1.1) refers (Special) to _scanf_int.o(.text) for _scanf_int
    shell_cmds.o(.rodata.shellCmdrd) refers (Special) to _scanf_int.o(.text) for _scanf_int
    shell_cmds.o(.rodata.shellDescrd) refers (Special) to _scanf_int.o(.text) for _scanf_int
    shell_cmds.o(shellCommand) refers (Special) to _scanf_int.o(.text) for _scanf_int
    shell_cmds.o(shellCommand) refers to shell_cmds.o(.rodata.shellCmdrd) for shellCmdrd
    shell_cmds.o(shellCommand) refers to shell_cmds.o(.text.cmd_rd) for cmd_rd
    shell_cmds.o(shellCommand) refers to shell_cmds.o(.rodata.shellDescrd) for shellDescrd
    shell_cmds.o(.rodata.shellCmdwr) refers (Special) to _scanf_int.o(.text) for _scanf_int
    shell_cmds.o(.rodata.shellDescwr) refers (Special) to _scanf_int.o(.text) for _scanf_int
    shell_cmds.o(shellCommand) refers (Special) to _scanf_int.o(.text) for _scanf_int
    shell_cmds.o(shellCommand) refers to shell_cmds.o(.rodata.shellCmdwr) for shellCmdwr
    shell_cmds.o(shellCommand) refers to shell_cmds.o(.text.cmd_wr) for cmd_wr
    shell_cmds.o(shellCommand) refers to shell_cmds.o(.rodata.shellDescwr) for shellDescwr
    shell_cmds.o(.rodata.shellCmdhex2dec) refers (Special) to _scanf_int.o(.text) for _scanf_int
    shell_cmds.o(.rodata.shellDeschex2dec) refers (Special) to _scanf_int.o(.text) for _scanf_int
    shell_cmds.o(shellCommand) refers (Special) to _scanf_int.o(.text) for _scanf_int
    shell_cmds.o(shellCommand) refers to shell_cmds.o(.rodata.shellCmdhex2dec) for shellCmdhex2dec
    shell_cmds.o(shellCommand) refers to shell_cmds.o(.text.cmd_hex2dec) for cmd_hex2dec
    shell_cmds.o(shellCommand) refers to shell_cmds.o(.rodata.shellDeschex2dec) for shellDeschex2dec
    shell_cmds.o(.rodata.shellCmdtimecal) refers (Special) to _scanf_int.o(.text) for _scanf_int
    shell_cmds.o(.rodata.shellDesctimecal) refers (Special) to _scanf_int.o(.text) for _scanf_int
    shell_cmds.o(shellCommand) refers (Special) to _scanf_int.o(.text) for _scanf_int
    shell_cmds.o(shellCommand) refers to shell_cmds.o(.rodata.shellCmdtimecal) for shellCmdtimecal
    shell_cmds.o(shellCommand) refers to shell_cmds.o(.text.cmd_time) for cmd_time
    shell_cmds.o(shellCommand) refers to shell_cmds.o(.rodata.shellDesctimecal) for shellDesctimecal
    shell_cmds.o(.bss.shell_get_ts_ns.cyc) refers (Special) to _scanf_int.o(.text) for _scanf_int
    log.o(.text.logRegister) refers to shell_companion.o(.text.shellCompanionAdd) for shellCompanionAdd
    log.o(.text.logRegister) refers to log.o(.bss.logList) for logList
    log.o(.ARM.exidx.text.logRegister) refers to log.o(.text.logRegister) for [Anonymous Symbol]
    log.o(.text.logUnRegister) refers to log.o(.bss.logList) for logList
    log.o(.ARM.exidx.text.logUnRegister) refers to log.o(.text.logUnRegister) for [Anonymous Symbol]
    log.o(.text.logSetLevel) refers to hal_entry.o(.bss.SysTickms) for SysTickms
    log.o(.text.logSetLevel) refers to log.o(.rodata.str1.1) for .L.str
    log.o(.text.logSetLevel) refers to log.o(.rodata.shellCmdlogSetLevel) for shellCmdlogSetLevel
    log.o(.text.logSetLevel) refers to log.o(.text.logWrite) for logWrite
    log.o(.ARM.exidx.text.logSetLevel) refers to log.o(.text.logSetLevel) for [Anonymous Symbol]
    log.o(.text.logWrite) refers to log.o(.bss.logBuffer) for logBuffer
    log.o(.text.logWrite) refers to printfa.o(i.__0vsnprintf) for vsnprintf
    log.o(.text.logWrite) refers to log.o(.text.logWriteBuffer) for logWriteBuffer
    log.o(.ARM.exidx.text.logWrite) refers to log.o(.text.logWrite) for [Anonymous Symbol]
    log.o(.text.agencylogSetLevel) refers to shell.o(.text.shellGetCurrent) for shellGetCurrent
    log.o(.text.agencylogSetLevel) refers to shell_companion.o(.text.shellCompanionGet) for shellCompanionGet
    log.o(.text.agencylogSetLevel) refers to hal_entry.o(.bss.SysTickms) for SysTickms
    log.o(.text.agencylogSetLevel) refers to log.o(.rodata.str1.1) for .L.str
    log.o(.text.agencylogSetLevel) refers to log.o(.rodata.shellCmdlogSetLevel) for shellCmdlogSetLevel
    log.o(.text.agencylogSetLevel) refers to log.o(.text.logWrite) for logWrite
    log.o(.ARM.exidx.text.agencylogSetLevel) refers to log.o(.text.agencylogSetLevel) for [Anonymous Symbol]
    log.o(.text.logWriteBuffer) refers to log.o(.bss.logList) for logList
    log.o(.text.logWriteBuffer) refers to log.o(.bss.logBuffer) for logBuffer
    log.o(.ARM.exidx.text.logWriteBuffer) refers to log.o(.text.logWriteBuffer) for [Anonymous Symbol]
    log.o(.text.logHexDump) refers to log.o(.rodata.str1.1) for .L.str.3
    log.o(.text.logHexDump) refers to log.o(.bss.logBuffer) for logBuffer
    log.o(.text.logHexDump) refers to printfa.o(i.__0snprintf) for __2snprintf
    log.o(.text.logHexDump) refers to log.o(.text.logWriteBuffer) for logWriteBuffer
    log.o(.text.logHexDump) refers to printfa.o(i.__0sprintf) for __2sprintf
    log.o(.ARM.exidx.text.logHexDump) refers to log.o(.text.logHexDump) for [Anonymous Symbol]
    log.o(.text.agencylogHexDump) refers to shell.o(.text.shellGetCurrent) for shellGetCurrent
    log.o(.text.agencylogHexDump) refers to shell_companion.o(.text.shellCompanionGet) for shellCompanionGet
    log.o(.text.agencylogHexDump) refers to log.o(.text.logHexDump) for logHexDump
    log.o(.ARM.exidx.text.agencylogHexDump) refers to log.o(.text.agencylogHexDump) for [Anonymous Symbol]
    log.o(.text.logSwitchLevel) refers to shell_companion.o(.text.shellCompanionGet) for shellCompanionGet
    log.o(.text.logSwitchLevel) refers to log.o(.text.logWrite) for logWrite
    log.o(.ARM.exidx.text.logSwitchLevel) refers to log.o(.text.logSwitchLevel) for [Anonymous Symbol]
    log.o(shellCommand) refers to log.o(.rodata.shellCmdlogSetLevel) for shellCmdlogSetLevel
    log.o(shellCommand) refers to log.o(.text.agencylogSetLevel) for agencylogSetLevel
    log.o(shellCommand) refers to log.o(.rodata.shellDesclogSetLevel) for shellDesclogSetLevel
    log.o(shellCommand) refers to log.o(.rodata.shellCmdhexdump) for shellCmdhexdump
    log.o(shellCommand) refers to log.o(.text.agencylogHexDump) for agencylogHexDump
    log.o(shellCommand) refers to log.o(.rodata.shellDeschexdump) for shellDeschexdump
    log.o(shellCommand) refers to log.o(.text.logSwitchLevel) for logSwitchLevel
    log.o(shellCommand) refers to log.o(.rodata.shellDesc0x04000000) for shellDesc0x04000000
    lwrb.o(.ARM.exidx.text.lwrb_init) refers to lwrb.o(.text.lwrb_init) for [Anonymous Symbol]
    lwrb.o(.ARM.exidx.text.lwrb_is_ready) refers to lwrb.o(.text.lwrb_is_ready) for [Anonymous Symbol]
    lwrb.o(.ARM.exidx.text.lwrb_free) refers to lwrb.o(.text.lwrb_free) for [Anonymous Symbol]
    lwrb.o(.ARM.exidx.text.lwrb_set_evt_fn) refers to lwrb.o(.text.lwrb_set_evt_fn) for [Anonymous Symbol]
    lwrb.o(.ARM.exidx.text.lwrb_set_arg) refers to lwrb.o(.text.lwrb_set_arg) for [Anonymous Symbol]
    lwrb.o(.ARM.exidx.text.lwrb_get_arg) refers to lwrb.o(.text.lwrb_get_arg) for [Anonymous Symbol]
    lwrb.o(.text.lwrb_write) refers to lwrb.o(.text.lwrb_write_ex) for lwrb_write_ex
    lwrb.o(.ARM.exidx.text.lwrb_write) refers to lwrb.o(.text.lwrb_write) for [Anonymous Symbol]
    lwrb.o(.text.lwrb_write_ex) refers to memcpya.o(.text) for __aeabi_memcpy
    lwrb.o(.ARM.exidx.text.lwrb_write_ex) refers to lwrb.o(.text.lwrb_write_ex) for [Anonymous Symbol]
    lwrb.o(.ARM.exidx.text.lwrb_get_free) refers to lwrb.o(.text.lwrb_get_free) for [Anonymous Symbol]
    lwrb.o(.text.lwrb_read) refers to lwrb.o(.text.lwrb_read_ex) for lwrb_read_ex
    lwrb.o(.ARM.exidx.text.lwrb_read) refers to lwrb.o(.text.lwrb_read) for [Anonymous Symbol]
    lwrb.o(.text.lwrb_read_ex) refers to memcpya.o(.text) for __aeabi_memcpy
    lwrb.o(.ARM.exidx.text.lwrb_read_ex) refers to lwrb.o(.text.lwrb_read_ex) for [Anonymous Symbol]
    lwrb.o(.ARM.exidx.text.lwrb_get_full) refers to lwrb.o(.text.lwrb_get_full) for [Anonymous Symbol]
    lwrb.o(.text.lwrb_peek) refers to memcpya.o(.text) for __aeabi_memcpy
    lwrb.o(.ARM.exidx.text.lwrb_peek) refers to lwrb.o(.text.lwrb_peek) for [Anonymous Symbol]
    lwrb.o(.ARM.exidx.text.lwrb_reset) refers to lwrb.o(.text.lwrb_reset) for [Anonymous Symbol]
    lwrb.o(.ARM.exidx.text.lwrb_get_linear_block_read_address) refers to lwrb.o(.text.lwrb_get_linear_block_read_address) for [Anonymous Symbol]
    lwrb.o(.ARM.exidx.text.lwrb_get_linear_block_read_length) refers to lwrb.o(.text.lwrb_get_linear_block_read_length) for [Anonymous Symbol]
    lwrb.o(.ARM.exidx.text.lwrb_skip) refers to lwrb.o(.text.lwrb_skip) for [Anonymous Symbol]
    lwrb.o(.ARM.exidx.text.lwrb_get_linear_block_write_address) refers to lwrb.o(.text.lwrb_get_linear_block_write_address) for [Anonymous Symbol]
    lwrb.o(.ARM.exidx.text.lwrb_get_linear_block_write_length) refers to lwrb.o(.text.lwrb_get_linear_block_write_length) for [Anonymous Symbol]
    lwrb.o(.ARM.exidx.text.lwrb_advance) refers to lwrb.o(.text.lwrb_advance) for [Anonymous Symbol]
    lwrb.o(.ARM.exidx.text.lwrb_find) refers to lwrb.o(.text.lwrb_find) for [Anonymous Symbol]
    multi_button.o(.text.button_init) refers to memseta.o(.text) for __aeabi_memclr4
    multi_button.o(.ARM.exidx.text.button_init) refers to multi_button.o(.text.button_init) for [Anonymous Symbol]
    multi_button.o(.ARM.exidx.text.button_attach) refers to multi_button.o(.text.button_attach) for [Anonymous Symbol]
    multi_button.o(.ARM.exidx.text.get_button_event) refers to multi_button.o(.text.get_button_event) for [Anonymous Symbol]
    multi_button.o(.text.button_start) refers to multi_button.o(.bss.head_handle) for head_handle
    multi_button.o(.ARM.exidx.text.button_start) refers to multi_button.o(.text.button_start) for [Anonymous Symbol]
    multi_button.o(.text.button_stop) refers to multi_button.o(.bss.head_handle) for head_handle
    multi_button.o(.ARM.exidx.text.button_stop) refers to multi_button.o(.text.button_stop) for [Anonymous Symbol]
    multi_button.o(.text.button_ticks) refers to multi_button.o(.bss.head_handle) for head_handle
    multi_button.o(.ARM.exidx.text.button_ticks) refers to multi_button.o(.text.button_ticks) for [Anonymous Symbol]
    startup.o(.text.Reset_Handler) refers to system.o(.text.SystemInit) for SystemInit
    startup.o(.text.Reset_Handler) refers to main.o(.text.main) for main
    startup.o(.ARM.exidx.text.Reset_Handler) refers to startup.o(.text.Reset_Handler) for [Anonymous Symbol]
    startup.o(.ARM.exidx.text.Default_Handler) refers to startup.o(.text.Default_Handler) for [Anonymous Symbol]
    startup.o(.fixed_vectors) refers to startup.o(.bss.stack) for [Anonymous Symbol]
    startup.o(.fixed_vectors) refers to startup.o(.text.Reset_Handler) for Reset_Handler
    startup.o(.fixed_vectors) refers to bsp_group_irq.o(.text.NMI_Handler) for NMI_Handler
    startup.o(.fixed_vectors) refers to startup.o(.text.Default_Handler) for HardFault_Handler
    startup.o(.fixed_vectors) refers to hal_entry.o(.text.SysTick_Handler) for SysTick_Handler
    system.o(.text.SystemInit) refers to startup.o(.fixed_vectors) for __Vectors
    system.o(.text.SystemInit) refers to hal_entry.o(.text.R_BSP_WarmStart) for R_BSP_WarmStart
    system.o(.text.SystemInit) refers to bsp_clocks.o(.text.bsp_clock_init) for bsp_clock_init
    system.o(.text.SystemInit) refers to memseta.o(.text) for __aeabi_memclr4
    system.o(.text.SystemInit) refers to memcpya.o(.text) for __aeabi_memcpy4
    system.o(.text.SystemInit) refers to bsp_clocks.o(.text.SystemCoreClockUpdate) for SystemCoreClockUpdate
    system.o(.text.SystemInit) refers to bsp_clocks.o(.text.R_BSP_Init_RTC) for R_BSP_Init_RTC
    system.o(.text.SystemInit) refers to bsp_register_protection.o(.text.R_BSP_RegisterProtectDisable) for R_BSP_RegisterProtectDisable
    system.o(.text.SystemInit) refers to bsp_register_protection.o(.text.R_BSP_RegisterProtectEnable) for R_BSP_RegisterProtectEnable
    system.o(.text.SystemInit) refers to bsp_irq.o(.text.bsp_irq_cfg) for bsp_irq_cfg
    system.o(.text.SystemInit) refers to bsp_common.o(.text.bsp_init_internal) for bsp_init
    system.o(.ARM.exidx.text.SystemInit) refers to system.o(.text.SystemInit) for [Anonymous Symbol]
    system.o(.ARM.exidx.text.R_BSP_WarmStart) refers to system.o(.text.R_BSP_WarmStart) for [Anonymous Symbol]
    bsp_clocks.o(.ARM.exidx.text.bsp_prv_operating_mode_set) refers to bsp_clocks.o(.text.bsp_prv_operating_mode_set) for [Anonymous Symbol]
    bsp_clocks.o(.text.bsp_prv_prepare_pll) refers to bsp_clocks.o(.bss.noinit) for g_clock_freq
    bsp_clocks.o(.ARM.exidx.text.bsp_prv_prepare_pll) refers to bsp_clocks.o(.text.bsp_prv_prepare_pll) for [Anonymous Symbol]
    bsp_clocks.o(.text.SystemCoreClockUpdate) refers to bsp_clocks.o(.bss.noinit) for g_clock_freq
    bsp_clocks.o(.text.SystemCoreClockUpdate) refers to system.o(.bss.SystemCoreClock) for SystemCoreClock
    bsp_clocks.o(.ARM.exidx.text.SystemCoreClockUpdate) refers to bsp_clocks.o(.text.SystemCoreClockUpdate) for [Anonymous Symbol]
    bsp_clocks.o(.ARM.exidx.text.prv_clock_dividers_set) refers to bsp_clocks.o(.text.prv_clock_dividers_set) for [Anonymous Symbol]
    bsp_clocks.o(.text.bsp_prv_clock_set) refers to bsp_clocks.o(.bss.noinit) for g_clock_freq
    bsp_clocks.o(.text.bsp_prv_clock_set) refers to system.o(.bss.SystemCoreClock) for SystemCoreClock
    bsp_clocks.o(.ARM.exidx.text.bsp_prv_clock_set) refers to bsp_clocks.o(.text.bsp_prv_clock_set) for [Anonymous Symbol]
    bsp_clocks.o(.text.bsp_clock_init) refers to bsp_clocks.o(.bss.noinit) for g_clock_freq
    bsp_clocks.o(.text.bsp_clock_init) refers to system.o(.bss.SystemCoreClock) for SystemCoreClock
    bsp_clocks.o(.text.bsp_clock_init) refers to bsp_delay.o(.text.R_BSP_SoftwareDelay) for R_BSP_SoftwareDelay
    bsp_clocks.o(.text.bsp_clock_init) refers to bsp_clocks.o(.text.R_BSP_SubClockStabilizeWaitAfterReset) for R_BSP_SubClockStabilizeWaitAfterReset
    bsp_clocks.o(.ARM.exidx.text.bsp_clock_init) refers to bsp_clocks.o(.text.bsp_clock_init) for [Anonymous Symbol]
    bsp_clocks.o(.text.R_BSP_SubClockStabilizeWait) refers to bsp_delay.o(.text.R_BSP_SoftwareDelay) for R_BSP_SoftwareDelay
    bsp_clocks.o(.ARM.exidx.text.R_BSP_SubClockStabilizeWait) refers to bsp_clocks.o(.text.R_BSP_SubClockStabilizeWait) for [Anonymous Symbol]
    bsp_clocks.o(.ARM.exidx.text.R_BSP_SubClockStabilizeWaitAfterReset) refers to bsp_clocks.o(.text.R_BSP_SubClockStabilizeWaitAfterReset) for [Anonymous Symbol]
    bsp_clocks.o(.ARM.exidx.text.R_BSP_OctaclkUpdate) refers to bsp_clocks.o(.text.R_BSP_OctaclkUpdate) for [Anonymous Symbol]
    bsp_clocks.o(.text.R_BSP_SourceClockHzGet) refers to bsp_clocks.o(.bss.noinit) for g_clock_freq
    bsp_clocks.o(.ARM.exidx.text.R_BSP_SourceClockHzGet) refers to bsp_clocks.o(.text.R_BSP_SourceClockHzGet) for [Anonymous Symbol]
    bsp_clocks.o(.text.R_BSP_Init_RTC) refers to bsp_delay.o(.text.R_BSP_SoftwareDelay) for R_BSP_SoftwareDelay
    bsp_clocks.o(.text.R_BSP_Init_RTC) refers to bsp_register_protection.o(.text.R_BSP_RegisterProtectDisable) for R_BSP_RegisterProtectDisable
    bsp_clocks.o(.text.R_BSP_Init_RTC) refers to bsp_register_protection.o(.text.R_BSP_RegisterProtectEnable) for R_BSP_RegisterProtectEnable
    bsp_clocks.o(.ARM.exidx.text.R_BSP_Init_RTC) refers to bsp_clocks.o(.text.R_BSP_Init_RTC) for [Anonymous Symbol]
    bsp_common.o(.ARM.exidx.text.bsp_init_internal) refers to bsp_common.o(.text.bsp_init_internal) for [Anonymous Symbol]
    bsp_common.o(.ARM.exidx.text.R_FSP_VersionGet) refers to bsp_common.o(.text.R_FSP_VersionGet) for [Anonymous Symbol]
    bsp_common.o(.ARM.exidx.text.__aeabi_assert) refers to bsp_common.o(.text.__aeabi_assert) for [Anonymous Symbol]
    bsp_delay.o(.text.R_BSP_SoftwareDelay) refers to system.o(.bss.SystemCoreClock) for SystemCoreClock
    bsp_delay.o(.text.R_BSP_SoftwareDelay) refers to bsp_delay.o(.text.bsp_prv_software_delay_loop) for bsp_prv_software_delay_loop
    bsp_delay.o(.ARM.exidx.text.R_BSP_SoftwareDelay) refers to bsp_delay.o(.text.R_BSP_SoftwareDelay) for [Anonymous Symbol]
    bsp_delay.o(.ARM.exidx.text.bsp_prv_software_delay_loop) refers to bsp_delay.o(.text.bsp_prv_software_delay_loop) for [Anonymous Symbol]
    bsp_group_irq.o(.text.R_BSP_GroupIrqWrite) refers to bsp_group_irq.o(.bss.g_bsp_group_irq_sources) for g_bsp_group_irq_sources
    bsp_group_irq.o(.ARM.exidx.text.R_BSP_GroupIrqWrite) refers to bsp_group_irq.o(.text.R_BSP_GroupIrqWrite) for [Anonymous Symbol]
    bsp_group_irq.o(.text.NMI_Handler) refers to bsp_group_irq.o(.bss.g_bsp_group_irq_sources) for g_bsp_group_irq_sources
    bsp_group_irq.o(.ARM.exidx.text.NMI_Handler) refers to bsp_group_irq.o(.text.NMI_Handler) for [Anonymous Symbol]
    bsp_irq.o(.text.bsp_irq_cfg) refers to bsp_register_protection.o(.text.R_BSP_RegisterProtectDisable) for R_BSP_RegisterProtectDisable
    bsp_irq.o(.text.bsp_irq_cfg) refers to vector_data.o(.rodata.g_interrupt_event_link_select) for g_interrupt_event_link_select
    bsp_irq.o(.text.bsp_irq_cfg) refers to bsp_register_protection.o(.text.R_BSP_RegisterProtectEnable) for R_BSP_RegisterProtectEnable
    bsp_irq.o(.ARM.exidx.text.bsp_irq_cfg) refers to bsp_irq.o(.text.bsp_irq_cfg) for [Anonymous Symbol]
    bsp_register_protection.o(.text.R_BSP_RegisterProtectEnable) refers to bsp_register_protection.o(.bss.g_protect_counters) for g_protect_counters
    bsp_register_protection.o(.text.R_BSP_RegisterProtectEnable) refers to bsp_register_protection.o(.rodata.cst8) for g_prcr_masks
    bsp_register_protection.o(.ARM.exidx.text.R_BSP_RegisterProtectEnable) refers to bsp_register_protection.o(.text.R_BSP_RegisterProtectEnable) for [Anonymous Symbol]
    bsp_register_protection.o(.text.R_BSP_RegisterProtectDisable) refers to bsp_register_protection.o(.bss.g_protect_counters) for g_protect_counters
    bsp_register_protection.o(.text.R_BSP_RegisterProtectDisable) refers to bsp_register_protection.o(.rodata.cst8) for g_prcr_masks
    bsp_register_protection.o(.ARM.exidx.text.R_BSP_RegisterProtectDisable) refers to bsp_register_protection.o(.text.R_BSP_RegisterProtectDisable) for [Anonymous Symbol]
    r_ioport.o(.text.R_IOPORT_Open) refers to r_ioport.o(.text.r_ioport_pins_config) for r_ioport_pins_config
    r_ioport.o(.ARM.exidx.text.R_IOPORT_Open) refers to r_ioport.o(.text.R_IOPORT_Open) for [Anonymous Symbol]
    r_ioport.o(.ARM.exidx.text.R_IOPORT_Close) refers to r_ioport.o(.text.R_IOPORT_Close) for [Anonymous Symbol]
    r_ioport.o(.text.R_IOPORT_PinsCfg) refers to r_ioport.o(.text.r_ioport_pins_config) for r_ioport_pins_config
    r_ioport.o(.ARM.exidx.text.R_IOPORT_PinsCfg) refers to r_ioport.o(.text.R_IOPORT_PinsCfg) for [Anonymous Symbol]
    r_ioport.o(.text.R_IOPORT_PinCfg) refers to r_ioport.o(.text.bsp_vbatt_init) for bsp_vbatt_init
    r_ioport.o(.text.R_IOPORT_PinCfg) refers to bsp_io.o(.bss.g_protect_pfswe_counter) for g_protect_pfswe_counter
    r_ioport.o(.ARM.exidx.text.R_IOPORT_PinCfg) refers to r_ioport.o(.text.R_IOPORT_PinCfg) for [Anonymous Symbol]
    r_ioport.o(.ARM.exidx.text.R_IOPORT_PinEventInputRead) refers to r_ioport.o(.text.R_IOPORT_PinEventInputRead) for [Anonymous Symbol]
    r_ioport.o(.ARM.exidx.text.R_IOPORT_PinEventOutputWrite) refers to r_ioport.o(.text.R_IOPORT_PinEventOutputWrite) for [Anonymous Symbol]
    r_ioport.o(.ARM.exidx.text.R_IOPORT_PinRead) refers to r_ioport.o(.text.R_IOPORT_PinRead) for [Anonymous Symbol]
    r_ioport.o(.ARM.exidx.text.R_IOPORT_PinWrite) refers to r_ioport.o(.text.R_IOPORT_PinWrite) for [Anonymous Symbol]
    r_ioport.o(.ARM.exidx.text.R_IOPORT_PortDirectionSet) refers to r_ioport.o(.text.R_IOPORT_PortDirectionSet) for [Anonymous Symbol]
    r_ioport.o(.ARM.exidx.text.R_IOPORT_PortEventInputRead) refers to r_ioport.o(.text.R_IOPORT_PortEventInputRead) for [Anonymous Symbol]
    r_ioport.o(.ARM.exidx.text.R_IOPORT_PortEventOutputWrite) refers to r_ioport.o(.text.R_IOPORT_PortEventOutputWrite) for [Anonymous Symbol]
    r_ioport.o(.ARM.exidx.text.R_IOPORT_PortRead) refers to r_ioport.o(.text.R_IOPORT_PortRead) for [Anonymous Symbol]
    r_ioport.o(.ARM.exidx.text.R_IOPORT_PortWrite) refers to r_ioport.o(.text.R_IOPORT_PortWrite) for [Anonymous Symbol]
    r_ioport.o(.text.r_ioport_pins_config) refers to r_ioport.o(.text.bsp_vbatt_init) for bsp_vbatt_init
    r_ioport.o(.text.r_ioport_pins_config) refers to bsp_io.o(.bss.g_protect_pfswe_counter) for g_protect_pfswe_counter
    r_ioport.o(.ARM.exidx.text.r_ioport_pins_config) refers to r_ioport.o(.text.r_ioport_pins_config) for [Anonymous Symbol]
    r_ioport.o(.text.bsp_vbatt_init) refers to bsp_register_protection.o(.text.R_BSP_RegisterProtectDisable) for R_BSP_RegisterProtectDisable
    r_ioport.o(.text.bsp_vbatt_init) refers to bsp_register_protection.o(.text.R_BSP_RegisterProtectEnable) for R_BSP_RegisterProtectEnable
    r_ioport.o(.text.bsp_vbatt_init) refers to bsp_delay.o(.text.R_BSP_SoftwareDelay) for R_BSP_SoftwareDelay
    r_ioport.o(.ARM.exidx.text.bsp_vbatt_init) refers to r_ioport.o(.text.bsp_vbatt_init) for [Anonymous Symbol]
    r_ioport.o(.rodata.g_ioport_on_ioport) refers to r_ioport.o(.text.R_IOPORT_Open) for R_IOPORT_Open
    r_ioport.o(.rodata.g_ioport_on_ioport) refers to r_ioport.o(.text.R_IOPORT_Close) for R_IOPORT_Close
    r_ioport.o(.rodata.g_ioport_on_ioport) refers to r_ioport.o(.text.R_IOPORT_PinsCfg) for R_IOPORT_PinsCfg
    r_ioport.o(.rodata.g_ioport_on_ioport) refers to r_ioport.o(.text.R_IOPORT_PinCfg) for R_IOPORT_PinCfg
    r_ioport.o(.rodata.g_ioport_on_ioport) refers to r_ioport.o(.text.R_IOPORT_PinEventInputRead) for R_IOPORT_PinEventInputRead
    r_ioport.o(.rodata.g_ioport_on_ioport) refers to r_ioport.o(.text.R_IOPORT_PinEventOutputWrite) for R_IOPORT_PinEventOutputWrite
    r_ioport.o(.rodata.g_ioport_on_ioport) refers to r_ioport.o(.text.R_IOPORT_PinRead) for R_IOPORT_PinRead
    r_ioport.o(.rodata.g_ioport_on_ioport) refers to r_ioport.o(.text.R_IOPORT_PinWrite) for R_IOPORT_PinWrite
    r_ioport.o(.rodata.g_ioport_on_ioport) refers to r_ioport.o(.text.R_IOPORT_PortDirectionSet) for R_IOPORT_PortDirectionSet
    r_ioport.o(.rodata.g_ioport_on_ioport) refers to r_ioport.o(.text.R_IOPORT_PortEventInputRead) for R_IOPORT_PortEventInputRead
    r_ioport.o(.rodata.g_ioport_on_ioport) refers to r_ioport.o(.text.R_IOPORT_PortEventOutputWrite) for R_IOPORT_PortEventOutputWrite
    r_ioport.o(.rodata.g_ioport_on_ioport) refers to r_ioport.o(.text.R_IOPORT_PortRead) for R_IOPORT_PortRead
    r_ioport.o(.rodata.g_ioport_on_ioport) refers to r_ioport.o(.text.R_IOPORT_PortWrite) for R_IOPORT_PortWrite
    r_sci_uart.o(.text.user_uart9_callback) refers to r_sci_uart.o(.bss.g_uart9_tx_complete) for g_uart9_tx_complete
    r_sci_uart.o(.text.user_uart9_callback) refers to r_sci_uart.o(.bss.g_uart9_rx_complete) for g_uart9_rx_complete
    r_sci_uart.o(.text.user_uart9_callback) refers to hal_entry.o(.bss.buff) for buff
    r_sci_uart.o(.text.user_uart9_callback) refers to lwrb.o(.text.lwrb_write) for lwrb_write
    r_sci_uart.o(.ARM.exidx.text.user_uart9_callback) refers to r_sci_uart.o(.text.user_uart9_callback) for [Anonymous Symbol]
    r_sci_uart.o(.text.uart9_wait_for_tx) refers to r_sci_uart.o(.bss.g_uart9_tx_complete) for g_uart9_tx_complete
    r_sci_uart.o(.ARM.exidx.text.uart9_wait_for_tx) refers to r_sci_uart.o(.text.uart9_wait_for_tx) for [Anonymous Symbol]
    r_sci_uart.o(.text.uart9_wait_for_rx) refers to r_sci_uart.o(.bss.g_uart9_rx_complete) for g_uart9_rx_complete
    r_sci_uart.o(.ARM.exidx.text.uart9_wait_for_rx) refers to r_sci_uart.o(.text.uart9_wait_for_rx) for [Anonymous Symbol]
    r_sci_uart.o(.text.R_SCI_UART_Open) refers to bsp_irq.o(.bss.gp_renesas_isr_context) for gp_renesas_isr_context
    r_sci_uart.o(.ARM.exidx.text.R_SCI_UART_Open) refers to r_sci_uart.o(.text.R_SCI_UART_Open) for [Anonymous Symbol]
    r_sci_uart.o(.ARM.exidx.text.R_SCI_UART_Read) refers to r_sci_uart.o(.text.R_SCI_UART_Read) for [Anonymous Symbol]
    r_sci_uart.o(.ARM.exidx.text.R_SCI_UART_Write) refers to r_sci_uart.o(.text.R_SCI_UART_Write) for [Anonymous Symbol]
    r_sci_uart.o(.ARM.exidx.text.R_SCI_UART_BaudSet) refers to r_sci_uart.o(.text.R_SCI_UART_BaudSet) for [Anonymous Symbol]
    r_sci_uart.o(.ARM.exidx.text.R_SCI_UART_InfoGet) refers to r_sci_uart.o(.text.R_SCI_UART_InfoGet) for [Anonymous Symbol]
    r_sci_uart.o(.ARM.exidx.text.R_SCI_UART_Abort) refers to r_sci_uart.o(.text.R_SCI_UART_Abort) for [Anonymous Symbol]
    r_sci_uart.o(.ARM.exidx.text.R_SCI_UART_CallbackSet) refers to r_sci_uart.o(.text.R_SCI_UART_CallbackSet) for [Anonymous Symbol]
    r_sci_uart.o(.ARM.exidx.text.R_SCI_UART_Close) refers to r_sci_uart.o(.text.R_SCI_UART_Close) for [Anonymous Symbol]
    r_sci_uart.o(.ARM.exidx.text.R_SCI_UART_ReadStop) refers to r_sci_uart.o(.text.R_SCI_UART_ReadStop) for [Anonymous Symbol]
    r_sci_uart.o(.text.R_SCI_UART_BaudCalculate) refers to system.o(.bss.SystemCoreClock) for SystemCoreClock
    r_sci_uart.o(.text.R_SCI_UART_BaudCalculate) refers to r_sci_uart.o(.rodata.g_async_baud) for g_async_baud
    r_sci_uart.o(.text.R_SCI_UART_BaudCalculate) refers to r_sci_uart.o(.rodata.g_div_coefficient) for g_div_coefficient
    r_sci_uart.o(.text.R_SCI_UART_BaudCalculate) refers to ldiv.o(.text) for __aeabi_ldivmod
    r_sci_uart.o(.ARM.exidx.text.R_SCI_UART_BaudCalculate) refers to r_sci_uart.o(.text.R_SCI_UART_BaudCalculate) for [Anonymous Symbol]
    r_sci_uart.o(.text.sci_uart_txi_isr) refers to bsp_irq.o(.bss.gp_renesas_isr_context) for gp_renesas_isr_context
    r_sci_uart.o(.text.sci_uart_txi_isr) refers to r_sci_uart.o(.text.r_sci_uart_call_callback) for r_sci_uart_call_callback
    r_sci_uart.o(.ARM.exidx.text.sci_uart_txi_isr) refers to r_sci_uart.o(.text.sci_uart_txi_isr) for [Anonymous Symbol]
    r_sci_uart.o(.ARM.exidx.text.r_sci_uart_call_callback) refers to r_sci_uart.o(.text.r_sci_uart_call_callback) for [Anonymous Symbol]
    r_sci_uart.o(.text.sci_uart_rxi_isr) refers to bsp_irq.o(.bss.gp_renesas_isr_context) for gp_renesas_isr_context
    r_sci_uart.o(.text.sci_uart_rxi_isr) refers to memcpya.o(.text) for __aeabi_memcpy
    r_sci_uart.o(.text.sci_uart_rxi_isr) refers to r_sci_uart.o(.text.r_sci_uart_call_callback) for r_sci_uart_call_callback
    r_sci_uart.o(.ARM.exidx.text.sci_uart_rxi_isr) refers to r_sci_uart.o(.text.sci_uart_rxi_isr) for [Anonymous Symbol]
    r_sci_uart.o(.text.sci_uart_tei_isr) refers to bsp_irq.o(.bss.gp_renesas_isr_context) for gp_renesas_isr_context
    r_sci_uart.o(.text.sci_uart_tei_isr) refers to r_sci_uart.o(.text.r_sci_uart_call_callback) for r_sci_uart_call_callback
    r_sci_uart.o(.ARM.exidx.text.sci_uart_tei_isr) refers to r_sci_uart.o(.text.sci_uart_tei_isr) for [Anonymous Symbol]
    r_sci_uart.o(.text.sci_uart_eri_isr) refers to bsp_irq.o(.bss.gp_renesas_isr_context) for gp_renesas_isr_context
    r_sci_uart.o(.text.sci_uart_eri_isr) refers to r_sci_uart.o(.text.r_sci_uart_call_callback) for r_sci_uart_call_callback
    r_sci_uart.o(.ARM.exidx.text.sci_uart_eri_isr) refers to r_sci_uart.o(.text.sci_uart_eri_isr) for [Anonymous Symbol]
    r_sci_uart.o(.rodata.g_uart_on_sci) refers to r_sci_uart.o(.text.R_SCI_UART_Open) for R_SCI_UART_Open
    r_sci_uart.o(.rodata.g_uart_on_sci) refers to r_sci_uart.o(.text.R_SCI_UART_Read) for R_SCI_UART_Read
    r_sci_uart.o(.rodata.g_uart_on_sci) refers to r_sci_uart.o(.text.R_SCI_UART_Write) for R_SCI_UART_Write
    r_sci_uart.o(.rodata.g_uart_on_sci) refers to r_sci_uart.o(.text.R_SCI_UART_BaudSet) for R_SCI_UART_BaudSet
    r_sci_uart.o(.rodata.g_uart_on_sci) refers to r_sci_uart.o(.text.R_SCI_UART_InfoGet) for R_SCI_UART_InfoGet
    r_sci_uart.o(.rodata.g_uart_on_sci) refers to r_sci_uart.o(.text.R_SCI_UART_Abort) for R_SCI_UART_Abort
    r_sci_uart.o(.rodata.g_uart_on_sci) refers to r_sci_uart.o(.text.R_SCI_UART_CallbackSet) for R_SCI_UART_CallbackSet
    r_sci_uart.o(.rodata.g_uart_on_sci) refers to r_sci_uart.o(.text.R_SCI_UART_Close) for R_SCI_UART_Close
    r_sci_uart.o(.rodata.g_uart_on_sci) refers to r_sci_uart.o(.text.R_SCI_UART_ReadStop) for R_SCI_UART_ReadStop
    common_data.o(.ARM.exidx.text.g_common_init) refers to common_data.o(.text.g_common_init) for [Anonymous Symbol]
    common_data.o(.rodata.g_ioport) refers to common_data.o(.bss.g_ioport_ctrl) for g_ioport_ctrl
    common_data.o(.rodata.g_ioport) refers to pin_data.o(.rodata.g_bsp_pin_cfg) for g_bsp_pin_cfg
    common_data.o(.rodata.g_ioport) refers to r_ioport.o(.rodata.g_ioport_on_ioport) for g_ioport_on_ioport
    hal_data.o(.text.g_hal_init) refers to common_data.o(.text.g_common_init) for g_common_init
    hal_data.o(.ARM.exidx.text.g_hal_init) refers to hal_data.o(.text.g_hal_init) for [Anonymous Symbol]
    hal_data.o(.rodata.g_timer5_cfg) refers to hal_entry.o(.text.user_timer5_callback) for user_timer5_callback
    hal_data.o(.rodata.g_timer5_cfg) refers to hal_data.o(.rodata.g_timer5_extend) for g_timer5_extend
    hal_data.o(.rodata.g_timer5) refers to hal_data.o(.bss.g_timer5_ctrl) for g_timer5_ctrl
    hal_data.o(.rodata.g_timer5) refers to hal_data.o(.rodata.g_timer5_cfg) for g_timer5_cfg
    hal_data.o(.rodata.g_timer5) refers to r_gpt.o(.rodata.g_timer_on_gpt) for g_timer_on_gpt
    hal_data.o(.rodata.g_timer2_cfg) refers to hal_data.o(.rodata.g_timer2_extend) for g_timer2_extend
    hal_data.o(.rodata.g_timer2) refers to hal_data.o(.bss.g_timer2_ctrl) for g_timer2_ctrl
    hal_data.o(.rodata.g_timer2) refers to hal_data.o(.rodata.g_timer2_cfg) for g_timer2_cfg
    hal_data.o(.rodata.g_timer2) refers to r_gpt.o(.rodata.g_timer_on_gpt) for g_timer_on_gpt
    hal_data.o(.rodata.g_timer0_cfg) refers to hal_entry.o(.text.user_timer0_callback) for user_timer0_callback
    hal_data.o(.rodata.g_timer0_cfg) refers to hal_data.o(.rodata.g_timer0_extend) for g_timer0_extend
    hal_data.o(.rodata.g_timer0) refers to hal_data.o(.bss.g_timer0_ctrl) for g_timer0_ctrl
    hal_data.o(.rodata.g_timer0) refers to hal_data.o(.rodata.g_timer0_cfg) for g_timer0_cfg
    hal_data.o(.rodata.g_timer0) refers to r_gpt.o(.rodata.g_timer_on_gpt) for g_timer_on_gpt
    hal_data.o(.rodata.g_dac0_cfg) refers to hal_data.o(.rodata.g_dac0_ext_cfg) for g_dac0_ext_cfg
    hal_data.o(.rodata.g_dac0) refers to hal_data.o(.bss.g_dac0_ctrl) for g_dac0_ctrl
    hal_data.o(.rodata.g_dac0) refers to hal_data.o(.rodata.g_dac0_cfg) for g_dac0_cfg
    hal_data.o(.rodata.g_dac0) refers to r_dac.o(.rodata.g_dac_on_dac) for g_dac_on_dac
    hal_data.o(.rodata.g_adc0_cfg) refers to r_adc.o(.text.user_adc_callback) for user_adc_callback
    hal_data.o(.rodata.g_adc0_cfg) refers to hal_data.o(.rodata.g_adc0_cfg_extend) for g_adc0_cfg_extend
    hal_data.o(.rodata.g_adc0) refers to hal_data.o(.bss.g_adc0_ctrl) for g_adc0_ctrl
    hal_data.o(.rodata.g_adc0) refers to hal_data.o(.rodata.g_adc0_cfg) for g_adc0_cfg
    hal_data.o(.rodata.g_adc0) refers to hal_data.o(.rodata.g_adc0_channel_cfg) for g_adc0_channel_cfg
    hal_data.o(.rodata.g_adc0) refers to r_adc.o(.rodata.g_adc_on_adc) for g_adc_on_adc
    hal_data.o(.rodata.g_uart9_cfg_extend) refers to hal_data.o(.data.g_uart9_baud_setting) for g_uart9_baud_setting
    hal_data.o(.rodata.g_uart9_cfg) refers to r_sci_uart.o(.text.user_uart9_callback) for user_uart9_callback
    hal_data.o(.rodata.g_uart9_cfg) refers to hal_data.o(.rodata.g_uart9_cfg_extend) for g_uart9_cfg_extend
    hal_data.o(.rodata.g_uart9) refers to hal_data.o(.bss.g_uart9_ctrl) for g_uart9_ctrl
    hal_data.o(.rodata.g_uart9) refers to hal_data.o(.rodata.g_uart9_cfg) for g_uart9_cfg
    hal_data.o(.rodata.g_uart9) refers to r_sci_uart.o(.rodata.g_uart_on_sci) for g_uart_on_sci
    main.o(.text.main) refers to hal_entry.o(.text.hal_entry) for hal_entry
    main.o(.ARM.exidx.text.main) refers to main.o(.text.main) for [Anonymous Symbol]
    pin_data.o(.rodata.g_bsp_pin_cfg) refers to pin_data.o(.rodata.g_bsp_pin_cfg_data) for g_bsp_pin_cfg_data
    vector_data.o(.application_vectors) refers to r_sci_uart.o(.text.sci_uart_rxi_isr) for sci_uart_rxi_isr
    vector_data.o(.application_vectors) refers to r_sci_uart.o(.text.sci_uart_txi_isr) for sci_uart_txi_isr
    vector_data.o(.application_vectors) refers to r_sci_uart.o(.text.sci_uart_tei_isr) for sci_uart_tei_isr
    vector_data.o(.application_vectors) refers to r_sci_uart.o(.text.sci_uart_eri_isr) for sci_uart_eri_isr
    vector_data.o(.application_vectors) refers to r_adc.o(.text.adc_scan_end_isr) for adc_scan_end_isr
    vector_data.o(.application_vectors) refers to r_gpt.o(.text.gpt_counter_overflow_isr) for gpt_counter_overflow_isr
    vector_data.o(.application_vectors) refers to r_gpt.o(.text.gpt_capture_compare_a_isr) for gpt_capture_compare_a_isr
    vector_data.o(.application_vectors) refers to r_gpt.o(.text.gpt_capture_compare_b_isr) for gpt_capture_compare_b_isr
    r_adc.o(.text.R_ADC_Open) refers to r_adc.o(.text.r_adc_irq_enable) for r_adc_irq_enable
    r_adc.o(.ARM.exidx.text.R_ADC_Open) refers to r_adc.o(.text.R_ADC_Open) for [Anonymous Symbol]
    r_adc.o(.text.R_ADC_ScanCfg) refers to system.o(.bss.SystemCoreClock) for SystemCoreClock
    r_adc.o(.ARM.exidx.text.R_ADC_ScanCfg) refers to r_adc.o(.text.R_ADC_ScanCfg) for [Anonymous Symbol]
    r_adc.o(.ARM.exidx.text.R_ADC_ScanStart) refers to r_adc.o(.text.R_ADC_ScanStart) for [Anonymous Symbol]
    r_adc.o(.ARM.exidx.text.R_ADC_ScanGroupStart) refers to r_adc.o(.text.R_ADC_ScanGroupStart) for [Anonymous Symbol]
    r_adc.o(.ARM.exidx.text.R_ADC_ScanStop) refers to r_adc.o(.text.R_ADC_ScanStop) for [Anonymous Symbol]
    r_adc.o(.ARM.exidx.text.R_ADC_StatusGet) refers to r_adc.o(.text.R_ADC_StatusGet) for [Anonymous Symbol]
    r_adc.o(.ARM.exidx.text.R_ADC_Read) refers to r_adc.o(.text.R_ADC_Read) for [Anonymous Symbol]
    r_adc.o(.ARM.exidx.text.R_ADC_Read32) refers to r_adc.o(.text.R_ADC_Read32) for [Anonymous Symbol]
    r_adc.o(.ARM.exidx.text.R_ADC_Calibrate) refers to r_adc.o(.text.R_ADC_Calibrate) for [Anonymous Symbol]
    r_adc.o(.ARM.exidx.text.R_ADC_OffsetSet) refers to r_adc.o(.text.R_ADC_OffsetSet) for [Anonymous Symbol]
    r_adc.o(.ARM.exidx.text.R_ADC_CallbackSet) refers to r_adc.o(.text.R_ADC_CallbackSet) for [Anonymous Symbol]
    r_adc.o(.text.R_ADC_Close) refers to bsp_irq.o(.bss.gp_renesas_isr_context) for gp_renesas_isr_context
    r_adc.o(.ARM.exidx.text.R_ADC_Close) refers to r_adc.o(.text.R_ADC_Close) for [Anonymous Symbol]
    r_adc.o(.ARM.exidx.text.R_ADC_InfoGet) refers to r_adc.o(.text.R_ADC_InfoGet) for [Anonymous Symbol]
    r_adc.o(.text.r_adc_irq_enable) refers to bsp_irq.o(.bss.gp_renesas_isr_context) for gp_renesas_isr_context
    r_adc.o(.ARM.exidx.text.r_adc_irq_enable) refers to r_adc.o(.text.r_adc_irq_enable) for [Anonymous Symbol]
    r_adc.o(.ARM.exidx.text.R_ADC_SampleStateCountSet) refers to r_adc.o(.text.R_ADC_SampleStateCountSet) for [Anonymous Symbol]
    r_adc.o(.text.adc_scan_end_isr) refers to r_adc.o(.text.r_adc_scan_end_common_isr) for r_adc_scan_end_common_isr
    r_adc.o(.ARM.exidx.text.adc_scan_end_isr) refers to r_adc.o(.text.adc_scan_end_isr) for [Anonymous Symbol]
    r_adc.o(.text.r_adc_scan_end_common_isr) refers to bsp_irq.o(.bss.gp_renesas_isr_context) for gp_renesas_isr_context
    r_adc.o(.ARM.exidx.text.r_adc_scan_end_common_isr) refers to r_adc.o(.text.r_adc_scan_end_common_isr) for [Anonymous Symbol]
    r_adc.o(.text.adc_scan_end_b_isr) refers to r_adc.o(.text.r_adc_scan_end_common_isr) for r_adc_scan_end_common_isr
    r_adc.o(.ARM.exidx.text.adc_scan_end_b_isr) refers to r_adc.o(.text.adc_scan_end_b_isr) for [Anonymous Symbol]
    r_adc.o(.text.adc_window_compare_isr) refers to bsp_irq.o(.bss.gp_renesas_isr_context) for gp_renesas_isr_context
    r_adc.o(.ARM.exidx.text.adc_window_compare_isr) refers to r_adc.o(.text.adc_window_compare_isr) for [Anonymous Symbol]
    r_adc.o(.text.user_adc_callback) refers to r_adc.o(.bss.scan_complete_flag) for scan_complete_flag
    r_adc.o(.ARM.exidx.text.user_adc_callback) refers to r_adc.o(.text.user_adc_callback) for [Anonymous Symbol]
    r_adc.o(.text.adc_wait_for_scan) refers to r_adc.o(.bss.scan_complete_flag) for scan_complete_flag
    r_adc.o(.ARM.exidx.text.adc_wait_for_scan) refers to r_adc.o(.text.adc_wait_for_scan) for [Anonymous Symbol]
    r_adc.o(.text.get_adc_scan_status) refers to r_adc.o(.bss.scan_complete_flag) for scan_complete_flag
    r_adc.o(.ARM.exidx.text.get_adc_scan_status) refers to r_adc.o(.text.get_adc_scan_status) for [Anonymous Symbol]
    r_adc.o(.text.reset_adc_scan_state) refers to r_adc.o(.bss.scan_complete_flag) for scan_complete_flag
    r_adc.o(.ARM.exidx.text.reset_adc_scan_state) refers to r_adc.o(.text.reset_adc_scan_state) for [Anonymous Symbol]
    r_adc.o(.rodata.g_adc_on_adc) refers to r_adc.o(.text.R_ADC_Open) for R_ADC_Open
    r_adc.o(.rodata.g_adc_on_adc) refers to r_adc.o(.text.R_ADC_ScanCfg) for R_ADC_ScanCfg
    r_adc.o(.rodata.g_adc_on_adc) refers to r_adc.o(.text.R_ADC_ScanStart) for R_ADC_ScanStart
    r_adc.o(.rodata.g_adc_on_adc) refers to r_adc.o(.text.R_ADC_ScanGroupStart) for R_ADC_ScanGroupStart
    r_adc.o(.rodata.g_adc_on_adc) refers to r_adc.o(.text.R_ADC_ScanStop) for R_ADC_ScanStop
    r_adc.o(.rodata.g_adc_on_adc) refers to r_adc.o(.text.R_ADC_StatusGet) for R_ADC_StatusGet
    r_adc.o(.rodata.g_adc_on_adc) refers to r_adc.o(.text.R_ADC_Read) for R_ADC_Read
    r_adc.o(.rodata.g_adc_on_adc) refers to r_adc.o(.text.R_ADC_Read32) for R_ADC_Read32
    r_adc.o(.rodata.g_adc_on_adc) refers to r_adc.o(.text.R_ADC_Calibrate) for R_ADC_Calibrate
    r_adc.o(.rodata.g_adc_on_adc) refers to r_adc.o(.text.R_ADC_OffsetSet) for R_ADC_OffsetSet
    r_adc.o(.rodata.g_adc_on_adc) refers to r_adc.o(.text.R_ADC_CallbackSet) for R_ADC_CallbackSet
    r_adc.o(.rodata.g_adc_on_adc) refers to r_adc.o(.text.R_ADC_Close) for R_ADC_Close
    r_adc.o(.rodata.g_adc_on_adc) refers to r_adc.o(.text.R_ADC_InfoGet) for R_ADC_InfoGet
    r_dac.o(.ARM.exidx.text.R_DAC_Open) refers to r_dac.o(.text.R_DAC_Open) for [Anonymous Symbol]
    r_dac.o(.ARM.exidx.text.R_DAC_Close) refers to r_dac.o(.text.R_DAC_Close) for [Anonymous Symbol]
    r_dac.o(.ARM.exidx.text.R_DAC_Write) refers to r_dac.o(.text.R_DAC_Write) for [Anonymous Symbol]
    r_dac.o(.text.R_DAC_Start) refers to bsp_delay.o(.text.R_BSP_SoftwareDelay) for R_BSP_SoftwareDelay
    r_dac.o(.ARM.exidx.text.R_DAC_Start) refers to r_dac.o(.text.R_DAC_Start) for [Anonymous Symbol]
    r_dac.o(.ARM.exidx.text.R_DAC_Stop) refers to r_dac.o(.text.R_DAC_Stop) for [Anonymous Symbol]
    r_dac.o(.rodata.g_dac_on_dac) refers to r_dac.o(.text.R_DAC_Open) for R_DAC_Open
    r_dac.o(.rodata.g_dac_on_dac) refers to r_dac.o(.text.R_DAC_Close) for R_DAC_Close
    r_dac.o(.rodata.g_dac_on_dac) refers to r_dac.o(.text.R_DAC_Write) for R_DAC_Write
    r_dac.o(.rodata.g_dac_on_dac) refers to r_dac.o(.text.R_DAC_Start) for R_DAC_Start
    r_dac.o(.rodata.g_dac_on_dac) refers to r_dac.o(.text.R_DAC_Stop) for R_DAC_Stop
    r_gpt.o(.text.R_GPT_Open) refers to r_gpt.o(.text.gpt_calculate_duty_cycle) for gpt_calculate_duty_cycle
    r_gpt.o(.text.R_GPT_Open) refers to r_gpt.o(.text.r_gpt_enable_irq) for r_gpt_enable_irq
    r_gpt.o(.ARM.exidx.text.R_GPT_Open) refers to r_gpt.o(.text.R_GPT_Open) for [Anonymous Symbol]
    r_gpt.o(.ARM.exidx.text.R_GPT_Start) refers to r_gpt.o(.text.R_GPT_Start) for [Anonymous Symbol]
    r_gpt.o(.ARM.exidx.text.R_GPT_Stop) refers to r_gpt.o(.text.R_GPT_Stop) for [Anonymous Symbol]
    r_gpt.o(.ARM.exidx.text.R_GPT_Reset) refers to r_gpt.o(.text.R_GPT_Reset) for [Anonymous Symbol]
    r_gpt.o(.ARM.exidx.text.R_GPT_Enable) refers to r_gpt.o(.text.R_GPT_Enable) for [Anonymous Symbol]
    r_gpt.o(.ARM.exidx.text.R_GPT_Disable) refers to r_gpt.o(.text.R_GPT_Disable) for [Anonymous Symbol]
    r_gpt.o(.ARM.exidx.text.R_GPT_PeriodSet) refers to r_gpt.o(.text.R_GPT_PeriodSet) for [Anonymous Symbol]
    r_gpt.o(.text.R_GPT_DutyCycleSet) refers to r_gpt.o(.text.gpt_calculate_duty_cycle) for gpt_calculate_duty_cycle
    r_gpt.o(.ARM.exidx.text.R_GPT_DutyCycleSet) refers to r_gpt.o(.text.R_GPT_DutyCycleSet) for [Anonymous Symbol]
    r_gpt.o(.ARM.exidx.text.R_GPT_CompareMatchSet) refers to r_gpt.o(.text.R_GPT_CompareMatchSet) for [Anonymous Symbol]
    r_gpt.o(.text.R_GPT_InfoGet) refers to system.o(.bss.SystemCoreClock) for SystemCoreClock
    r_gpt.o(.ARM.exidx.text.R_GPT_InfoGet) refers to r_gpt.o(.text.R_GPT_InfoGet) for [Anonymous Symbol]
    r_gpt.o(.ARM.exidx.text.R_GPT_StatusGet) refers to r_gpt.o(.text.R_GPT_StatusGet) for [Anonymous Symbol]
    r_gpt.o(.ARM.exidx.text.R_GPT_CallbackSet) refers to r_gpt.o(.text.R_GPT_CallbackSet) for [Anonymous Symbol]
    r_gpt.o(.text.R_GPT_Close) refers to bsp_irq.o(.bss.gp_renesas_isr_context) for gp_renesas_isr_context
    r_gpt.o(.ARM.exidx.text.R_GPT_Close) refers to r_gpt.o(.text.R_GPT_Close) for [Anonymous Symbol]
    r_gpt.o(.ARM.exidx.text.gpt_calculate_duty_cycle) refers to r_gpt.o(.text.gpt_calculate_duty_cycle) for [Anonymous Symbol]
    r_gpt.o(.ARM.exidx.text.R_GPT_CounterSet) refers to r_gpt.o(.text.R_GPT_CounterSet) for [Anonymous Symbol]
    r_gpt.o(.ARM.exidx.text.R_GPT_OutputEnable) refers to r_gpt.o(.text.R_GPT_OutputEnable) for [Anonymous Symbol]
    r_gpt.o(.ARM.exidx.text.R_GPT_OutputDisable) refers to r_gpt.o(.text.R_GPT_OutputDisable) for [Anonymous Symbol]
    r_gpt.o(.ARM.exidx.text.R_GPT_AdcTriggerSet) refers to r_gpt.o(.text.R_GPT_AdcTriggerSet) for [Anonymous Symbol]
    r_gpt.o(.ARM.exidx.text.R_GPT_PwmOutputDelaySet) refers to r_gpt.o(.text.R_GPT_PwmOutputDelaySet) for [Anonymous Symbol]
    r_gpt.o(.ARM.exidx.text.R_GPT_PwmOutputDelayInitialize) refers to r_gpt.o(.text.R_GPT_PwmOutputDelayInitialize) for [Anonymous Symbol]
    r_gpt.o(.text.gpt_counter_overflow_isr) refers to bsp_irq.o(.bss.gp_renesas_isr_context) for gp_renesas_isr_context
    r_gpt.o(.ARM.exidx.text.gpt_counter_overflow_isr) refers to r_gpt.o(.text.gpt_counter_overflow_isr) for [Anonymous Symbol]
    r_gpt.o(.text.gpt_capture_compare_a_isr) refers to r_gpt.o(.text.r_gpt_ccmp_common_isr) for r_gpt_ccmp_common_isr
    r_gpt.o(.ARM.exidx.text.gpt_capture_compare_a_isr) refers to r_gpt.o(.text.gpt_capture_compare_a_isr) for [Anonymous Symbol]
    r_gpt.o(.text.r_gpt_ccmp_common_isr) refers to bsp_irq.o(.bss.gp_renesas_isr_context) for gp_renesas_isr_context
    r_gpt.o(.ARM.exidx.text.r_gpt_ccmp_common_isr) refers to r_gpt.o(.text.r_gpt_ccmp_common_isr) for [Anonymous Symbol]
    r_gpt.o(.text.gpt_capture_compare_b_isr) refers to r_gpt.o(.text.r_gpt_ccmp_common_isr) for r_gpt_ccmp_common_isr
    r_gpt.o(.ARM.exidx.text.gpt_capture_compare_b_isr) refers to r_gpt.o(.text.gpt_capture_compare_b_isr) for [Anonymous Symbol]
    r_gpt.o(.text.r_gpt_enable_irq) refers to bsp_irq.o(.bss.gp_renesas_isr_context) for gp_renesas_isr_context
    r_gpt.o(.ARM.exidx.text.r_gpt_enable_irq) refers to r_gpt.o(.text.r_gpt_enable_irq) for [Anonymous Symbol]
    r_gpt.o(.rodata.g_timer_on_gpt) refers to r_gpt.o(.text.R_GPT_Open) for R_GPT_Open
    r_gpt.o(.rodata.g_timer_on_gpt) refers to r_gpt.o(.text.R_GPT_Start) for R_GPT_Start
    r_gpt.o(.rodata.g_timer_on_gpt) refers to r_gpt.o(.text.R_GPT_Stop) for R_GPT_Stop
    r_gpt.o(.rodata.g_timer_on_gpt) refers to r_gpt.o(.text.R_GPT_Reset) for R_GPT_Reset
    r_gpt.o(.rodata.g_timer_on_gpt) refers to r_gpt.o(.text.R_GPT_Enable) for R_GPT_Enable
    r_gpt.o(.rodata.g_timer_on_gpt) refers to r_gpt.o(.text.R_GPT_Disable) for R_GPT_Disable
    r_gpt.o(.rodata.g_timer_on_gpt) refers to r_gpt.o(.text.R_GPT_PeriodSet) for R_GPT_PeriodSet
    r_gpt.o(.rodata.g_timer_on_gpt) refers to r_gpt.o(.text.R_GPT_DutyCycleSet) for R_GPT_DutyCycleSet
    r_gpt.o(.rodata.g_timer_on_gpt) refers to r_gpt.o(.text.R_GPT_CompareMatchSet) for R_GPT_CompareMatchSet
    r_gpt.o(.rodata.g_timer_on_gpt) refers to r_gpt.o(.text.R_GPT_InfoGet) for R_GPT_InfoGet
    r_gpt.o(.rodata.g_timer_on_gpt) refers to r_gpt.o(.text.R_GPT_StatusGet) for R_GPT_StatusGet
    r_gpt.o(.rodata.g_timer_on_gpt) refers to r_gpt.o(.text.R_GPT_CallbackSet) for R_GPT_CallbackSet
    r_gpt.o(.rodata.g_timer_on_gpt) refers to r_gpt.o(.text.R_GPT_Close) for R_GPT_Close
    puts.o(i.puts) refers to fputc.o(i.fputc) for fputc
    puts.o(i.puts) refers to stdout.o(.data) for __stdout
    puts_e.o(.text) refers to fputc.o(i.fputc) for fputc
    puts_e.o(.text) refers to stdout.o(.data) for __stdout
    uldiv.o(.text) refers to llushr.o(.text) for __aeabi_llsr
    uldiv.o(.text) refers to llshl.o(.text) for __aeabi_llsl
    ldiv.o(.text) refers to uldiv.o(.text) for __aeabi_uldivmod
    printfb.o(i.__0fprintf$bare) refers to printfb.o(i._printf_core) for _printf_core
    printfb.o(i.__0fprintf$bare) refers to fputc.o(i.fputc) for fputc
    printfb.o(i.__0printf$bare) refers to printfb.o(i._printf_core) for _printf_core
    printfb.o(i.__0printf$bare) refers to fputc.o(i.fputc) for fputc
    printfb.o(i.__0printf$bare) refers to stdout.o(.data) for __stdout
    printfb.o(i.__0snprintf$bare) refers to printfb.o(i._printf_core) for _printf_core
    printfb.o(i.__0snprintf$bare) refers to printfb.o(i._snputc) for _snputc
    printfb.o(i.__0sprintf$bare) refers to printfb.o(i._printf_core) for _printf_core
    printfb.o(i.__0sprintf$bare) refers to printfb.o(i._sputc) for _sputc
    printfb.o(i.__0vfprintf$bare) refers to printfb.o(i._printf_core) for _printf_core
    printfb.o(i.__0vfprintf$bare) refers to fputc.o(i.fputc) for fputc
    printfb.o(i.__0vprintf$bare) refers to printfb.o(i._printf_core) for _printf_core
    printfb.o(i.__0vprintf$bare) refers to fputc.o(i.fputc) for fputc
    printfb.o(i.__0vprintf$bare) refers to stdout.o(.data) for __stdout
    printfb.o(i.__0vsnprintf$bare) refers to printfb.o(i._printf_core) for _printf_core
    printfb.o(i.__0vsnprintf$bare) refers to printfb.o(i._snputc) for _snputc
    printfb.o(i.__0vsprintf$bare) refers to printfb.o(i._printf_core) for _printf_core
    printfb.o(i.__0vsprintf$bare) refers to printfb.o(i._sputc) for _sputc
    printf0.o(i.__0fprintf$0) refers to printf0.o(i._printf_core) for _printf_core
    printf0.o(i.__0fprintf$0) refers to fputc.o(i.fputc) for fputc
    printf0.o(i.__0printf$0) refers to printf0.o(i._printf_core) for _printf_core
    printf0.o(i.__0printf$0) refers to fputc.o(i.fputc) for fputc
    printf0.o(i.__0printf$0) refers to stdout.o(.data) for __stdout
    printf0.o(i.__0snprintf$0) refers to printf0.o(i._printf_core) for _printf_core
    printf0.o(i.__0snprintf$0) refers to printf0.o(i._snputc) for _snputc
    printf0.o(i.__0sprintf$0) refers to printf0.o(i._printf_core) for _printf_core
    printf0.o(i.__0sprintf$0) refers to printf0.o(i._sputc) for _sputc
    printf0.o(i.__0vfprintf$0) refers to printf0.o(i._printf_core) for _printf_core
    printf0.o(i.__0vfprintf$0) refers to fputc.o(i.fputc) for fputc
    printf0.o(i.__0vprintf$0) refers to printf0.o(i._printf_core) for _printf_core
    printf0.o(i.__0vprintf$0) refers to fputc.o(i.fputc) for fputc
    printf0.o(i.__0vprintf$0) refers to stdout.o(.data) for __stdout
    printf0.o(i.__0vsnprintf$0) refers to printf0.o(i._printf_core) for _printf_core
    printf0.o(i.__0vsnprintf$0) refers to printf0.o(i._snputc) for _snputc
    printf0.o(i.__0vsprintf$0) refers to printf0.o(i._printf_core) for _printf_core
    printf0.o(i.__0vsprintf$0) refers to printf0.o(i._sputc) for _sputc
    printf1.o(i.__0fprintf$1) refers to printf1.o(i._printf_core) for _printf_core
    printf1.o(i.__0fprintf$1) refers to fputc.o(i.fputc) for fputc
    printf1.o(i.__0printf$1) refers to printf1.o(i._printf_core) for _printf_core
    printf1.o(i.__0printf$1) refers to fputc.o(i.fputc) for fputc
    printf1.o(i.__0printf$1) refers to stdout.o(.data) for __stdout
    printf1.o(i.__0snprintf$1) refers to printf1.o(i._printf_core) for _printf_core
    printf1.o(i.__0snprintf$1) refers to printf1.o(i._snputc) for _snputc
    printf1.o(i.__0sprintf$1) refers to printf1.o(i._printf_core) for _printf_core
    printf1.o(i.__0sprintf$1) refers to printf1.o(i._sputc) for _sputc
    printf1.o(i.__0vfprintf$1) refers to printf1.o(i._printf_core) for _printf_core
    printf1.o(i.__0vfprintf$1) refers to fputc.o(i.fputc) for fputc
    printf1.o(i.__0vprintf$1) refers to printf1.o(i._printf_core) for _printf_core
    printf1.o(i.__0vprintf$1) refers to fputc.o(i.fputc) for fputc
    printf1.o(i.__0vprintf$1) refers to stdout.o(.data) for __stdout
    printf1.o(i.__0vsnprintf$1) refers to printf1.o(i._printf_core) for _printf_core
    printf1.o(i.__0vsnprintf$1) refers to printf1.o(i._snputc) for _snputc
    printf1.o(i.__0vsprintf$1) refers to printf1.o(i._printf_core) for _printf_core
    printf1.o(i.__0vsprintf$1) refers to printf1.o(i._sputc) for _sputc
    printf1.o(i._printf_core) refers to uidiv.o(.text) for __aeabi_uidivmod
    printf2.o(i.__0fprintf$2) refers to printf2.o(i._printf_core) for _printf_core
    printf2.o(i.__0fprintf$2) refers to fputc.o(i.fputc) for fputc
    printf2.o(i.__0printf$2) refers to printf2.o(i._printf_core) for _printf_core
    printf2.o(i.__0printf$2) refers to fputc.o(i.fputc) for fputc
    printf2.o(i.__0printf$2) refers to stdout.o(.data) for __stdout
    printf2.o(i.__0snprintf$2) refers to printf2.o(i._printf_core) for _printf_core
    printf2.o(i.__0snprintf$2) refers to printf2.o(i._snputc) for _snputc
    printf2.o(i.__0sprintf$2) refers to printf2.o(i._printf_core) for _printf_core
    printf2.o(i.__0sprintf$2) refers to printf2.o(i._sputc) for _sputc
    printf2.o(i.__0vfprintf$2) refers to printf2.o(i._printf_core) for _printf_core
    printf2.o(i.__0vfprintf$2) refers to fputc.o(i.fputc) for fputc
    printf2.o(i.__0vprintf$2) refers to printf2.o(i._printf_core) for _printf_core
    printf2.o(i.__0vprintf$2) refers to fputc.o(i.fputc) for fputc
    printf2.o(i.__0vprintf$2) refers to stdout.o(.data) for __stdout
    printf2.o(i.__0vsnprintf$2) refers to printf2.o(i._printf_core) for _printf_core
    printf2.o(i.__0vsnprintf$2) refers to printf2.o(i._snputc) for _snputc
    printf2.o(i.__0vsprintf$2) refers to printf2.o(i._printf_core) for _printf_core
    printf2.o(i.__0vsprintf$2) refers to printf2.o(i._sputc) for _sputc
    printf3.o(i.__0fprintf$3) refers to printf3.o(i._printf_core) for _printf_core
    printf3.o(i.__0fprintf$3) refers to fputc.o(i.fputc) for fputc
    printf3.o(i.__0printf$3) refers to printf3.o(i._printf_core) for _printf_core
    printf3.o(i.__0printf$3) refers to fputc.o(i.fputc) for fputc
    printf3.o(i.__0printf$3) refers to stdout.o(.data) for __stdout
    printf3.o(i.__0snprintf$3) refers to printf3.o(i._printf_core) for _printf_core
    printf3.o(i.__0snprintf$3) refers to printf3.o(i._snputc) for _snputc
    printf3.o(i.__0sprintf$3) refers to printf3.o(i._printf_core) for _printf_core
    printf3.o(i.__0sprintf$3) refers to printf3.o(i._sputc) for _sputc
    printf3.o(i.__0vfprintf$3) refers to printf3.o(i._printf_core) for _printf_core
    printf3.o(i.__0vfprintf$3) refers to fputc.o(i.fputc) for fputc
    printf3.o(i.__0vprintf$3) refers to printf3.o(i._printf_core) for _printf_core
    printf3.o(i.__0vprintf$3) refers to fputc.o(i.fputc) for fputc
    printf3.o(i.__0vprintf$3) refers to stdout.o(.data) for __stdout
    printf3.o(i.__0vsnprintf$3) refers to printf3.o(i._printf_core) for _printf_core
    printf3.o(i.__0vsnprintf$3) refers to printf3.o(i._snputc) for _snputc
    printf3.o(i.__0vsprintf$3) refers to printf3.o(i._printf_core) for _printf_core
    printf3.o(i.__0vsprintf$3) refers to printf3.o(i._sputc) for _sputc
    printf3.o(i._printf_core) refers to uidiv.o(.text) for __aeabi_uidivmod
    printf4.o(i.__0fprintf$4) refers to printf4.o(i._printf_core) for _printf_core
    printf4.o(i.__0fprintf$4) refers to fputc.o(i.fputc) for fputc
    printf4.o(i.__0printf$4) refers to printf4.o(i._printf_core) for _printf_core
    printf4.o(i.__0printf$4) refers to fputc.o(i.fputc) for fputc
    printf4.o(i.__0printf$4) refers to stdout.o(.data) for __stdout
    printf4.o(i.__0snprintf$4) refers to printf4.o(i._printf_core) for _printf_core
    printf4.o(i.__0snprintf$4) refers to printf4.o(i._snputc) for _snputc
    printf4.o(i.__0sprintf$4) refers to printf4.o(i._printf_core) for _printf_core
    printf4.o(i.__0sprintf$4) refers to printf4.o(i._sputc) for _sputc
    printf4.o(i.__0vfprintf$4) refers to printf4.o(i._printf_core) for _printf_core
    printf4.o(i.__0vfprintf$4) refers to fputc.o(i.fputc) for fputc
    printf4.o(i.__0vprintf$4) refers to printf4.o(i._printf_core) for _printf_core
    printf4.o(i.__0vprintf$4) refers to fputc.o(i.fputc) for fputc
    printf4.o(i.__0vprintf$4) refers to stdout.o(.data) for __stdout
    printf4.o(i.__0vsnprintf$4) refers to printf4.o(i._printf_core) for _printf_core
    printf4.o(i.__0vsnprintf$4) refers to printf4.o(i._snputc) for _snputc
    printf4.o(i.__0vsprintf$4) refers to printf4.o(i._printf_core) for _printf_core
    printf4.o(i.__0vsprintf$4) refers to printf4.o(i._sputc) for _sputc
    printf4.o(i._printf_core) refers to uldiv.o(.text) for __aeabi_uldivmod
    printf5.o(i.__0fprintf$5) refers to printf5.o(i._printf_core) for _printf_core
    printf5.o(i.__0fprintf$5) refers to fputc.o(i.fputc) for fputc
    printf5.o(i.__0printf$5) refers to printf5.o(i._printf_core) for _printf_core
    printf5.o(i.__0printf$5) refers to fputc.o(i.fputc) for fputc
    printf5.o(i.__0printf$5) refers to stdout.o(.data) for __stdout
    printf5.o(i.__0snprintf$5) refers to printf5.o(i._printf_core) for _printf_core
    printf5.o(i.__0snprintf$5) refers to printf5.o(i._snputc) for _snputc
    printf5.o(i.__0sprintf$5) refers to printf5.o(i._printf_core) for _printf_core
    printf5.o(i.__0sprintf$5) refers to printf5.o(i._sputc) for _sputc
    printf5.o(i.__0vfprintf$5) refers to printf5.o(i._printf_core) for _printf_core
    printf5.o(i.__0vfprintf$5) refers to fputc.o(i.fputc) for fputc
    printf5.o(i.__0vprintf$5) refers to printf5.o(i._printf_core) for _printf_core
    printf5.o(i.__0vprintf$5) refers to fputc.o(i.fputc) for fputc
    printf5.o(i.__0vprintf$5) refers to stdout.o(.data) for __stdout
    printf5.o(i.__0vsnprintf$5) refers to printf5.o(i._printf_core) for _printf_core
    printf5.o(i.__0vsnprintf$5) refers to printf5.o(i._snputc) for _snputc
    printf5.o(i.__0vsprintf$5) refers to printf5.o(i._printf_core) for _printf_core
    printf5.o(i.__0vsprintf$5) refers to printf5.o(i._sputc) for _sputc
    printf5.o(i._printf_core) refers to uldiv.o(.text) for __aeabi_uldivmod
    printf6.o(i.__0fprintf$6) refers to printf6.o(i._printf_core) for _printf_core
    printf6.o(i.__0fprintf$6) refers to fputc.o(i.fputc) for fputc
    printf6.o(i.__0printf$6) refers to printf6.o(i._printf_core) for _printf_core
    printf6.o(i.__0printf$6) refers to fputc.o(i.fputc) for fputc
    printf6.o(i.__0printf$6) refers to stdout.o(.data) for __stdout
    printf6.o(i.__0snprintf$6) refers to printf6.o(i._printf_core) for _printf_core
    printf6.o(i.__0snprintf$6) refers to printf6.o(i._snputc) for _snputc
    printf6.o(i.__0sprintf$6) refers to printf6.o(i._printf_core) for _printf_core
    printf6.o(i.__0sprintf$6) refers to printf6.o(i._sputc) for _sputc
    printf6.o(i.__0vfprintf$6) refers to printf6.o(i._printf_core) for _printf_core
    printf6.o(i.__0vfprintf$6) refers to fputc.o(i.fputc) for fputc
    printf6.o(i.__0vprintf$6) refers to printf6.o(i._printf_core) for _printf_core
    printf6.o(i.__0vprintf$6) refers to fputc.o(i.fputc) for fputc
    printf6.o(i.__0vprintf$6) refers to stdout.o(.data) for __stdout
    printf6.o(i.__0vsnprintf$6) refers to printf6.o(i._printf_core) for _printf_core
    printf6.o(i.__0vsnprintf$6) refers to printf6.o(i._snputc) for _snputc
    printf6.o(i.__0vsprintf$6) refers to printf6.o(i._printf_core) for _printf_core
    printf6.o(i.__0vsprintf$6) refers to printf6.o(i._sputc) for _sputc
    printf6.o(i._printf_core) refers to printf6.o(i._printf_pre_padding) for _printf_pre_padding
    printf6.o(i._printf_core) refers to uidiv.o(.text) for __aeabi_uidivmod
    printf6.o(i._printf_core) refers to printf6.o(i._printf_post_padding) for _printf_post_padding
    printf7.o(i.__0fprintf$7) refers to printf7.o(i._printf_core) for _printf_core
    printf7.o(i.__0fprintf$7) refers to fputc.o(i.fputc) for fputc
    printf7.o(i.__0printf$7) refers to printf7.o(i._printf_core) for _printf_core
    printf7.o(i.__0printf$7) refers to fputc.o(i.fputc) for fputc
    printf7.o(i.__0printf$7) refers to stdout.o(.data) for __stdout
    printf7.o(i.__0snprintf$7) refers to printf7.o(i._printf_core) for _printf_core
    printf7.o(i.__0snprintf$7) refers to printf7.o(i._snputc) for _snputc
    printf7.o(i.__0sprintf$7) refers to printf7.o(i._printf_core) for _printf_core
    printf7.o(i.__0sprintf$7) refers to printf7.o(i._sputc) for _sputc
    printf7.o(i.__0vfprintf$7) refers to printf7.o(i._printf_core) for _printf_core
    printf7.o(i.__0vfprintf$7) refers to fputc.o(i.fputc) for fputc
    printf7.o(i.__0vprintf$7) refers to printf7.o(i._printf_core) for _printf_core
    printf7.o(i.__0vprintf$7) refers to fputc.o(i.fputc) for fputc
    printf7.o(i.__0vprintf$7) refers to stdout.o(.data) for __stdout
    printf7.o(i.__0vsnprintf$7) refers to printf7.o(i._printf_core) for _printf_core
    printf7.o(i.__0vsnprintf$7) refers to printf7.o(i._snputc) for _snputc
    printf7.o(i.__0vsprintf$7) refers to printf7.o(i._printf_core) for _printf_core
    printf7.o(i.__0vsprintf$7) refers to printf7.o(i._sputc) for _sputc
    printf7.o(i._printf_core) refers to printf7.o(i._printf_pre_padding) for _printf_pre_padding
    printf7.o(i._printf_core) refers to uldiv.o(.text) for __aeabi_uldivmod
    printf7.o(i._printf_core) refers to printf7.o(i._printf_post_padding) for _printf_post_padding
    printf8.o(i.__0fprintf$8) refers to printf8.o(i._printf_core) for _printf_core
    printf8.o(i.__0fprintf$8) refers to fputc.o(i.fputc) for fputc
    printf8.o(i.__0printf$8) refers to printf8.o(i._printf_core) for _printf_core
    printf8.o(i.__0printf$8) refers to fputc.o(i.fputc) for fputc
    printf8.o(i.__0printf$8) refers to stdout.o(.data) for __stdout
    printf8.o(i.__0snprintf$8) refers to printf8.o(i._printf_core) for _printf_core
    printf8.o(i.__0snprintf$8) refers to printf8.o(i._snputc) for _snputc
    printf8.o(i.__0sprintf$8) refers to printf8.o(i._printf_core) for _printf_core
    printf8.o(i.__0sprintf$8) refers to printf8.o(i._sputc) for _sputc
    printf8.o(i.__0vfprintf$8) refers to printf8.o(i._printf_core) for _printf_core
    printf8.o(i.__0vfprintf$8) refers to fputc.o(i.fputc) for fputc
    printf8.o(i.__0vprintf$8) refers to printf8.o(i._printf_core) for _printf_core
    printf8.o(i.__0vprintf$8) refers to fputc.o(i.fputc) for fputc
    printf8.o(i.__0vprintf$8) refers to stdout.o(.data) for __stdout
    printf8.o(i.__0vsnprintf$8) refers to printf8.o(i._printf_core) for _printf_core
    printf8.o(i.__0vsnprintf$8) refers to printf8.o(i._snputc) for _snputc
    printf8.o(i.__0vsprintf$8) refers to printf8.o(i._printf_core) for _printf_core
    printf8.o(i.__0vsprintf$8) refers to printf8.o(i._sputc) for _sputc
    printf8.o(i._printf_core) refers to printf8.o(i._printf_pre_padding) for _printf_pre_padding
    printf8.o(i._printf_core) refers to uldiv.o(.text) for __aeabi_uldivmod
    printf8.o(i._printf_core) refers to printf8.o(i._printf_post_padding) for _printf_post_padding
    printfa.o(i.__0fprintf) refers (Special) to iusefp.o(.text) for __I$use$fp
    printfa.o(i.__0fprintf) refers to printfa.o(i._printf_core) for _printf_core
    printfa.o(i.__0fprintf) refers to fputc.o(i.fputc) for fputc
    printfa.o(i.__0printf) refers (Special) to iusefp.o(.text) for __I$use$fp
    printfa.o(i.__0printf) refers to printfa.o(i._printf_core) for _printf_core
    printfa.o(i.__0printf) refers to fputc.o(i.fputc) for fputc
    printfa.o(i.__0printf) refers to stdout.o(.data) for __stdout
    printfa.o(i.__0snprintf) refers (Special) to iusefp.o(.text) for __I$use$fp
    printfa.o(i.__0snprintf) refers to printfa.o(i._printf_core) for _printf_core
    printfa.o(i.__0snprintf) refers to printfa.o(i._snputc) for _snputc
    printfa.o(i.__0sprintf) refers (Special) to iusefp.o(.text) for __I$use$fp
    printfa.o(i.__0sprintf) refers to printfa.o(i._printf_core) for _printf_core
    printfa.o(i.__0sprintf) refers to printfa.o(i._sputc) for _sputc
    printfa.o(i.__0vfprintf) refers (Special) to iusefp.o(.text) for __I$use$fp
    printfa.o(i.__0vfprintf) refers to printfa.o(i._printf_core) for _printf_core
    printfa.o(i.__0vfprintf) refers to fputc.o(i.fputc) for fputc
    printfa.o(i.__0vprintf) refers (Special) to iusefp.o(.text) for __I$use$fp
    printfa.o(i.__0vprintf) refers to printfa.o(i._printf_core) for _printf_core
    printfa.o(i.__0vprintf) refers to fputc.o(i.fputc) for fputc
    printfa.o(i.__0vprintf) refers to stdout.o(.data) for __stdout
    printfa.o(i.__0vsnprintf) refers (Special) to iusefp.o(.text) for __I$use$fp
    printfa.o(i.__0vsnprintf) refers to printfa.o(i._printf_core) for _printf_core
    printfa.o(i.__0vsnprintf) refers to printfa.o(i._snputc) for _snputc
    printfa.o(i.__0vsprintf) refers (Special) to iusefp.o(.text) for __I$use$fp
    printfa.o(i.__0vsprintf) refers to printfa.o(i._printf_core) for _printf_core
    printfa.o(i.__0vsprintf) refers to printfa.o(i._sputc) for _sputc
    printfa.o(i._fp_digits) refers (Special) to iusefp.o(.text) for __I$use$fp
    printfa.o(i._fp_digits) refers to dmul.o(.text) for __aeabi_dmul
    printfa.o(i._fp_digits) refers to ddiv.o(.text) for __aeabi_ddiv
    printfa.o(i._fp_digits) refers to cdrcmple.o(.text) for __aeabi_cdrcmple
    printfa.o(i._fp_digits) refers to dadd.o(.text) for __aeabi_dadd
    printfa.o(i._fp_digits) refers to dfixul.o(.text) for __aeabi_d2ulz
    printfa.o(i._fp_digits) refers to uldiv.o(.text) for __aeabi_uldivmod
    printfa.o(i._printf_core) refers (Special) to iusefp.o(.text) for __I$use$fp
    printfa.o(i._printf_core) refers to printfa.o(i._printf_pre_padding) for _printf_pre_padding
    printfa.o(i._printf_core) refers to uldiv.o(.text) for __aeabi_uldivmod
    printfa.o(i._printf_core) refers to printfa.o(i._printf_post_padding) for _printf_post_padding
    printfa.o(i._printf_core) refers to printfa.o(i._fp_digits) for _fp_digits
    printfa.o(i._printf_core) refers to uidiv.o(.text) for __aeabi_uidivmod
    printfa.o(i._printf_post_padding) refers (Special) to iusefp.o(.text) for __I$use$fp
    printfa.o(i._printf_pre_padding) refers (Special) to iusefp.o(.text) for __I$use$fp
    printfa.o(i._snputc) refers (Special) to iusefp.o(.text) for __I$use$fp
    printfa.o(i._sputc) refers (Special) to iusefp.o(.text) for __I$use$fp
    __0sscanf.o(.text) refers to scanf_char.o(.text) for __vfscanf_char
    __0sscanf.o(.text) refers to _sgetc.o(.text) for _sgetc
    _scanf_int.o(.text) refers to _chval.o(.text) for _chval
    fputc.o(i.fputc) refers (Special) to iusesemip.o(.text) for __I$use$semihosting$fputc
    fputc.o(i.fputc) refers (Special) to semi.o(.text) for __semihosting_library_function
    fputc_h.o(i._fputc$hlt) refers (Special) to iusesemip.o(.text) for __I$use$semihosting$fputc
    fputc_h.o(i._fputc$hlt) refers (Special) to semi.o(.text) for __semihosting_library_function
    scanf_char.o(.text) refers to _scanf.o(.text) for __vfscanf
    scanf_char.o(.text) refers to isspace_c.o(.text) for isspace
    dadd.o(.text) refers (Special) to iusefp.o(.text) for __I$use$fp
    dadd.o(.text) refers to llshl.o(.text) for __aeabi_llsl
    dadd.o(.text) refers to llsshr.o(.text) for __aeabi_lasr
    dadd.o(.text) refers to depilogue.o(.text) for _double_epilogue
    dmul.o(.text) refers (Special) to iusefp.o(.text) for __I$use$fp
    dmul.o(.text) refers to depilogue.o(.text) for _double_epilogue
    ddiv.o(.text) refers (Special) to iusefp.o(.text) for __I$use$fp
    ddiv.o(.text) refers to depilogue.o(.text) for _double_round
    dfixul.o(.text) refers (Special) to iusefp.o(.text) for __I$use$fp
    dfixul.o(.text) refers to llushr.o(.text) for __aeabi_llsr
    dfixul.o(.text) refers to llshl.o(.text) for __aeabi_llsl
    cdrcmple.o(.text) refers (Special) to iusefp.o(.text) for __I$use$fp
    isspace_c.o(.text) refers to ctype_c.o(.text) for __ctype_lookup
    _scanf.o(.text) refers (Weak) to _scanf_int.o(.text) for _scanf_int
    depilogue.o(.text) refers (Special) to iusefp.o(.text) for __I$use$fp
    depilogue.o(.text) refers to llshl.o(.text) for __aeabi_llsl
    depilogue.o(.text) refers to llushr.o(.text) for __aeabi_llsr
    ctype_c.o(.text) refers to ctype_c.o(.constdata) for .constdata


==============================================================================

Removing Unused input sections from the image.

    Removing hal_entry.o(.text), (0 bytes).
    Removing hal_entry.o(.text.getSystemTicks), (14 bytes).
    Removing hal_entry.o(.ARM.exidx.text.getSystemTicks), (8 bytes).
    Removing hal_entry.o(.text.SystickInit), (70 bytes).
    Removing hal_entry.o(.ARM.exidx.text.SystickInit), (8 bytes).
    Removing hal_entry.o(.ARM.exidx.text.SysTick_Handler), (8 bytes).
    Removing hal_entry.o(.ARM.exidx.text.read_button_GPIO), (8 bytes).
    Removing hal_entry.o(.ARM.exidx.text.Callback_btn_Handler), (8 bytes).
    Removing hal_entry.o(.text.DAC_SetVoltage), (48 bytes).
    Removing hal_entry.o(.ARM.exidx.text.DAC_SetVoltage), (8 bytes).
    Removing hal_entry.o(.text.GPT2_PWMA_SetDuty), (70 bytes).
    Removing hal_entry.o(.ARM.exidx.text.GPT2_PWMA_SetDuty), (8 bytes).
    Removing hal_entry.o(.text.dwt_timestamp_init), (38 bytes).
    Removing hal_entry.o(.ARM.exidx.text.dwt_timestamp_init), (8 bytes).
    Removing hal_entry.o(.ARM.exidx.text.hal_entry), (8 bytes).
    Removing hal_entry.o(.ARM.exidx.text.R_BSP_WarmStart), (8 bytes).
    Removing hal_entry.o(.ARM.exidx.text.user_timer0_callback), (8 bytes).
    Removing hal_entry.o(.ARM.exidx.text.user_timer5_callback), (8 bytes).
    Removing shell.o(.text), (0 bytes).
    Removing shell.o(.ARM.exidx.text.shellInit), (8 bytes).
    Removing shell.o(.ARM.exidx.text.shellSetUser), (8 bytes).
    Removing shell.o(.ARM.exidx.text.shellSeekCommand), (8 bytes).
    Removing shell.o(.ARM.exidx.text.shellWritePrompt), (8 bytes).
    Removing shell.o(.text.shellRemove), (36 bytes).
    Removing shell.o(.ARM.exidx.text.shellRemove), (8 bytes).
    Removing shell.o(.ARM.exidx.text.shellGetCurrent), (8 bytes).
    Removing shell.o(.text.shellWriteString), (50 bytes).
    Removing shell.o(.ARM.exidx.text.shellWriteString), (8 bytes).
    Removing shell.o(.ARM.exidx.text.shellPrint), (8 bytes).
    Removing shell.o(.ARM.exidx.text.shellCheckPermission), (8 bytes).
    Removing shell.o(.text.shellToHex), (54 bytes).
    Removing shell.o(.ARM.exidx.text.shellToHex), (8 bytes).
    Removing shell.o(.ARM.exidx.text.shellToDec), (8 bytes).
    Removing shell.o(.ARM.exidx.text.shellListItem), (8 bytes).
    Removing shell.o(.ARM.exidx.text.shellGetCommandName), (8 bytes).
    Removing shell.o(.ARM.exidx.text.shellListCommand), (8 bytes).
    Removing shell.o(.ARM.exidx.text.shellListVar), (8 bytes).
    Removing shell.o(.ARM.exidx.text.shellListUser), (8 bytes).
    Removing shell.o(.ARM.exidx.text.shellListKey), (8 bytes).
    Removing shell.o(.text.shellListAll), (4 bytes).
    Removing shell.o(.ARM.exidx.text.shellListAll), (8 bytes).
    Removing shell.o(.text.shellDeleteCommandLine), (34 bytes).
    Removing shell.o(.ARM.exidx.text.shellDeleteCommandLine), (8 bytes).
    Removing shell.o(.ARM.exidx.text.shellClearCommandLine), (8 bytes).
    Removing shell.o(.ARM.exidx.text.shellInsertByte), (8 bytes).
    Removing shell.o(.ARM.exidx.text.shellDeleteByte), (8 bytes).
    Removing shell.o(.ARM.exidx.text.shellSplit), (8 bytes).
    Removing shell.o(.ARM.exidx.text.shellGetVarValue), (8 bytes).
    Removing shell.o(.ARM.exidx.text.shellSetVarValue), (8 bytes).
    Removing shell.o(.ARM.exidx.text.shellShowVar), (8 bytes).
    Removing shell.o(.ARM.exidx.text.shellSetVar), (8 bytes).
    Removing shell.o(.ARM.exidx.text.shellRunCommand), (8 bytes).
    Removing shell.o(.ARM.exidx.text.shellWriteReturnValue), (8 bytes).
    Removing shell.o(.text.shellNormalInput), (16 bytes).
    Removing shell.o(.ARM.exidx.text.shellNormalInput), (8 bytes).
    Removing shell.o(.ARM.exidx.text.shellExec), (8 bytes).
    Removing shell.o(.ARM.exidx.text.shellUp), (8 bytes).
    Removing shell.o(.ARM.exidx.text.shellHistory), (8 bytes).
    Removing shell.o(.ARM.exidx.text.shellDown), (8 bytes).
    Removing shell.o(.ARM.exidx.text.shellRight), (8 bytes).
    Removing shell.o(.ARM.exidx.text.shellLeft), (8 bytes).
    Removing shell.o(.ARM.exidx.text.shellTab), (8 bytes).
    Removing shell.o(.ARM.exidx.text.shellBackspace), (8 bytes).
    Removing shell.o(.ARM.exidx.text.shellDelete), (8 bytes).
    Removing shell.o(.ARM.exidx.text.shellEnter), (8 bytes).
    Removing shell.o(.ARM.exidx.text.shellHelp), (8 bytes).
    Removing shell.o(.ARM.exidx.text.shellHandler), (8 bytes).
    Removing shell.o(.ARM.exidx.text.shellWriteEndLine), (8 bytes).
    Removing shell.o(.text.shellTask), (36 bytes).
    Removing shell.o(.ARM.exidx.text.shellTask), (8 bytes).
    Removing shell.o(.ARM.exidx.text.shellUsers), (8 bytes).
    Removing shell.o(.ARM.exidx.text.shellCmds), (8 bytes).
    Removing shell.o(.ARM.exidx.text.shellVars), (8 bytes).
    Removing shell.o(.ARM.exidx.text.shellKeys), (8 bytes).
    Removing shell.o(.ARM.exidx.text.shellClear), (8 bytes).
    Removing shell.o(.text.shellRun), (124 bytes).
    Removing shell.o(.ARM.exidx.text.shellRun), (8 bytes).
    Removing shell_cmd_list.o(.text), (0 bytes).
    Removing shell_companion.o(.text), (0 bytes).
    Removing shell_companion.o(.ARM.exidx.text.shellCompanionAdd), (8 bytes).
    Removing shell_companion.o(.text.shellCompanionDel), (74 bytes).
    Removing shell_companion.o(.ARM.exidx.text.shellCompanionDel), (8 bytes).
    Removing shell_companion.o(.ARM.exidx.text.shellCompanionGet), (8 bytes).
    Removing shell_ext.o(.text), (0 bytes).
    Removing shell_ext.o(.ARM.exidx.text.shellExtParsePara), (8 bytes).
    Removing shell_ext.o(.ARM.exidx.text.shellExtParseChar), (8 bytes).
    Removing shell_ext.o(.ARM.exidx.text.shellExtRun), (8 bytes).
    Removing shell_port_1.o(.text), (0 bytes).
    Removing shell_port_1.o(.ARM.exidx.text.userShellWrite), (8 bytes).
    Removing shell_port_1.o(.text.userShellRead), (4 bytes).
    Removing shell_port_1.o(.ARM.exidx.text.userShellRead), (8 bytes).
    Removing shell_port_1.o(.text.userShellLock), (4 bytes).
    Removing shell_port_1.o(.ARM.exidx.text.userShellLock), (8 bytes).
    Removing shell_port_1.o(.text.userShellUnlock), (4 bytes).
    Removing shell_port_1.o(.ARM.exidx.text.userShellUnlock), (8 bytes).
    Removing shell_port_1.o(.ARM.exidx.text.uartLogWrite), (8 bytes).
    Removing shell_port_1.o(.ARM.exidx.text.userShellInit), (8 bytes).
    Removing shell_cmds.o(.text), (0 bytes).
    Removing shell_cmds.o(.ARM.exidx.text.cmd_rd), (8 bytes).
    Removing shell_cmds.o(.ARM.exidx.text.cmd_wr), (8 bytes).
    Removing shell_cmds.o(.ARM.exidx.text.cmd_hex2dec), (8 bytes).
    Removing shell_cmds.o(.ARM.exidx.text.cmd_time), (8 bytes).
    Removing log.o(.text), (0 bytes).
    Removing log.o(.ARM.exidx.text.logRegister), (8 bytes).
    Removing log.o(.text.logUnRegister), (36 bytes).
    Removing log.o(.ARM.exidx.text.logUnRegister), (8 bytes).
    Removing log.o(.text.logSetLevel), (74 bytes).
    Removing log.o(.ARM.exidx.text.logSetLevel), (8 bytes).
    Removing log.o(.ARM.exidx.text.logWrite), (8 bytes).
    Removing log.o(.ARM.exidx.text.agencylogSetLevel), (8 bytes).
    Removing log.o(.ARM.exidx.text.logWriteBuffer), (8 bytes).
    Removing log.o(.ARM.exidx.text.logHexDump), (8 bytes).
    Removing log.o(.ARM.exidx.text.agencylogHexDump), (8 bytes).
    Removing log.o(.ARM.exidx.text.logSwitchLevel), (8 bytes).
    Removing lwrb.o(.text), (0 bytes).
    Removing lwrb.o(.ARM.exidx.text.lwrb_init), (8 bytes).
    Removing lwrb.o(.text.lwrb_is_ready), (20 bytes).
    Removing lwrb.o(.ARM.exidx.text.lwrb_is_ready), (8 bytes).
    Removing lwrb.o(.text.lwrb_free), (16 bytes).
    Removing lwrb.o(.ARM.exidx.text.lwrb_free), (8 bytes).
    Removing lwrb.o(.text.lwrb_set_evt_fn), (14 bytes).
    Removing lwrb.o(.ARM.exidx.text.lwrb_set_evt_fn), (8 bytes).
    Removing lwrb.o(.text.lwrb_set_arg), (14 bytes).
    Removing lwrb.o(.ARM.exidx.text.lwrb_set_arg), (8 bytes).
    Removing lwrb.o(.text.lwrb_get_arg), (10 bytes).
    Removing lwrb.o(.ARM.exidx.text.lwrb_get_arg), (8 bytes).
    Removing lwrb.o(.ARM.exidx.text.lwrb_write), (8 bytes).
    Removing lwrb.o(.ARM.exidx.text.lwrb_write_ex), (8 bytes).
    Removing lwrb.o(.text.lwrb_get_free), (32 bytes).
    Removing lwrb.o(.ARM.exidx.text.lwrb_get_free), (8 bytes).
    Removing lwrb.o(.ARM.exidx.text.lwrb_read), (8 bytes).
    Removing lwrb.o(.ARM.exidx.text.lwrb_read_ex), (8 bytes).
    Removing lwrb.o(.ARM.exidx.text.lwrb_get_full), (8 bytes).
    Removing lwrb.o(.text.lwrb_peek), (110 bytes).
    Removing lwrb.o(.ARM.exidx.text.lwrb_peek), (8 bytes).
    Removing lwrb.o(.text.lwrb_reset), (40 bytes).
    Removing lwrb.o(.ARM.exidx.text.lwrb_reset), (8 bytes).
    Removing lwrb.o(.text.lwrb_get_linear_block_read_address), (20 bytes).
    Removing lwrb.o(.ARM.exidx.text.lwrb_get_linear_block_read_address), (8 bytes).
    Removing lwrb.o(.text.lwrb_get_linear_block_read_length), (36 bytes).
    Removing lwrb.o(.ARM.exidx.text.lwrb_get_linear_block_read_length), (8 bytes).
    Removing lwrb.o(.text.lwrb_skip), (78 bytes).
    Removing lwrb.o(.ARM.exidx.text.lwrb_skip), (8 bytes).
    Removing lwrb.o(.text.lwrb_get_linear_block_write_address), (20 bytes).
    Removing lwrb.o(.ARM.exidx.text.lwrb_get_linear_block_write_address), (8 bytes).
    Removing lwrb.o(.text.lwrb_get_linear_block_write_length), (38 bytes).
    Removing lwrb.o(.ARM.exidx.text.lwrb_get_linear_block_write_length), (8 bytes).
    Removing lwrb.o(.text.lwrb_advance), (82 bytes).
    Removing lwrb.o(.ARM.exidx.text.lwrb_advance), (8 bytes).
    Removing lwrb.o(.text.lwrb_find), (172 bytes).
    Removing lwrb.o(.ARM.exidx.text.lwrb_find), (8 bytes).
    Removing lwrb_ex.o(.text), (0 bytes).
    Removing multi_button.o(.text), (0 bytes).
    Removing multi_button.o(.ARM.exidx.text.button_init), (8 bytes).
    Removing multi_button.o(.ARM.exidx.text.button_attach), (8 bytes).
    Removing multi_button.o(.text.get_button_event), (6 bytes).
    Removing multi_button.o(.ARM.exidx.text.get_button_event), (8 bytes).
    Removing multi_button.o(.ARM.exidx.text.button_start), (8 bytes).
    Removing multi_button.o(.text.button_stop), (48 bytes).
    Removing multi_button.o(.ARM.exidx.text.button_stop), (8 bytes).
    Removing multi_button.o(.ARM.exidx.text.button_ticks), (8 bytes).
    Removing startup.o(.text), (0 bytes).
    Removing startup.o(.ARM.exidx.text.Reset_Handler), (8 bytes).
    Removing startup.o(.ARM.exidx.text.Default_Handler), (8 bytes).
    Removing system.o(.text), (0 bytes).
    Removing system.o(.ARM.exidx.text.SystemInit), (8 bytes).
    Removing system.o(.text.R_BSP_WarmStart), (2 bytes).
    Removing system.o(.ARM.exidx.text.R_BSP_WarmStart), (8 bytes).
    Removing bsp_clocks.o(.text), (0 bytes).
    Removing bsp_clocks.o(.text.bsp_prv_operating_mode_set), (68 bytes).
    Removing bsp_clocks.o(.ARM.exidx.text.bsp_prv_operating_mode_set), (8 bytes).
    Removing bsp_clocks.o(.text.bsp_prv_prepare_pll), (24 bytes).
    Removing bsp_clocks.o(.ARM.exidx.text.bsp_prv_prepare_pll), (8 bytes).
    Removing bsp_clocks.o(.ARM.exidx.text.SystemCoreClockUpdate), (8 bytes).
    Removing bsp_clocks.o(.text.prv_clock_dividers_set), (12 bytes).
    Removing bsp_clocks.o(.ARM.exidx.text.prv_clock_dividers_set), (8 bytes).
    Removing bsp_clocks.o(.text.bsp_prv_clock_set), (182 bytes).
    Removing bsp_clocks.o(.ARM.exidx.text.bsp_prv_clock_set), (8 bytes).
    Removing bsp_clocks.o(.ARM.exidx.text.bsp_clock_init), (8 bytes).
    Removing bsp_clocks.o(.text.R_BSP_SubClockStabilizeWait), (8 bytes).
    Removing bsp_clocks.o(.ARM.exidx.text.R_BSP_SubClockStabilizeWait), (8 bytes).
    Removing bsp_clocks.o(.ARM.exidx.text.R_BSP_SubClockStabilizeWaitAfterReset), (8 bytes).
    Removing bsp_clocks.o(.text.R_BSP_OctaclkUpdate), (2 bytes).
    Removing bsp_clocks.o(.ARM.exidx.text.R_BSP_OctaclkUpdate), (8 bytes).
    Removing bsp_clocks.o(.ARM.exidx.text.R_BSP_SourceClockHzGet), (8 bytes).
    Removing bsp_clocks.o(.ARM.exidx.text.R_BSP_Init_RTC), (8 bytes).
    Removing bsp_common.o(.text), (0 bytes).
    Removing bsp_common.o(.ARM.exidx.text.bsp_init_internal), (8 bytes).
    Removing bsp_common.o(.text.R_FSP_VersionGet), (14 bytes).
    Removing bsp_common.o(.ARM.exidx.text.R_FSP_VersionGet), (8 bytes).
    Removing bsp_common.o(.ARM.exidx.text.__aeabi_assert), (8 bytes).
    Removing bsp_delay.o(.text), (0 bytes).
    Removing bsp_delay.o(.ARM.exidx.text.R_BSP_SoftwareDelay), (8 bytes).
    Removing bsp_delay.o(.ARM.exidx.text.bsp_prv_software_delay_loop), (8 bytes).
    Removing bsp_group_irq.o(.text), (0 bytes).
    Removing bsp_group_irq.o(.text.R_BSP_GroupIrqWrite), (18 bytes).
    Removing bsp_group_irq.o(.ARM.exidx.text.R_BSP_GroupIrqWrite), (8 bytes).
    Removing bsp_group_irq.o(.ARM.exidx.text.NMI_Handler), (8 bytes).
    Removing bsp_guard.o(.text), (0 bytes).
    Removing bsp_io.o(.text), (0 bytes).
    Removing bsp_irq.o(.text), (0 bytes).
    Removing bsp_irq.o(.ARM.exidx.text.bsp_irq_cfg), (8 bytes).
    Removing bsp_irq.o(.rodata.g_interrupt_event_link_select), (36 bytes).
    Removing bsp_macl.o(.text), (0 bytes).
    Removing bsp_register_protection.o(.text), (0 bytes).
    Removing bsp_register_protection.o(.ARM.exidx.text.R_BSP_RegisterProtectEnable), (8 bytes).
    Removing bsp_register_protection.o(.ARM.exidx.text.R_BSP_RegisterProtectDisable), (8 bytes).
    Removing bsp_rom_registers.o(.text), (0 bytes).
    Removing bsp_sbrk.o(.text), (0 bytes).
    Removing bsp_sdram.o(.text), (0 bytes).
    Removing bsp_security.o(.text), (0 bytes).
    Removing r_ioport.o(.text), (0 bytes).
    Removing r_ioport.o(.ARM.exidx.text.R_IOPORT_Open), (8 bytes).
    Removing r_ioport.o(.ARM.exidx.text.R_IOPORT_Close), (8 bytes).
    Removing r_ioport.o(.ARM.exidx.text.R_IOPORT_PinsCfg), (8 bytes).
    Removing r_ioport.o(.ARM.exidx.text.R_IOPORT_PinCfg), (8 bytes).
    Removing r_ioport.o(.ARM.exidx.text.R_IOPORT_PinEventInputRead), (8 bytes).
    Removing r_ioport.o(.ARM.exidx.text.R_IOPORT_PinEventOutputWrite), (8 bytes).
    Removing r_ioport.o(.ARM.exidx.text.R_IOPORT_PinRead), (8 bytes).
    Removing r_ioport.o(.ARM.exidx.text.R_IOPORT_PinWrite), (8 bytes).
    Removing r_ioport.o(.ARM.exidx.text.R_IOPORT_PortDirectionSet), (8 bytes).
    Removing r_ioport.o(.ARM.exidx.text.R_IOPORT_PortEventInputRead), (8 bytes).
    Removing r_ioport.o(.ARM.exidx.text.R_IOPORT_PortEventOutputWrite), (8 bytes).
    Removing r_ioport.o(.ARM.exidx.text.R_IOPORT_PortRead), (8 bytes).
    Removing r_ioport.o(.ARM.exidx.text.R_IOPORT_PortWrite), (8 bytes).
    Removing r_ioport.o(.ARM.exidx.text.r_ioport_pins_config), (8 bytes).
    Removing r_ioport.o(.ARM.exidx.text.bsp_vbatt_init), (8 bytes).
    Removing r_sci_uart.o(.text), (0 bytes).
    Removing r_sci_uart.o(.ARM.exidx.text.user_uart9_callback), (8 bytes).
    Removing r_sci_uart.o(.ARM.exidx.text.uart9_wait_for_tx), (8 bytes).
    Removing r_sci_uart.o(.text.uart9_wait_for_rx), (20 bytes).
    Removing r_sci_uart.o(.ARM.exidx.text.uart9_wait_for_rx), (8 bytes).
    Removing r_sci_uart.o(.ARM.exidx.text.R_SCI_UART_Open), (8 bytes).
    Removing r_sci_uart.o(.ARM.exidx.text.R_SCI_UART_Read), (8 bytes).
    Removing r_sci_uart.o(.ARM.exidx.text.R_SCI_UART_Write), (8 bytes).
    Removing r_sci_uart.o(.ARM.exidx.text.R_SCI_UART_BaudSet), (8 bytes).
    Removing r_sci_uart.o(.ARM.exidx.text.R_SCI_UART_InfoGet), (8 bytes).
    Removing r_sci_uart.o(.ARM.exidx.text.R_SCI_UART_Abort), (8 bytes).
    Removing r_sci_uart.o(.ARM.exidx.text.R_SCI_UART_CallbackSet), (8 bytes).
    Removing r_sci_uart.o(.ARM.exidx.text.R_SCI_UART_Close), (8 bytes).
    Removing r_sci_uart.o(.ARM.exidx.text.R_SCI_UART_ReadStop), (8 bytes).
    Removing r_sci_uart.o(.text.R_SCI_UART_BaudCalculate), (400 bytes).
    Removing r_sci_uart.o(.ARM.exidx.text.R_SCI_UART_BaudCalculate), (8 bytes).
    Removing r_sci_uart.o(.ARM.exidx.text.sci_uart_txi_isr), (8 bytes).
    Removing r_sci_uart.o(.ARM.exidx.text.r_sci_uart_call_callback), (8 bytes).
    Removing r_sci_uart.o(.ARM.exidx.text.sci_uart_rxi_isr), (8 bytes).
    Removing r_sci_uart.o(.ARM.exidx.text.sci_uart_tei_isr), (8 bytes).
    Removing r_sci_uart.o(.ARM.exidx.text.sci_uart_eri_isr), (8 bytes).
    Removing r_sci_uart.o(.rodata.g_async_baud), (13 bytes).
    Removing r_sci_uart.o(.rodata.g_div_coefficient), (26 bytes).
    Removing common_data.o(.text), (0 bytes).
    Removing common_data.o(.text.g_common_init), (2 bytes).
    Removing common_data.o(.ARM.exidx.text.g_common_init), (8 bytes).
    Removing hal_data.o(.text), (0 bytes).
    Removing hal_data.o(.text.g_hal_init), (4 bytes).
    Removing hal_data.o(.ARM.exidx.text.g_hal_init), (8 bytes).
    Removing main.o(.text), (0 bytes).
    Removing main.o(.ARM.exidx.text.main), (8 bytes).
    Removing main.o(.ARM.use_no_argv), (4 bytes).
    Removing pin_data.o(.text), (0 bytes).
    Removing vector_data.o(.text), (0 bytes).
    Removing r_adc.o(.text), (0 bytes).
    Removing r_adc.o(.ARM.exidx.text.R_ADC_Open), (8 bytes).
    Removing r_adc.o(.ARM.exidx.text.R_ADC_ScanCfg), (8 bytes).
    Removing r_adc.o(.ARM.exidx.text.R_ADC_ScanStart), (8 bytes).
    Removing r_adc.o(.ARM.exidx.text.R_ADC_ScanGroupStart), (8 bytes).
    Removing r_adc.o(.ARM.exidx.text.R_ADC_ScanStop), (8 bytes).
    Removing r_adc.o(.ARM.exidx.text.R_ADC_StatusGet), (8 bytes).
    Removing r_adc.o(.ARM.exidx.text.R_ADC_Read), (8 bytes).
    Removing r_adc.o(.ARM.exidx.text.R_ADC_Read32), (8 bytes).
    Removing r_adc.o(.ARM.exidx.text.R_ADC_Calibrate), (8 bytes).
    Removing r_adc.o(.ARM.exidx.text.R_ADC_OffsetSet), (8 bytes).
    Removing r_adc.o(.ARM.exidx.text.R_ADC_CallbackSet), (8 bytes).
    Removing r_adc.o(.ARM.exidx.text.R_ADC_Close), (8 bytes).
    Removing r_adc.o(.ARM.exidx.text.R_ADC_InfoGet), (8 bytes).
    Removing r_adc.o(.ARM.exidx.text.r_adc_irq_enable), (8 bytes).
    Removing r_adc.o(.text.R_ADC_SampleStateCountSet), (16 bytes).
    Removing r_adc.o(.ARM.exidx.text.R_ADC_SampleStateCountSet), (8 bytes).
    Removing r_adc.o(.ARM.exidx.text.adc_scan_end_isr), (8 bytes).
    Removing r_adc.o(.ARM.exidx.text.r_adc_scan_end_common_isr), (8 bytes).
    Removing r_adc.o(.text.adc_scan_end_b_isr), (6 bytes).
    Removing r_adc.o(.ARM.exidx.text.adc_scan_end_b_isr), (8 bytes).
    Removing r_adc.o(.text.adc_window_compare_isr), (324 bytes).
    Removing r_adc.o(.ARM.exidx.text.adc_window_compare_isr), (8 bytes).
    Removing r_adc.o(.ARM.exidx.text.user_adc_callback), (8 bytes).
    Removing r_adc.o(.text.adc_wait_for_scan), (20 bytes).
    Removing r_adc.o(.ARM.exidx.text.adc_wait_for_scan), (8 bytes).
    Removing r_adc.o(.ARM.exidx.text.get_adc_scan_status), (8 bytes).
    Removing r_adc.o(.ARM.exidx.text.reset_adc_scan_state), (8 bytes).
    Removing r_dac.o(.text), (0 bytes).
    Removing r_dac.o(.ARM.exidx.text.R_DAC_Open), (8 bytes).
    Removing r_dac.o(.ARM.exidx.text.R_DAC_Close), (8 bytes).
    Removing r_dac.o(.ARM.exidx.text.R_DAC_Write), (8 bytes).
    Removing r_dac.o(.ARM.exidx.text.R_DAC_Start), (8 bytes).
    Removing r_dac.o(.ARM.exidx.text.R_DAC_Stop), (8 bytes).
    Removing r_gpt.o(.text), (0 bytes).
    Removing r_gpt.o(.ARM.exidx.text.R_GPT_Open), (8 bytes).
    Removing r_gpt.o(.ARM.exidx.text.R_GPT_Start), (8 bytes).
    Removing r_gpt.o(.ARM.exidx.text.R_GPT_Stop), (8 bytes).
    Removing r_gpt.o(.ARM.exidx.text.R_GPT_Reset), (8 bytes).
    Removing r_gpt.o(.ARM.exidx.text.R_GPT_Enable), (8 bytes).
    Removing r_gpt.o(.ARM.exidx.text.R_GPT_Disable), (8 bytes).
    Removing r_gpt.o(.ARM.exidx.text.R_GPT_PeriodSet), (8 bytes).
    Removing r_gpt.o(.ARM.exidx.text.R_GPT_DutyCycleSet), (8 bytes).
    Removing r_gpt.o(.ARM.exidx.text.R_GPT_CompareMatchSet), (8 bytes).
    Removing r_gpt.o(.ARM.exidx.text.R_GPT_InfoGet), (8 bytes).
    Removing r_gpt.o(.ARM.exidx.text.R_GPT_StatusGet), (8 bytes).
    Removing r_gpt.o(.ARM.exidx.text.R_GPT_CallbackSet), (8 bytes).
    Removing r_gpt.o(.ARM.exidx.text.R_GPT_Close), (8 bytes).
    Removing r_gpt.o(.ARM.exidx.text.gpt_calculate_duty_cycle), (8 bytes).
    Removing r_gpt.o(.text.R_GPT_CounterSet), (8 bytes).
    Removing r_gpt.o(.ARM.exidx.text.R_GPT_CounterSet), (8 bytes).
    Removing r_gpt.o(.text.R_GPT_OutputEnable), (26 bytes).
    Removing r_gpt.o(.ARM.exidx.text.R_GPT_OutputEnable), (8 bytes).
    Removing r_gpt.o(.text.R_GPT_OutputDisable), (26 bytes).
    Removing r_gpt.o(.ARM.exidx.text.R_GPT_OutputDisable), (8 bytes).
    Removing r_gpt.o(.text.R_GPT_AdcTriggerSet), (12 bytes).
    Removing r_gpt.o(.ARM.exidx.text.R_GPT_AdcTriggerSet), (8 bytes).
    Removing r_gpt.o(.text.R_GPT_PwmOutputDelaySet), (4 bytes).
    Removing r_gpt.o(.ARM.exidx.text.R_GPT_PwmOutputDelaySet), (8 bytes).
    Removing r_gpt.o(.text.R_GPT_PwmOutputDelayInitialize), (4 bytes).
    Removing r_gpt.o(.ARM.exidx.text.R_GPT_PwmOutputDelayInitialize), (8 bytes).
    Removing r_gpt.o(.ARM.exidx.text.gpt_counter_overflow_isr), (8 bytes).
    Removing r_gpt.o(.ARM.exidx.text.gpt_capture_compare_a_isr), (8 bytes).
    Removing r_gpt.o(.ARM.exidx.text.r_gpt_ccmp_common_isr), (8 bytes).
    Removing r_gpt.o(.ARM.exidx.text.gpt_capture_compare_b_isr), (8 bytes).
    Removing r_gpt.o(.ARM.exidx.text.r_gpt_enable_irq), (8 bytes).

327 unused section(s) (total 4651 bytes) removed from the image.

==============================================================================

Image Symbol Table

    Local Symbols

    Symbol Name                              Value     Ov Type        Size  Object(Section)

    ../clib/division.s                       0x00000000   Number         0  aeabi_sdiv.o ABSOLUTE
    ../clib/microlib/ctype/ctype.c           0x00000000   Number         0  isspace_c.o ABSOLUTE
    ../clib/microlib/ctype/ctype.c           0x00000000   Number         0  ctype_c.o ABSOLUTE
    ../clib/microlib/division.c              0x00000000   Number         0  uldiv.o ABSOLUTE
    ../clib/microlib/division.c              0x00000000   Number         0  ldiv.o ABSOLUTE
    ../clib/microlib/division.c              0x00000000   Number         0  uidiv.o ABSOLUTE
    ../clib/microlib/longlong.c              0x00000000   Number         0  llshl.o ABSOLUTE
    ../clib/microlib/longlong.c              0x00000000   Number         0  llushr.o ABSOLUTE
    ../clib/microlib/longlong.c              0x00000000   Number         0  llsshr.o ABSOLUTE
    ../clib/microlib/printf/printf.c         0x00000000   Number         0  printfb.o ABSOLUTE
    ../clib/microlib/printf/printf.c         0x00000000   Number         0  printf0.o ABSOLUTE
    ../clib/microlib/printf/printf.c         0x00000000   Number         0  printf1.o ABSOLUTE
    ../clib/microlib/printf/printf.c         0x00000000   Number         0  printf2.o ABSOLUTE
    ../clib/microlib/printf/printf.c         0x00000000   Number         0  printf3.o ABSOLUTE
    ../clib/microlib/printf/printf.c         0x00000000   Number         0  printf4.o ABSOLUTE
    ../clib/microlib/printf/printf.c         0x00000000   Number         0  printf5.o ABSOLUTE
    ../clib/microlib/printf/printf.c         0x00000000   Number         0  printf6.o ABSOLUTE
    ../clib/microlib/printf/printf.c         0x00000000   Number         0  printf7.o ABSOLUTE
    ../clib/microlib/printf/printf.c         0x00000000   Number         0  printf8.o ABSOLUTE
    ../clib/microlib/printf/printf.c         0x00000000   Number         0  printfa.o ABSOLUTE
    ../clib/microlib/printf/stubs.s          0x00000000   Number         0  printfstubs.o ABSOLUTE
    ../clib/microlib/stdio/fputc.c           0x00000000   Number         0  fputc.o ABSOLUTE
    ../clib/microlib/stdio/fputc.c           0x00000000   Number         0  fputc_h.o ABSOLUTE
    ../clib/microlib/stdio/puts.c            0x00000000   Number         0  puts.o ABSOLUTE
    ../clib/microlib/stdio/puts.c            0x00000000   Number         0  puts_e.o ABSOLUTE
    ../clib/microlib/stdio/semi.s            0x00000000   Number         0  semi.o ABSOLUTE
    ../clib/microlib/stdio/streams.c         0x00000000   Number         0  stdout.o ABSOLUTE
    ../clib/microlib/string/memcpy.c         0x00000000   Number         0  memcpya.o ABSOLUTE
    ../clib/microlib/string/memcpy.c         0x00000000   Number         0  memcpyb.o ABSOLUTE
    ../clib/microlib/string/memset.c         0x00000000   Number         0  memseta.o ABSOLUTE
    ../clib/microlib/string/strcmp.c         0x00000000   Number         0  strcmp.o ABSOLUTE
    ../clib/microlib/string/strlen.c         0x00000000   Number         0  strlen.o ABSOLUTE
    ../clib/microlib/string/strncmp.c        0x00000000   Number         0  strncmp.o ABSOLUTE
    ../clib/microlib/stubs.s                 0x00000000   Number         0  iusefp.o ABSOLUTE
    ../clib/microlib/stubs.s                 0x00000000   Number         0  iusesemip.o ABSOLUTE
    ../clib/scanf.c                          0x00000000   Number         0  __0sscanf.o ABSOLUTE
    ../clib/scanf.c                          0x00000000   Number         0  _scanf_int.o ABSOLUTE
    ../clib/scanf.c                          0x00000000   Number         0  _chval.o ABSOLUTE
    ../clib/scanf.c                          0x00000000   Number         0  scanf_char.o ABSOLUTE
    ../clib/scanf.c                          0x00000000   Number         0  _sgetc.o ABSOLUTE
    ../clib/scanf.c                          0x00000000   Number         0  _scanf.o ABSOLUTE
    ../fplib/microlib/fpadd.c                0x00000000   Number         0  dadd.o ABSOLUTE
    ../fplib/microlib/fpdiv.c                0x00000000   Number         0  ddiv.o ABSOLUTE
    ../fplib/microlib/fpepilogue.c           0x00000000   Number         0  depilogue.o ABSOLUTE
    ../fplib/microlib/fpfix.c                0x00000000   Number         0  dfixul.o ABSOLUTE
    ../fplib/microlib/fpmul.c                0x00000000   Number         0  dmul.o ABSOLUTE
    __tagsym$$used.1                         0x00000000   Number         0  startup.o(.fixed_vectors)
    bsp_clocks.c                             0x00000000   Number         0  bsp_clocks.o ABSOLUTE
    bsp_common.c                             0x00000000   Number         0  bsp_common.o ABSOLUTE
    bsp_delay.c                              0x00000000   Number         0  bsp_delay.o ABSOLUTE
    bsp_group_irq.c                          0x00000000   Number         0  bsp_group_irq.o ABSOLUTE
    bsp_guard.c                              0x00000000   Number         0  bsp_guard.o ABSOLUTE
    bsp_io.c                                 0x00000000   Number         0  bsp_io.o ABSOLUTE
    bsp_irq.c                                0x00000000   Number         0  bsp_irq.o ABSOLUTE
    bsp_macl.c                               0x00000000   Number         0  bsp_macl.o ABSOLUTE
    bsp_register_protection.c                0x00000000   Number         0  bsp_register_protection.o ABSOLUTE
    bsp_rom_registers.c                      0x00000000   Number         0  bsp_rom_registers.o ABSOLUTE
    bsp_sbrk.c                               0x00000000   Number         0  bsp_sbrk.o ABSOLUTE
    bsp_sdram.c                              0x00000000   Number         0  bsp_sdram.o ABSOLUTE
    bsp_security.c                           0x00000000   Number         0  bsp_security.o ABSOLUTE
    cdrcmple.s                               0x00000000   Number         0  cdrcmple.o ABSOLUTE
    common_data.c                            0x00000000   Number         0  common_data.o ABSOLUTE
    dc.s                                     0x00000000   Number         0  dc.o ABSOLUTE
    hal_data.c                               0x00000000   Number         0  hal_data.o ABSOLUTE
    hal_entry.c                              0x00000000   Number         0  hal_entry.o ABSOLUTE
    log.c                                    0x00000000   Number         0  log.o ABSOLUTE
    lwrb.c                                   0x00000000   Number         0  lwrb.o ABSOLUTE
    lwrb_ex.c                                0x00000000   Number         0  lwrb_ex.o ABSOLUTE
    main.c                                   0x00000000   Number         0  main.o ABSOLUTE
    multi_button.c                           0x00000000   Number         0  multi_button.o ABSOLUTE
    pin_data.c                               0x00000000   Number         0  pin_data.o ABSOLUTE
    r_adc.c                                  0x00000000   Number         0  r_adc.o ABSOLUTE
    r_dac.c                                  0x00000000   Number         0  r_dac.o ABSOLUTE
    r_gpt.c                                  0x00000000   Number         0  r_gpt.o ABSOLUTE
    r_ioport.c                               0x00000000   Number         0  r_ioport.o ABSOLUTE
    r_sci_uart.c                             0x00000000   Number         0  r_sci_uart.o ABSOLUTE
    shell.c                                  0x00000000   Number         0  shell.o ABSOLUTE
    shell_cmd_list.c                         0x00000000   Number         0  shell_cmd_list.o ABSOLUTE
    shell_cmds.c                             0x00000000   Number         0  shell_cmds.o ABSOLUTE
    shell_companion.c                        0x00000000   Number         0  shell_companion.o ABSOLUTE
    shell_ext.c                              0x00000000   Number         0  shell_ext.o ABSOLUTE
    shell_port.c                             0x00000000   Number         0  shell_port_1.o ABSOLUTE
    startup.c                                0x00000000   Number         0  startup.o ABSOLUTE
    system.c                                 0x00000000   Number         0  system.o ABSOLUTE
    vector_data.c                            0x00000000   Number         0  vector_data.o ABSOLUTE
    __tagsym$$used.0                         0x00000040   Number         0  vector_data.o(.application_vectors)
    .text                                    0x00000064   Section        0  uldiv.o(.text)
    .text                                    0x000000c6   Section        0  memcpya.o(.text)
    .text                                    0x000000ea   Section        0  memseta.o(.text)
    .text                                    0x0000010e   Section        0  strlen.o(.text)
    .text                                    0x0000011c   Section        0  strcmp.o(.text)
    .text                                    0x00000138   Section        0  strncmp.o(.text)
    .text                                    0x00000158   Section        0  __0sscanf.o(.text)
    .text                                    0x00000190   Section        0  _scanf_int.o(.text)
    .text                                    0x000002dc   Section        0  uidiv.o(.text)
    .text                                    0x00000308   Section        0  llshl.o(.text)
    .text                                    0x00000326   Section        0  llushr.o(.text)
    .text                                    0x00000346   Section        0  _chval.o(.text)
    _scanf_char_input                        0x00000365   Thumb Code    12  scanf_char.o(.text)
    .text                                    0x00000364   Section        0  scanf_char.o(.text)
    .text                                    0x0000038c   Section        0  _sgetc.o(.text)
    .text                                    0x000003cc   Section        0  iusefp.o(.text)
    .text                                    0x000003cc   Section        0  dadd.o(.text)
    .text                                    0x0000051a   Section        0  dmul.o(.text)
    .text                                    0x000005fe   Section        0  ddiv.o(.text)
    .text                                    0x000006dc   Section        0  dfixul.o(.text)
    .text                                    0x0000070c   Section       48  cdrcmple.o(.text)
    .text                                    0x0000073c   Section        0  semi.o(.text)
    .text                                    0x0000073c   Section        0  llsshr.o(.text)
    .text                                    0x00000760   Section        0  isspace_c.o(.text)
    .text                                    0x0000076c   Section        0  _scanf.o(.text)
    .text                                    0x00000a98   Section        0  iusesemip.o(.text)
    .text                                    0x00000a98   Section        0  depilogue.o(.text)
    .text                                    0x00000b54   Section        0  ctype_c.o(.text)
    [Anonymous Symbol]                       0x00000b7c   Section        0  hal_entry.o(.text.Callback_btn_Handler)
    [Anonymous Symbol]                       0x00000bf0   Section        0  startup.o(.text.Default_Handler)
    [Anonymous Symbol]                       0x00000bf4   Section        0  bsp_group_irq.o(.text.NMI_Handler)
    [Anonymous Symbol]                       0x00000c38   Section        0  r_adc.o(.text.R_ADC_Calibrate)
    [Anonymous Symbol]                       0x00000c3c   Section        0  r_adc.o(.text.R_ADC_CallbackSet)
    [Anonymous Symbol]                       0x00000c4a   Section        0  r_adc.o(.text.R_ADC_Close)
    [Anonymous Symbol]                       0x00000d30   Section        0  r_adc.o(.text.R_ADC_InfoGet)
    [Anonymous Symbol]                       0x00000d9c   Section        0  r_adc.o(.text.R_ADC_OffsetSet)
    [Anonymous Symbol]                       0x00000da0   Section        0  r_adc.o(.text.R_ADC_Open)
    [Anonymous Symbol]                       0x00000eae   Section        0  r_adc.o(.text.R_ADC_Read)
    [Anonymous Symbol]                       0x00000ebc   Section        0  r_adc.o(.text.R_ADC_Read32)
    [Anonymous Symbol]                       0x00000ed4   Section        0  r_adc.o(.text.R_ADC_ScanCfg)
    [Anonymous Symbol]                       0x000010a8   Section        0  r_adc.o(.text.R_ADC_ScanGroupStart)
    [Anonymous Symbol]                       0x000010ac   Section        0  r_adc.o(.text.R_ADC_ScanStart)
    [Anonymous Symbol]                       0x000010b6   Section        0  r_adc.o(.text.R_ADC_ScanStop)
    [Anonymous Symbol]                       0x000010c0   Section        0  r_adc.o(.text.R_ADC_StatusGet)
    [Anonymous Symbol]                       0x000010cc   Section        0  bsp_clocks.o(.text.R_BSP_Init_RTC)
    [Anonymous Symbol]                       0x00001146   Section        0  bsp_register_protection.o(.text.R_BSP_RegisterProtectDisable)
    [Anonymous Symbol]                       0x00001194   Section        0  bsp_register_protection.o(.text.R_BSP_RegisterProtectEnable)
    [Anonymous Symbol]                       0x000011e6   Section        0  bsp_delay.o(.text.R_BSP_SoftwareDelay)
    [Anonymous Symbol]                       0x0000122e   Section        0  bsp_clocks.o(.text.R_BSP_SourceClockHzGet)
    [Anonymous Symbol]                       0x0000123c   Section        0  bsp_clocks.o(.text.R_BSP_SubClockStabilizeWaitAfterReset)
    [Anonymous Symbol]                       0x0000123e   Section        0  hal_entry.o(.text.R_BSP_WarmStart)
    [Anonymous Symbol]                       0x00001258   Section        0  r_dac.o(.text.R_DAC_Close)
    [Anonymous Symbol]                       0x00001292   Section        0  r_dac.o(.text.R_DAC_Open)
    [Anonymous Symbol]                       0x00001350   Section        0  r_dac.o(.text.R_DAC_Start)
    [Anonymous Symbol]                       0x0000140e   Section        0  r_dac.o(.text.R_DAC_Stop)
    [Anonymous Symbol]                       0x00001436   Section        0  r_dac.o(.text.R_DAC_Write)
    [Anonymous Symbol]                       0x00001442   Section        0  r_gpt.o(.text.R_GPT_CallbackSet)
    [Anonymous Symbol]                       0x00001450   Section        0  r_gpt.o(.text.R_GPT_Close)
    [Anonymous Symbol]                       0x000014e4   Section        0  r_gpt.o(.text.R_GPT_CompareMatchSet)
    [Anonymous Symbol]                       0x000014f2   Section        0  r_gpt.o(.text.R_GPT_Disable)
    [Anonymous Symbol]                       0x00001510   Section        0  r_gpt.o(.text.R_GPT_DutyCycleSet)
    [Anonymous Symbol]                       0x000015bc   Section        0  r_gpt.o(.text.R_GPT_Enable)
    [Anonymous Symbol]                       0x000015f4   Section        0  r_gpt.o(.text.R_GPT_InfoGet)
    [Anonymous Symbol]                       0x00001630   Section        0  r_gpt.o(.text.R_GPT_Open)
    [Anonymous Symbol]                       0x00001870   Section        0  r_gpt.o(.text.R_GPT_PeriodSet)
    [Anonymous Symbol]                       0x000018a8   Section        0  r_gpt.o(.text.R_GPT_Reset)
    [Anonymous Symbol]                       0x000018b2   Section        0  r_gpt.o(.text.R_GPT_Start)
    [Anonymous Symbol]                       0x000018bc   Section        0  r_gpt.o(.text.R_GPT_StatusGet)
    [Anonymous Symbol]                       0x000018ce   Section        0  r_gpt.o(.text.R_GPT_Stop)
    [Anonymous Symbol]                       0x000018d8   Section        0  r_ioport.o(.text.R_IOPORT_Close)
    [Anonymous Symbol]                       0x000018e2   Section        0  r_ioport.o(.text.R_IOPORT_Open)
    [Anonymous Symbol]                       0x000018f8   Section        0  r_ioport.o(.text.R_IOPORT_PinCfg)
    [Anonymous Symbol]                       0x000019aa   Section        0  r_ioport.o(.text.R_IOPORT_PinEventInputRead)
    [Anonymous Symbol]                       0x000019d2   Section        0  r_ioport.o(.text.R_IOPORT_PinEventOutputWrite)
    [Anonymous Symbol]                       0x00001a24   Section        0  r_ioport.o(.text.R_IOPORT_PinRead)
    [Anonymous Symbol]                       0x00001a46   Section        0  r_ioport.o(.text.R_IOPORT_PinWrite)
    [Anonymous Symbol]                       0x00001a6e   Section        0  r_ioport.o(.text.R_IOPORT_PinsCfg)
    [Anonymous Symbol]                       0x00001a7a   Section        0  r_ioport.o(.text.R_IOPORT_PortDirectionSet)
    [Anonymous Symbol]                       0x00001aa6   Section        0  r_ioport.o(.text.R_IOPORT_PortEventInputRead)
    [Anonymous Symbol]                       0x00001abe   Section        0  r_ioport.o(.text.R_IOPORT_PortEventOutputWrite)
    [Anonymous Symbol]                       0x00001ade   Section        0  r_ioport.o(.text.R_IOPORT_PortRead)
    [Anonymous Symbol]                       0x00001af4   Section        0  r_ioport.o(.text.R_IOPORT_PortWrite)
    [Anonymous Symbol]                       0x00001b14   Section        0  r_sci_uart.o(.text.R_SCI_UART_Abort)
    [Anonymous Symbol]                       0x00001b36   Section        0  r_sci_uart.o(.text.R_SCI_UART_BaudSet)
    [Anonymous Symbol]                       0x00001b9e   Section        0  r_sci_uart.o(.text.R_SCI_UART_CallbackSet)
    [Anonymous Symbol]                       0x00001bac   Section        0  r_sci_uart.o(.text.R_SCI_UART_Close)
    [Anonymous Symbol]                       0x00001c52   Section        0  r_sci_uart.o(.text.R_SCI_UART_InfoGet)
    [Anonymous Symbol]                       0x00001c5e   Section        0  r_sci_uart.o(.text.R_SCI_UART_Open)
    [Anonymous Symbol]                       0x00001f98   Section        0  r_sci_uart.o(.text.R_SCI_UART_Read)
    [Anonymous Symbol]                       0x00001fa2   Section        0  r_sci_uart.o(.text.R_SCI_UART_ReadStop)
    [Anonymous Symbol]                       0x00001fb0   Section        0  r_sci_uart.o(.text.R_SCI_UART_Write)
    [Anonymous Symbol]                       0x00001ffc   Section        0  startup.o(.text.Reset_Handler)
    [Anonymous Symbol]                       0x00002006   Section        0  hal_entry.o(.text.SysTick_Handler)
    [Anonymous Symbol]                       0x0000201e   Section        0  bsp_clocks.o(.text.SystemCoreClockUpdate)
    [Anonymous Symbol]                       0x0000204c   Section        0  system.o(.text.SystemInit)
    [Anonymous Symbol]                       0x0000213c   Section        0  bsp_common.o(.text.__aeabi_assert)
    [Anonymous Symbol]                       0x00002142   Section        0  r_adc.o(.text.adc_scan_end_isr)
    [Anonymous Symbol]                       0x00002148   Section        0  log.o(.text.agencylogHexDump)
    [Anonymous Symbol]                       0x00002168   Section        0  log.o(.text.agencylogSetLevel)
    [Anonymous Symbol]                       0x000021c0   Section        0  bsp_clocks.o(.text.bsp_clock_init)
    [Anonymous Symbol]                       0x000022ea   Section        0  bsp_common.o(.text.bsp_init_internal)
    [Anonymous Symbol]                       0x000022ec   Section        0  bsp_irq.o(.text.bsp_irq_cfg)
    sw_delay_loop                            0x00002376   Number         0  bsp_delay.o(.text.bsp_prv_software_delay_loop)
    [Anonymous Symbol]                       0x00002376   Section        0  bsp_delay.o(.text.bsp_prv_software_delay_loop)
    bsp_vbatt_init                           0x00002381   Thumb Code   204  r_ioport.o(.text.bsp_vbatt_init)
    [Anonymous Symbol]                       0x00002380   Section        0  r_ioport.o(.text.bsp_vbatt_init)
    g_vbatt_pins_input                       0x0000244c   Number         0  r_ioport.o(.text.bsp_vbatt_init)
    [Anonymous Symbol]                       0x00002458   Section        0  multi_button.o(.text.button_attach)
    [Anonymous Symbol]                       0x00002460   Section        0  multi_button.o(.text.button_init)
    [Anonymous Symbol]                       0x0000248c   Section        0  multi_button.o(.text.button_start)
    [Anonymous Symbol]                       0x000024b4   Section        0  multi_button.o(.text.button_ticks)
    [Anonymous Symbol]                       0x00002690   Section        0  shell_cmds.o(.text.cmd_hex2dec)
    [Anonymous Symbol]                       0x00002720   Section        0  shell_cmds.o(.text.cmd_rd)
    [Anonymous Symbol]                       0x00002928   Section        0  shell_cmds.o(.text.cmd_time)
    [Anonymous Symbol]                       0x00002ae4   Section        0  shell_cmds.o(.text.cmd_wr)
    [Anonymous Symbol]                       0x00002c74   Section        0  r_adc.o(.text.get_adc_scan_status)
    gpt_calculate_duty_cycle                 0x00002c81   Thumb Code   110  r_gpt.o(.text.gpt_calculate_duty_cycle)
    [Anonymous Symbol]                       0x00002c80   Section        0  r_gpt.o(.text.gpt_calculate_duty_cycle)
    [Anonymous Symbol]                       0x00002cee   Section        0  r_gpt.o(.text.gpt_capture_compare_a_isr)
    [Anonymous Symbol]                       0x00002cf4   Section        0  r_gpt.o(.text.gpt_capture_compare_b_isr)
    [Anonymous Symbol]                       0x00002cfa   Section        0  r_gpt.o(.text.gpt_counter_overflow_isr)
    [Anonymous Symbol]                       0x00002da8   Section        0  hal_entry.o(.text.hal_entry)
    __arm_cp.8_8                             0x00003590   Number         4  hal_entry.o(.text.hal_entry)
    __arm_cp.8_9                             0x00003594   Number         4  hal_entry.o(.text.hal_entry)
    __arm_cp.8_10                            0x00003598   Number         4  hal_entry.o(.text.hal_entry)
    __arm_cp.8_11                            0x0000359c   Number         4  hal_entry.o(.text.hal_entry)
    __arm_cp.8_12                            0x000035a0   Number         4  hal_entry.o(.text.hal_entry)
    [Anonymous Symbol]                       0x00003624   Section        0  log.o(.text.logHexDump)
    [Anonymous Symbol]                       0x00003794   Section        0  log.o(.text.logRegister)
    [Anonymous Symbol]                       0x000037cc   Section        0  log.o(.text.logSwitchLevel)
    [Anonymous Symbol]                       0x00003810   Section        0  log.o(.text.logWrite)
    logWriteBuffer                           0x0000384d   Thumb Code    96  log.o(.text.logWriteBuffer)
    [Anonymous Symbol]                       0x0000384c   Section        0  log.o(.text.logWriteBuffer)
    [Anonymous Symbol]                       0x000038ac   Section        0  lwrb.o(.text.lwrb_get_full)
    [Anonymous Symbol]                       0x000038ca   Section        0  lwrb.o(.text.lwrb_init)
    [Anonymous Symbol]                       0x000038ee   Section        0  lwrb.o(.text.lwrb_read)
    [Anonymous Symbol]                       0x00003910   Section        0  lwrb.o(.text.lwrb_read_ex)
    [Anonymous Symbol]                       0x000039b4   Section        0  lwrb.o(.text.lwrb_write)
    [Anonymous Symbol]                       0x000039d6   Section        0  lwrb.o(.text.lwrb_write_ex)
    [Anonymous Symbol]                       0x00003a7e   Section        0  main.o(.text.main)
    r_adc_irq_enable                         0x00003a89   Thumb Code    88  r_adc.o(.text.r_adc_irq_enable)
    [Anonymous Symbol]                       0x00003a88   Section        0  r_adc.o(.text.r_adc_irq_enable)
    r_adc_scan_end_common_isr                0x00003ae1   Thumb Code   176  r_adc.o(.text.r_adc_scan_end_common_isr)
    [Anonymous Symbol]                       0x00003ae0   Section        0  r_adc.o(.text.r_adc_scan_end_common_isr)
    r_gpt_ccmp_common_isr                    0x00003b91   Thumb Code   214  r_gpt.o(.text.r_gpt_ccmp_common_isr)
    [Anonymous Symbol]                       0x00003b90   Section        0  r_gpt.o(.text.r_gpt_ccmp_common_isr)
    r_gpt_enable_irq                         0x00003c67   Thumb Code    88  r_gpt.o(.text.r_gpt_enable_irq)
    [Anonymous Symbol]                       0x00003c66   Section        0  r_gpt.o(.text.r_gpt_enable_irq)
    r_ioport_pins_config                     0x00003cc1   Thumb Code   196  r_ioport.o(.text.r_ioport_pins_config)
    [Anonymous Symbol]                       0x00003cc0   Section        0  r_ioport.o(.text.r_ioport_pins_config)
    r_sci_uart_call_callback                 0x00003d85   Thumb Code    64  r_sci_uart.o(.text.r_sci_uart_call_callback)
    [Anonymous Symbol]                       0x00003d84   Section        0  r_sci_uart.o(.text.r_sci_uart_call_callback)
    [Anonymous Symbol]                       0x00003dc4   Section        0  hal_entry.o(.text.read_button_GPIO)
    [Anonymous Symbol]                       0x00003dfc   Section        0  r_adc.o(.text.reset_adc_scan_state)
    [Anonymous Symbol]                       0x00003e0a   Section        0  r_sci_uart.o(.text.sci_uart_eri_isr)
    [Anonymous Symbol]                       0x00003e74   Section        0  r_sci_uart.o(.text.sci_uart_rxi_isr)
    [Anonymous Symbol]                       0x00003efc   Section        0  r_sci_uart.o(.text.sci_uart_tei_isr)
    [Anonymous Symbol]                       0x00003f46   Section        0  r_sci_uart.o(.text.sci_uart_txi_isr)
    [Anonymous Symbol]                       0x00003fd0   Section        0  shell.o(.text.shellBackspace)
    [Anonymous Symbol]                       0x00003fd6   Section        0  shell.o(.text.shellCheckPermission)
    [Anonymous Symbol]                       0x00004010   Section        0  shell.o(.text.shellClear)
    [Anonymous Symbol]                       0x00004044   Section        0  shell.o(.text.shellClearCommandLine)
    [Anonymous Symbol]                       0x00004090   Section        0  shell.o(.text.shellCmds)
    [Anonymous Symbol]                       0x000040b8   Section        0  shell_companion.o(.text.shellCompanionAdd)
    [Anonymous Symbol]                       0x000040c0   Section        0  shell_companion.o(.text.shellCompanionGet)
    [Anonymous Symbol]                       0x000040d8   Section        0  shell.o(.text.shellDelete)
    [Anonymous Symbol]                       0x000040e0   Section        0  shell.o(.text.shellDeleteByte)
    [Anonymous Symbol]                       0x000041d0   Section        0  shell.o(.text.shellDown)
    [Anonymous Symbol]                       0x000041d8   Section        0  shell.o(.text.shellEnter)
    [Anonymous Symbol]                       0x000041ec   Section        0  shell.o(.text.shellExec)
    shellExtParseChar                        0x00004349   Thumb Code    70  shell_ext.o(.text.shellExtParseChar)
    [Anonymous Symbol]                       0x00004348   Section        0  shell_ext.o(.text.shellExtParseChar)
    [Anonymous Symbol]                       0x00004390   Section        0  shell_ext.o(.text.shellExtParsePara)
    [Anonymous Symbol]                       0x00004554   Section        0  shell_ext.o(.text.shellExtRun)
    shellGetCommandName                      0x0000463d   Thumb Code    90  shell.o(.text.shellGetCommandName)
    [Anonymous Symbol]                       0x0000463c   Section        0  shell.o(.text.shellGetCommandName)
    [Anonymous Symbol]                       0x00004698   Section        0  shell.o(.text.shellGetCurrent)
    [Anonymous Symbol]                       0x000046c0   Section        0  shell.o(.text.shellGetVarValue)
    [Anonymous Symbol]                       0x000046fc   Section        0  shell.o(.text.shellHandler)
    [Anonymous Symbol]                       0x000047f4   Section        0  shell.o(.text.shellHelp)
    shellHistory                             0x000048e1   Thumb Code   218  shell.o(.text.shellHistory)
    [Anonymous Symbol]                       0x000048e0   Section        0  shell.o(.text.shellHistory)
    [Anonymous Symbol]                       0x000049bc   Section        0  shell.o(.text.shellInit)
    [Anonymous Symbol]                       0x00004a5c   Section        0  shell.o(.text.shellInsertByte)
    [Anonymous Symbol]                       0x00004b70   Section        0  shell.o(.text.shellKeys)
    [Anonymous Symbol]                       0x00004b98   Section        0  shell.o(.text.shellLeft)
    [Anonymous Symbol]                       0x00004bbc   Section        0  shell.o(.text.shellListCommand)
    [Anonymous Symbol]                       0x00004c1c   Section        0  shell.o(.text.shellListItem)
    [Anonymous Symbol]                       0x00004d74   Section        0  shell.o(.text.shellListKey)
    [Anonymous Symbol]                       0x00004dd0   Section        0  shell.o(.text.shellListUser)
    [Anonymous Symbol]                       0x00004e2c   Section        0  shell.o(.text.shellListVar)
    [Anonymous Symbol]                       0x00004e8c   Section        0  shell.o(.text.shellPrint)
    [Anonymous Symbol]                       0x00004ec6   Section        0  shell.o(.text.shellRight)
    [Anonymous Symbol]                       0x00004eec   Section        0  shell.o(.text.shellRunCommand)
    [Anonymous Symbol]                       0x00004fb4   Section        0  shell.o(.text.shellSeekCommand)
    [Anonymous Symbol]                       0x00005028   Section        0  shell.o(.text.shellSetUser)
    [Anonymous Symbol]                       0x000050a8   Section        0  shell.o(.text.shellSetVar)
    [Anonymous Symbol]                       0x00005154   Section        0  shell.o(.text.shellSetVarValue)
    shellShowVar                             0x00005215   Thumb Code   336  shell.o(.text.shellShowVar)
    [Anonymous Symbol]                       0x00005214   Section        0  shell.o(.text.shellShowVar)
    [Anonymous Symbol]                       0x00005368   Section        0  shell.o(.text.shellSplit)
    [Anonymous Symbol]                       0x00005458   Section        0  shell.o(.text.shellTab)
    [Anonymous Symbol]                       0x000055f4   Section        0  shell.o(.text.shellToDec)
    [Anonymous Symbol]                       0x0000565a   Section        0  shell.o(.text.shellUp)
    [Anonymous Symbol]                       0x00005660   Section        0  shell.o(.text.shellUsers)
    [Anonymous Symbol]                       0x00005688   Section        0  shell.o(.text.shellVars)
    [Anonymous Symbol]                       0x000056b0   Section        0  shell.o(.text.shellWriteEndLine)
    shellWritePrompt                         0x00005745   Thumb Code   160  shell.o(.text.shellWritePrompt)
    [Anonymous Symbol]                       0x00005744   Section        0  shell.o(.text.shellWritePrompt)
    shellWriteReturnValue                    0x00005809   Thumb Code   204  shell.o(.text.shellWriteReturnValue)
    [Anonymous Symbol]                       0x00005808   Section        0  shell.o(.text.shellWriteReturnValue)
    [Anonymous Symbol]                       0x000058e0   Section        0  r_sci_uart.o(.text.uart9_wait_for_tx)
    [Anonymous Symbol]                       0x000058f4   Section        0  shell_port_1.o(.text.uartLogWrite)
    [Anonymous Symbol]                       0x0000590e   Section        0  shell_port_1.o(.text.userShellInit)
    [Anonymous Symbol]                       0x00005946   Section        0  shell_port_1.o(.text.userShellWrite)
    [Anonymous Symbol]                       0x0000596a   Section        0  r_adc.o(.text.user_adc_callback)
    [Anonymous Symbol]                       0x00005978   Section        0  hal_entry.o(.text.user_timer0_callback)
    [Anonymous Symbol]                       0x000059aa   Section        0  hal_entry.o(.text.user_timer5_callback)
    [Anonymous Symbol]                       0x00005a6c   Section        0  r_sci_uart.o(.text.user_uart9_callback)
    i.__0snprintf                            0x00005aa8   Section        0  printfa.o(i.__0snprintf)
    i.__0sprintf                             0x00005adc   Section        0  printfa.o(i.__0sprintf)
    i.__0vsnprintf                           0x00005b04   Section        0  printfa.o(i.__0vsnprintf)
    _fp_digits                               0x00005b39   Thumb Code   366  printfa.o(i._fp_digits)
    i._fp_digits                             0x00005b38   Section        0  printfa.o(i._fp_digits)
    _printf_core                             0x00005cbd   Thumb Code  1744  printfa.o(i._printf_core)
    i._printf_core                           0x00005cbc   Section        0  printfa.o(i._printf_core)
    _printf_post_padding                     0x00006399   Thumb Code    36  printfa.o(i._printf_post_padding)
    i._printf_post_padding                   0x00006398   Section        0  printfa.o(i._printf_post_padding)
    _printf_pre_padding                      0x000063bd   Thumb Code    46  printfa.o(i._printf_pre_padding)
    i._printf_pre_padding                    0x000063bc   Section        0  printfa.o(i._printf_pre_padding)
    _snputc                                  0x000063eb   Thumb Code    22  printfa.o(i._snputc)
    i._snputc                                0x000063ea   Section        0  printfa.o(i._snputc)
    _sputc                                   0x00006401   Thumb Code    10  printfa.o(i._sputc)
    i._sputc                                 0x00006400   Section        0  printfa.o(i._sputc)
    i.fputc                                  0x0000640a   Section        0  fputc.o(i.fputc)
    i.puts                                   0x0000641c   Section        0  puts.o(i.puts)
    .constdata                               0x00006440   Section       64  ctype_c.o(.constdata)
    g_prcr_masks                             0x00006480   Data           8  bsp_register_protection.o(.rodata.cst8)
    [Anonymous Symbol]                       0x00006480   Section        0  bsp_register_protection.o(.rodata.cst8)
    __tagsym$$used.1                         0x000068c0   Number         0  bsp_security.o(.rodata.gp_start_of_nonsecure_callable_flash)
    __tagsym$$used.4                         0x000068c4   Number         0  bsp_security.o(.rodata.gp_start_of_nonsecure_callable_ram)
    __tagsym$$used.6                         0x000068c8   Number         0  bsp_security.o(.rodata.gp_start_of_nonsecure_data_flash)
    __tagsym$$used.0                         0x000068cc   Number         0  bsp_security.o(.rodata.gp_start_of_nonsecure_flash)
    __tagsym$$used.3                         0x000068d0   Number         0  bsp_security.o(.rodata.gp_start_of_nonsecure_ram)
    __tagsym$$used.7                         0x000068d4   Number         0  bsp_security.o(.rodata.gp_start_of_secure_data_flash)
    __tagsym$$used.2                         0x000068d8   Number         0  bsp_security.o(.rodata.gp_start_of_secure_flash)
    __tagsym$$used.5                         0x000068dc   Number         0  bsp_security.o(.rodata.gp_start_of_secure_ram)
    .L.str.23                                0x00006abc   Data          44  hal_entry.o(.rodata.str1.1)
    [Anonymous Symbol]                       0x00006abc   Section        0  hal_entry.o(.rodata.str1.1)
    .L.str.22                                0x00006b9d   Data          34  hal_entry.o(.rodata.str1.1)
    .L.str.24                                0x00006c46   Data          59  hal_entry.o(.rodata.str1.1)
    .L.str.12                                0x00006c81   Data          49  hal_entry.o(.rodata.str1.1)
    .L.str.14                                0x00006cb2   Data          51  hal_entry.o(.rodata.str1.1)
    .L.str.13                                0x00006ce5   Data          37  hal_entry.o(.rodata.str1.1)
    .L.str.15                                0x00006d0a   Data          39  hal_entry.o(.rodata.str1.1)
    .L.str.17                                0x00006d31   Data          43  hal_entry.o(.rodata.str1.1)
    .L.str.19                                0x00006d5c   Data          43  hal_entry.o(.rodata.str1.1)
    .L.str.16                                0x00006d87   Data          55  hal_entry.o(.rodata.str1.1)
    .L.str.21                                0x00006dbe   Data          39  hal_entry.o(.rodata.str1.1)
    .L.str.20                                0x00006de5   Data          35  hal_entry.o(.rodata.str1.1)
    .L.str.18                                0x00006e08   Data          55  hal_entry.o(.rodata.str1.1)
    .L.str.8                                 0x00006e3f   Data          16  hal_entry.o(.rodata.str1.1)
    .L.str.7                                 0x00006e4f   Data          19  hal_entry.o(.rodata.str1.1)
    .L__FUNCTION__.hal_entry                 0x00006e62   Data          10  hal_entry.o(.rodata.str1.1)
    .L.str.3                                 0x00006e6c   Data           4  shell.o(.rodata.str1.1)
    [Anonymous Symbol]                       0x00006e6c   Section        0  shell.o(.rodata.str1.1)
    .L.str.13                                0x00006e70   Data          20  shell.o(.rodata.str1.1)
    .L.str.8                                 0x00006e84   Data          33  shell.o(.rodata.str1.1)
    .L.str.7                                 0x00006ea5   Data         534  shell.o(.rodata.str1.1)
    .L.str.1                                 0x000070bb   Data           3  shell.o(.rodata.str1.1)
    .L.str.9                                 0x000070bc   Data           2  shell.o(.rodata.str1.1)
    .L.str.30                                0x000070be   Data           2  shell.o(.rodata.str1.1)
    .L.str.21                                0x000070c0   Data           9  shell.o(.rodata.str1.1)
    .L.str.31                                0x000070c9   Data           5  shell.o(.rodata.str1.1)
    .L.str.16                                0x000070ce   Data          21  shell_cmds.o(.rodata.str1.1)
    [Anonymous Symbol]                       0x000070ce   Section        0  shell_cmds.o(.rodata.str1.1)
    .L.str.17                                0x000070e3   Data          22  shell_cmds.o(.rodata.str1.1)
    .L.str.18                                0x000070f9   Data          31  shell_cmds.o(.rodata.str1.1)
    .L.str.27                                0x00007118   Data          24  shell_cmds.o(.rodata.str1.1)
    .L.str.15                                0x00007130   Data          43  shell_cmds.o(.rodata.str1.1)
    .L.str.29                                0x0000715b   Data          29  shell_cmds.o(.rodata.str1.1)
    .L.str.28                                0x00007178   Data          22  shell_cmds.o(.rodata.str1.1)
    .L.str.3                                 0x0000718e   Data          25  shell_cmds.o(.rodata.str1.1)
    .L.str.2                                 0x000071a4   Data           3  shell_cmds.o(.rodata.str1.1)
    .L.str.2                                 0x000071a7   Data           3  shell_cmds.o(.rodata.str1.1)
    .L.str                                   0x000071aa   Data          65  log.o(.rodata.str1.1)
    [Anonymous Symbol]                       0x000071aa   Section        0  log.o(.rodata.str1.1)
    .L.str.3                                 0x000071eb   Data          72  log.o(.rodata.str1.1)
    .L.str.1                                 0x00007233   Data          45  log.o(.rodata.str1.1)
    .L__const.shellWriteReturnValue.buffer   0x00007260   Data          12  shell.o(.rodata.str1.4)
    [Anonymous Symbol]                       0x00007260   Section        0  shell.o(.rodata.str1.4)
    __tagsym$$used.0                         0x0000726c   Number         0  bsp_common.o(.version)
    g_fsp_version                            0x0000726c   Data           4  bsp_common.o(.version)
    [Anonymous Symbol]                       0x0000726c   Section        0  bsp_common.o(.version)
    __tagsym$$used.1                         0x00007270   Number         0  bsp_common.o(.version)
    g_fsp_version_string                     0x00007270   Data           6  bsp_common.o(.version)
    [Anonymous Symbol]                       0x00007270   Section        0  bsp_common.o(.version)
    __tagsym$$used.2                         0x00007276   Number         0  bsp_common.o(.version)
    g_fsp_version_build_string               0x00007276   Data          68  bsp_common.o(.version)
    [Anonymous Symbol]                       0x00007276   Section        0  bsp_common.o(.version)
    __tagsym$$used.0                         0x000072ba   Number         0  hal_entry.o(shellCommand)
    __tagsym$$used.1                         0x000072ca   Number         0  hal_entry.o(shellCommand)
    __tagsym$$used.0                         0x000072da   Number         0  shell.o(shellCommand)
    __tagsym$$used.1                         0x000072ea   Number         0  shell.o(shellCommand)
    __tagsym$$used.2                         0x000072fa   Number         0  shell.o(shellCommand)
    __tagsym$$used.3                         0x0000730a   Number         0  shell.o(shellCommand)
    __tagsym$$used.4                         0x0000731a   Number         0  shell.o(shellCommand)
    __tagsym$$used.5                         0x0000732a   Number         0  shell.o(shellCommand)
    __tagsym$$used.6                         0x0000733a   Number         0  shell.o(shellCommand)
    __tagsym$$used.7                         0x0000734a   Number         0  shell.o(shellCommand)
    __tagsym$$used.8                         0x0000735a   Number         0  shell.o(shellCommand)
    __tagsym$$used.9                         0x0000736a   Number         0  shell.o(shellCommand)
    __tagsym$$used.10                        0x0000737a   Number         0  shell.o(shellCommand)
    __tagsym$$used.11                        0x0000738a   Number         0  shell.o(shellCommand)
    __tagsym$$used.12                        0x0000739a   Number         0  shell.o(shellCommand)
    __tagsym$$used.13                        0x000073aa   Number         0  shell.o(shellCommand)
    __tagsym$$used.14                        0x000073ba   Number         0  shell.o(shellCommand)
    __tagsym$$used.15                        0x000073ca   Number         0  shell.o(shellCommand)
    __tagsym$$used.16                        0x000073da   Number         0  shell.o(shellCommand)
    __tagsym$$used.17                        0x000073ea   Number         0  shell.o(shellCommand)
    __tagsym$$used.0                         0x000073fa   Number         0  shell_cmds.o(shellCommand)
    __tagsym$$used.1                         0x0000740a   Number         0  shell_cmds.o(shellCommand)
    __tagsym$$used.2                         0x0000741a   Number         0  shell_cmds.o(shellCommand)
    __tagsym$$used.3                         0x0000742a   Number         0  shell_cmds.o(shellCommand)
    __tagsym$$used.0                         0x0000743a   Number         0  log.o(shellCommand)
    __tagsym$$used.1                         0x0000744a   Number         0  log.o(shellCommand)
    __tagsym$$used.2                         0x0000745a   Number         0  log.o(shellCommand)
    __tagsym$$used.0                         0x0100a100   Number         0  bsp_rom_registers.o(.option_setting_ofs0)
    g_bsp_rom_ofs0                           0x0100a100   Data           4  bsp_rom_registers.o(.option_setting_ofs0)
    [Anonymous Symbol]                       0x0100a100   Section        0  bsp_rom_registers.o(.option_setting_ofs0)
    __tagsym$$used.1                         0x0100a134   Number         0  bsp_rom_registers.o(.option_setting_sas)
    g_bsp_rom_sas                            0x0100a134   Data           4  bsp_rom_registers.o(.option_setting_sas)
    [Anonymous Symbol]                       0x0100a134   Section        0  bsp_rom_registers.o(.option_setting_sas)
    __tagsym$$used.2                         0x0100a200   Number         0  bsp_rom_registers.o(.option_setting_ofs1_sec)
    g_bsp_rom_ofs1_sec                       0x0100a200   Data           4  bsp_rom_registers.o(.option_setting_ofs1_sec)
    [Anonymous Symbol]                       0x0100a200   Section        0  bsp_rom_registers.o(.option_setting_ofs1_sec)
    __tagsym$$used.3                         0x0100a210   Number         0  bsp_rom_registers.o(.option_setting_banksel_sec)
    g_bsp_rom_banksel_sec                    0x0100a210   Data           4  bsp_rom_registers.o(.option_setting_banksel_sec)
    [Anonymous Symbol]                       0x0100a210   Section        0  bsp_rom_registers.o(.option_setting_banksel_sec)
    __tagsym$$used.4                         0x0100a240   Number         0  bsp_rom_registers.o(.option_setting_bps_sec0)
    g_bsp_rom_bps_sec0                       0x0100a240   Data           4  bsp_rom_registers.o(.option_setting_bps_sec0)
    [Anonymous Symbol]                       0x0100a240   Section        0  bsp_rom_registers.o(.option_setting_bps_sec0)
    __tagsym$$used.5                         0x0100a244   Number         0  bsp_rom_registers.o(.option_setting_bps_sec1)
    g_bsp_rom_bps_sec1                       0x0100a244   Data           4  bsp_rom_registers.o(.option_setting_bps_sec1)
    [Anonymous Symbol]                       0x0100a244   Section        0  bsp_rom_registers.o(.option_setting_bps_sec1)
    __tagsym$$used.6                         0x0100a248   Number         0  bsp_rom_registers.o(.option_setting_bps_sec2)
    g_bsp_rom_bps_sec2                       0x0100a248   Data           4  bsp_rom_registers.o(.option_setting_bps_sec2)
    [Anonymous Symbol]                       0x0100a248   Section        0  bsp_rom_registers.o(.option_setting_bps_sec2)
    __tagsym$$used.7                         0x0100a24c   Number         0  bsp_rom_registers.o(.option_setting_bps_sec3)
    g_bsp_rom_bps_sec3                       0x0100a24c   Data           4  bsp_rom_registers.o(.option_setting_bps_sec3)
    [Anonymous Symbol]                       0x0100a24c   Section        0  bsp_rom_registers.o(.option_setting_bps_sec3)
    __tagsym$$used.8                         0x0100a260   Number         0  bsp_rom_registers.o(.option_setting_pbps_sec0)
    g_bsp_rom_pbps_sec0                      0x0100a260   Data           4  bsp_rom_registers.o(.option_setting_pbps_sec0)
    [Anonymous Symbol]                       0x0100a260   Section        0  bsp_rom_registers.o(.option_setting_pbps_sec0)
    __tagsym$$used.9                         0x0100a264   Number         0  bsp_rom_registers.o(.option_setting_pbps_sec1)
    g_bsp_rom_pbps_sec1                      0x0100a264   Data           4  bsp_rom_registers.o(.option_setting_pbps_sec1)
    [Anonymous Symbol]                       0x0100a264   Section        0  bsp_rom_registers.o(.option_setting_pbps_sec1)
    __tagsym$$used.10                        0x0100a268   Number         0  bsp_rom_registers.o(.option_setting_pbps_sec2)
    g_bsp_rom_pbps_sec2                      0x0100a268   Data           4  bsp_rom_registers.o(.option_setting_pbps_sec2)
    [Anonymous Symbol]                       0x0100a268   Section        0  bsp_rom_registers.o(.option_setting_pbps_sec2)
    __tagsym$$used.11                        0x0100a26c   Number         0  bsp_rom_registers.o(.option_setting_pbps_sec3)
    g_bsp_rom_pbps_sec3                      0x0100a26c   Data           4  bsp_rom_registers.o(.option_setting_pbps_sec3)
    [Anonymous Symbol]                       0x0100a26c   Section        0  bsp_rom_registers.o(.option_setting_pbps_sec3)
    __tagsym$$used.12                        0x0100a280   Number         0  bsp_rom_registers.o(.option_setting_ofs1_sel)
    g_bsp_rom_ofs1_sel                       0x0100a280   Data           4  bsp_rom_registers.o(.option_setting_ofs1_sel)
    [Anonymous Symbol]                       0x0100a280   Section        0  bsp_rom_registers.o(.option_setting_ofs1_sel)
    __tagsym$$used.13                        0x0100a2c0   Number         0  bsp_rom_registers.o(.option_setting_bps_sel0)
    g_bsp_rom_bps_sel0                       0x0100a2c0   Data           4  bsp_rom_registers.o(.option_setting_bps_sel0)
    [Anonymous Symbol]                       0x0100a2c0   Section        0  bsp_rom_registers.o(.option_setting_bps_sel0)
    __tagsym$$used.14                        0x0100a2c4   Number         0  bsp_rom_registers.o(.option_setting_bps_sel1)
    g_bsp_rom_bps_sel1                       0x0100a2c4   Data           4  bsp_rom_registers.o(.option_setting_bps_sel1)
    [Anonymous Symbol]                       0x0100a2c4   Section        0  bsp_rom_registers.o(.option_setting_bps_sel1)
    __tagsym$$used.15                        0x0100a2c8   Number         0  bsp_rom_registers.o(.option_setting_bps_sel2)
    g_bsp_rom_bps_sel2                       0x0100a2c8   Data           4  bsp_rom_registers.o(.option_setting_bps_sel2)
    [Anonymous Symbol]                       0x0100a2c8   Section        0  bsp_rom_registers.o(.option_setting_bps_sel2)
    __tagsym$$used.16                        0x0100a2cc   Number         0  bsp_rom_registers.o(.option_setting_bps_sel3)
    g_bsp_rom_bps_sel3                       0x0100a2cc   Data           4  bsp_rom_registers.o(.option_setting_bps_sel3)
    [Anonymous Symbol]                       0x0100a2cc   Section        0  bsp_rom_registers.o(.option_setting_bps_sel3)
    .data                                    0x20000000   Section        4  stdout.o(.data)
    user_timer0_callback.level_led3          0x2000001c   Data           4  hal_entry.o(.data.user_timer0_callback.level_led3)
    [Anonymous Symbol]                       0x2000001c   Section        0  hal_entry.o(.data.user_timer0_callback.level_led3)
    g_uart9_rx_complete                      0x200002e8   Data           1  r_sci_uart.o(.bss.g_uart9_rx_complete)
    [Anonymous Symbol]                       0x200002e8   Section        0  r_sci_uart.o(.bss.g_uart9_rx_complete)
    g_uart9_tx_complete                      0x200002e9   Data           1  r_sci_uart.o(.bss.g_uart9_tx_complete)
    [Anonymous Symbol]                       0x200002e9   Section        0  r_sci_uart.o(.bss.g_uart9_tx_complete)
    head_handle                              0x20000314   Data           4  multi_button.o(.bss.head_handle)
    [Anonymous Symbol]                       0x20000314   Section        0  multi_button.o(.bss.head_handle)
    logBuffer                                0x20000324   Data         256  log.o(.bss.logBuffer)
    [Anonymous Symbol]                       0x20000324   Section        0  log.o(.bss.logBuffer)
    shellGetCommandName.buffer               0x200005c0   Data           9  shell.o(.bss.shellGetCommandName.buffer)
    [Anonymous Symbol]                       0x200005c0   Section        0  shell.o(.bss.shellGetCommandName.buffer)
    shellList                                0x200005cc   Data          20  shell.o(.bss.shellList)
    [Anonymous Symbol]                       0x200005cc   Section        0  shell.o(.bss.shellList)
    shell_get_ts_ns.cyc                      0x200005e0   Data           4  shell_cmds.o(.bss.shell_get_ts_ns.cyc)
    [Anonymous Symbol]                       0x200005e0   Section        0  shell_cmds.o(.bss.shell_get_ts_ns.cyc)
    user_timer5_callback.a_time              0x200005e8   Data           4  hal_entry.o(.bss.user_timer5_callback.a_time)
    [Anonymous Symbol]                       0x200005e8   Section        0  hal_entry.o(.bss.user_timer5_callback.a_time)
    user_timer5_callback.one_period_flag     0x200005ec   Data           1  hal_entry.o(.bss.user_timer5_callback.one_period_flag)
    [Anonymous Symbol]                       0x200005ec   Section        0  hal_entry.o(.bss.user_timer5_callback.one_period_flag)
    user_timer5_callback.overflow_times      0x200005f0   Data           4  hal_entry.o(.bss.user_timer5_callback.overflow_times)
    [Anonymous Symbol]                       0x200005f0   Section        0  hal_entry.o(.bss.user_timer5_callback.overflow_times)
    __tagsym$$used.0                         0x200005f4   Number         0  bsp_clocks.o(.bss.noinit)
    g_clock_freq                             0x200005f4   Data          28  bsp_clocks.o(.bss.noinit)
    [Anonymous Symbol]                       0x200005f4   Section        0  bsp_clocks.o(.bss.noinit)
    __tagsym$$used.2                         0x20000610   Number         0  startup.o(.bss.heap)
    g_heap                                   0x20000610   Data        8192  startup.o(.bss.heap)
    [Anonymous Symbol]                       0x20000610   Section        0  startup.o(.bss.heap)
    __tagsym$$used.0                         0x20002610   Number         0  startup.o(.bss.stack)
    g_main_stack                             0x20002610   Data        1024  startup.o(.bss.stack)
    [Anonymous Symbol]                       0x20002610   Section        0  startup.o(.bss.stack)

    Global Symbols

    Symbol Name                              Value     Ov Type        Size  Object(Section)

    BuildAttributes$$THM_ISAv4$E$P$D$K$B$S$7EM$8M$VFPi5$EXTD16$VFPS$VFMA$PE$A:L22UL41UL21$X:L11$S22US41US21$IEEE1$IW$USESV6$~STKCKD$USESV7$WCHAR32$ENUMINT$~SHL$OSPACE$ROPI$MICROLIB$REQ8$PRES8$EABIv2 0x00000000   Number         0  anon$$obj.o ABSOLUTE
    Image$$__tz_FLASH_S$$Base                0x00000000   Number         0  anon$$obj.o ABSOLUTE
    __Vectors                                0x00000000   Data          64  startup.o(.fixed_vectors)
    _printf_a                                0x00000000   Number         0  printfstubs.o ABSOLUTE
    _printf_c                                0x00000000   Number         0  printfstubs.o ABSOLUTE
    _printf_charcount                        0x00000000   Number         0  printfstubs.o ABSOLUTE
    _printf_d                                0x00000000   Number         0  printfstubs.o ABSOLUTE
    _printf_e                                0x00000000   Number         0  printfstubs.o ABSOLUTE
    _printf_f                                0x00000000   Number         0  printfstubs.o ABSOLUTE
    _printf_flags                            0x00000000   Number         0  printfstubs.o ABSOLUTE
    _printf_fp_dec                           0x00000000   Number         0  printfstubs.o ABSOLUTE
    _printf_fp_hex                           0x00000000   Number         0  printfstubs.o ABSOLUTE
    _printf_g                                0x00000000   Number         0  printfstubs.o ABSOLUTE
    _printf_i                                0x00000000   Number         0  printfstubs.o ABSOLUTE
    _printf_int_dec                          0x00000000   Number         0  printfstubs.o ABSOLUTE
    _printf_l                                0x00000000   Number         0  printfstubs.o ABSOLUTE
    _printf_lc                               0x00000000   Number         0  printfstubs.o ABSOLUTE
    _printf_ll                               0x00000000   Number         0  printfstubs.o ABSOLUTE
    _printf_lld                              0x00000000   Number         0  printfstubs.o ABSOLUTE
    _printf_lli                              0x00000000   Number         0  printfstubs.o ABSOLUTE
    _printf_llo                              0x00000000   Number         0  printfstubs.o ABSOLUTE
    _printf_llu                              0x00000000   Number         0  printfstubs.o ABSOLUTE
    _printf_llx                              0x00000000   Number         0  printfstubs.o ABSOLUTE
    _printf_longlong_dec                     0x00000000   Number         0  printfstubs.o ABSOLUTE
    _printf_longlong_hex                     0x00000000   Number         0  printfstubs.o ABSOLUTE
    _printf_longlong_oct                     0x00000000   Number         0  printfstubs.o ABSOLUTE
    _printf_ls                               0x00000000   Number         0  printfstubs.o ABSOLUTE
    _printf_mbtowc                           0x00000000   Number         0  printfstubs.o ABSOLUTE
    _printf_n                                0x00000000   Number         0  printfstubs.o ABSOLUTE
    _printf_o                                0x00000000   Number         0  printfstubs.o ABSOLUTE
    _printf_p                                0x00000000   Number         0  printfstubs.o ABSOLUTE
    _printf_percent                          0x00000000   Number         0  printfstubs.o ABSOLUTE
    _printf_pre_padding                      0x00000000   Number         0  printfstubs.o ABSOLUTE
    _printf_return_value                     0x00000000   Number         0  printfstubs.o ABSOLUTE
    _printf_s                                0x00000000   Number         0  printfstubs.o ABSOLUTE
    _printf_sizespec                         0x00000000   Number         0  printfstubs.o ABSOLUTE
    _printf_str                              0x00000000   Number         0  printfstubs.o ABSOLUTE
    _printf_truncate_signed                  0x00000000   Number         0  printfstubs.o ABSOLUTE
    _printf_truncate_unsigned                0x00000000   Number         0  printfstubs.o ABSOLUTE
    _printf_u                                0x00000000   Number         0  printfstubs.o ABSOLUTE
    _printf_wc                               0x00000000   Number         0  printfstubs.o ABSOLUTE
    _printf_wctomb                           0x00000000   Number         0  printfstubs.o ABSOLUTE
    _printf_widthprec                        0x00000000   Number         0  printfstubs.o ABSOLUTE
    _printf_x                                0x00000000   Number         0  printfstubs.o ABSOLUTE
    _scanf_longlong                           - Undefined Weak Reference
    _scanf_real                               - Undefined Weak Reference
    _scanf_string                             - Undefined Weak Reference
    Image$$DATA$$Length                      0x00000020   Number         0  anon$$obj.o ABSOLUTE
    g_vector_table                           0x00000040   Data          36  vector_data.o(.application_vectors)
    Image$$INIT_ARRAY$$Base                  0x00000064   Number         0  anon$$obj.o ABSOLUTE
    Image$$INIT_ARRAY$$Limit                 0x00000064   Number         0  anon$$obj.o ABSOLUTE
    __aeabi_uldivmod                         0x00000065   Thumb Code    98  uldiv.o(.text)
    __aeabi_memcpy                           0x000000c7   Thumb Code    36  memcpya.o(.text)
    __aeabi_memcpy4                          0x000000c7   Thumb Code     0  memcpya.o(.text)
    __aeabi_memcpy8                          0x000000c7   Thumb Code     0  memcpya.o(.text)
    __aeabi_memset                           0x000000eb   Thumb Code    14  memseta.o(.text)
    __aeabi_memset4                          0x000000eb   Thumb Code     0  memseta.o(.text)
    __aeabi_memset8                          0x000000eb   Thumb Code     0  memseta.o(.text)
    __aeabi_memclr                           0x000000f9   Thumb Code     4  memseta.o(.text)
    __aeabi_memclr4                          0x000000f9   Thumb Code     0  memseta.o(.text)
    __aeabi_memclr8                          0x000000f9   Thumb Code     0  memseta.o(.text)
    _memset$wrapper                          0x000000fd   Thumb Code    18  memseta.o(.text)
    strlen                                   0x0000010f   Thumb Code    14  strlen.o(.text)
    strcmp                                   0x0000011d   Thumb Code    28  strcmp.o(.text)
    strncmp                                  0x00000139   Thumb Code    30  strncmp.o(.text)
    __0sscanf                                0x00000159   Thumb Code    48  __0sscanf.o(.text)
    _scanf_int                               0x00000191   Thumb Code   332  _scanf_int.o(.text)
    __aeabi_uidiv                            0x000002dd   Thumb Code     0  uidiv.o(.text)
    __aeabi_uidivmod                         0x000002dd   Thumb Code    44  uidiv.o(.text)
    __aeabi_llsl                             0x00000309   Thumb Code    30  llshl.o(.text)
    _ll_shift_l                              0x00000309   Thumb Code     0  llshl.o(.text)
    __aeabi_llsr                             0x00000327   Thumb Code    32  llushr.o(.text)
    _ll_ushift_r                             0x00000327   Thumb Code     0  llushr.o(.text)
    _chval                                   0x00000347   Thumb Code    28  _chval.o(.text)
    __vfscanf_char                           0x00000371   Thumb Code    20  scanf_char.o(.text)
    _sgetc                                   0x0000038d   Thumb Code    30  _sgetc.o(.text)
    _sbackspace                              0x000003ab   Thumb Code    34  _sgetc.o(.text)
    __I$use$fp                               0x000003cd   Thumb Code     0  iusefp.o(.text)
    __aeabi_dadd                             0x000003cd   Thumb Code   322  dadd.o(.text)
    __aeabi_dsub                             0x0000050f   Thumb Code     6  dadd.o(.text)
    __aeabi_drsub                            0x00000515   Thumb Code     6  dadd.o(.text)
    __aeabi_dmul                             0x0000051b   Thumb Code   228  dmul.o(.text)
    Image$$BSS$$ZI$$Length                   0x000005d4   Number         0  anon$$obj.o ABSOLUTE
    __aeabi_ddiv                             0x000005ff   Thumb Code   222  ddiv.o(.text)
    __aeabi_d2ulz                            0x000006dd   Thumb Code    48  dfixul.o(.text)
    __aeabi_cdrcmple                         0x0000070d   Thumb Code    48  cdrcmple.o(.text)
    __aeabi_lasr                             0x0000073d   Thumb Code    36  llsshr.o(.text)
    __semihosting_library_function           0x0000073d   Thumb Code     0  semi.o(.text)
    _ll_sshift_r                             0x0000073d   Thumb Code     0  llsshr.o(.text)
    isspace                                  0x00000761   Thumb Code    10  isspace_c.o(.text)
    __vfscanf                                0x0000076d   Thumb Code   808  _scanf.o(.text)
    __I$use$semihosting$fputc                0x00000a99   Thumb Code     0  iusesemip.o(.text)
    _double_round                            0x00000a99   Thumb Code    30  depilogue.o(.text)
    _double_epilogue                         0x00000ab7   Thumb Code   156  depilogue.o(.text)
    __ctype_lookup                           0x00000b55   Thumb Code    34  ctype_c.o(.text)
    Callback_btn_Handler                     0x00000b7d   Thumb Code    64  hal_entry.o(.text.Callback_btn_Handler)
    BusFault_Handler                         0x00000bf1   Thumb Code     4  startup.o(.text.Default_Handler)
    DebugMon_Handler                         0x00000bf1   Thumb Code     4  startup.o(.text.Default_Handler)
    Default_Handler                          0x00000bf1   Thumb Code     4  startup.o(.text.Default_Handler)
    HardFault_Handler                        0x00000bf1   Thumb Code     4  startup.o(.text.Default_Handler)
    MemManage_Handler                        0x00000bf1   Thumb Code     4  startup.o(.text.Default_Handler)
    PendSV_Handler                           0x00000bf1   Thumb Code     4  startup.o(.text.Default_Handler)
    SVC_Handler                              0x00000bf1   Thumb Code     4  startup.o(.text.Default_Handler)
    SecureFault_Handler                      0x00000bf1   Thumb Code     4  startup.o(.text.Default_Handler)
    UsageFault_Handler                       0x00000bf1   Thumb Code     4  startup.o(.text.Default_Handler)
    NMI_Handler                              0x00000bf5   Thumb Code    68  bsp_group_irq.o(.text.NMI_Handler)
    R_ADC_Calibrate                          0x00000c39   Thumb Code     4  r_adc.o(.text.R_ADC_Calibrate)
    R_ADC_CallbackSet                        0x00000c3d   Thumb Code    14  r_adc.o(.text.R_ADC_CallbackSet)
    R_ADC_Close                              0x00000c4b   Thumb Code   228  r_adc.o(.text.R_ADC_Close)
    R_ADC_InfoGet                            0x00000d31   Thumb Code   108  r_adc.o(.text.R_ADC_InfoGet)
    R_ADC_OffsetSet                          0x00000d9d   Thumb Code     4  r_adc.o(.text.R_ADC_OffsetSet)
    R_ADC_Open                               0x00000da1   Thumb Code   270  r_adc.o(.text.R_ADC_Open)
    R_ADC_Read                               0x00000eaf   Thumb Code    14  r_adc.o(.text.R_ADC_Read)
    R_ADC_Read32                             0x00000ebd   Thumb Code    24  r_adc.o(.text.R_ADC_Read32)
    R_ADC_ScanCfg                            0x00000ed5   Thumb Code   468  r_adc.o(.text.R_ADC_ScanCfg)
    R_ADC_ScanGroupStart                     0x000010a9   Thumb Code     4  r_adc.o(.text.R_ADC_ScanGroupStart)
    R_ADC_ScanStart                          0x000010ad   Thumb Code    10  r_adc.o(.text.R_ADC_ScanStart)
    R_ADC_ScanStop                           0x000010b7   Thumb Code    10  r_adc.o(.text.R_ADC_ScanStop)
    R_ADC_StatusGet                          0x000010c1   Thumb Code    12  r_adc.o(.text.R_ADC_StatusGet)
    R_BSP_Init_RTC                           0x000010cd   Thumb Code   122  bsp_clocks.o(.text.R_BSP_Init_RTC)
    R_BSP_RegisterProtectDisable             0x00001147   Thumb Code    78  bsp_register_protection.o(.text.R_BSP_RegisterProtectDisable)
    R_BSP_RegisterProtectEnable              0x00001195   Thumb Code    82  bsp_register_protection.o(.text.R_BSP_RegisterProtectEnable)
    R_BSP_SoftwareDelay                      0x000011e7   Thumb Code    72  bsp_delay.o(.text.R_BSP_SoftwareDelay)
    R_BSP_SourceClockHzGet                   0x0000122f   Thumb Code    14  bsp_clocks.o(.text.R_BSP_SourceClockHzGet)
    R_BSP_SubClockStabilizeWaitAfterReset    0x0000123d   Thumb Code     2  bsp_clocks.o(.text.R_BSP_SubClockStabilizeWaitAfterReset)
    R_BSP_WarmStart                          0x0000123f   Thumb Code    26  hal_entry.o(.text.R_BSP_WarmStart)
    R_DAC_Close                              0x00001259   Thumb Code    58  r_dac.o(.text.R_DAC_Close)
    R_DAC_Open                               0x00001293   Thumb Code   190  r_dac.o(.text.R_DAC_Open)
    R_DAC_Start                              0x00001351   Thumb Code   190  r_dac.o(.text.R_DAC_Start)
    R_DAC_Stop                               0x0000140f   Thumb Code    40  r_dac.o(.text.R_DAC_Stop)
    R_DAC_Write                              0x00001437   Thumb Code    12  r_dac.o(.text.R_DAC_Write)
    R_GPT_CallbackSet                        0x00001443   Thumb Code    14  r_gpt.o(.text.R_GPT_CallbackSet)
    R_GPT_Close                              0x00001451   Thumb Code   148  r_gpt.o(.text.R_GPT_Close)
    R_GPT_CompareMatchSet                    0x000014e5   Thumb Code    14  r_gpt.o(.text.R_GPT_CompareMatchSet)
    R_GPT_Disable                            0x000014f3   Thumb Code    30  r_gpt.o(.text.R_GPT_Disable)
    R_GPT_DutyCycleSet                       0x00001511   Thumb Code   172  r_gpt.o(.text.R_GPT_DutyCycleSet)
    R_GPT_Enable                             0x000015bd   Thumb Code    56  r_gpt.o(.text.R_GPT_Enable)
    R_GPT_InfoGet                            0x000015f5   Thumb Code    60  r_gpt.o(.text.R_GPT_InfoGet)
    R_GPT_Open                               0x00001631   Thumb Code   576  r_gpt.o(.text.R_GPT_Open)
    R_GPT_PeriodSet                          0x00001871   Thumb Code    56  r_gpt.o(.text.R_GPT_PeriodSet)
    R_GPT_Reset                              0x000018a9   Thumb Code    10  r_gpt.o(.text.R_GPT_Reset)
    R_GPT_Start                              0x000018b3   Thumb Code    10  r_gpt.o(.text.R_GPT_Start)
    R_GPT_StatusGet                          0x000018bd   Thumb Code    18  r_gpt.o(.text.R_GPT_StatusGet)
    R_GPT_Stop                               0x000018cf   Thumb Code    10  r_gpt.o(.text.R_GPT_Stop)
    R_IOPORT_Close                           0x000018d9   Thumb Code    10  r_ioport.o(.text.R_IOPORT_Close)
    R_IOPORT_Open                            0x000018e3   Thumb Code    22  r_ioport.o(.text.R_IOPORT_Open)
    R_IOPORT_PinCfg                          0x000018f9   Thumb Code   178  r_ioport.o(.text.R_IOPORT_PinCfg)
    R_IOPORT_PinEventInputRead               0x000019ab   Thumb Code    40  r_ioport.o(.text.R_IOPORT_PinEventInputRead)
    R_IOPORT_PinEventOutputWrite             0x000019d3   Thumb Code    82  r_ioport.o(.text.R_IOPORT_PinEventOutputWrite)
    R_IOPORT_PinRead                         0x00001a25   Thumb Code    34  r_ioport.o(.text.R_IOPORT_PinRead)
    R_IOPORT_PinWrite                        0x00001a47   Thumb Code    40  r_ioport.o(.text.R_IOPORT_PinWrite)
    R_IOPORT_PinsCfg                         0x00001a6f   Thumb Code    12  r_ioport.o(.text.R_IOPORT_PinsCfg)
    R_IOPORT_PortDirectionSet                0x00001a7b   Thumb Code    44  r_ioport.o(.text.R_IOPORT_PortDirectionSet)
    R_IOPORT_PortEventInputRead              0x00001aa7   Thumb Code    24  r_ioport.o(.text.R_IOPORT_PortEventInputRead)
    R_IOPORT_PortEventOutputWrite            0x00001abf   Thumb Code    32  r_ioport.o(.text.R_IOPORT_PortEventOutputWrite)
    R_IOPORT_PortRead                        0x00001adf   Thumb Code    22  r_ioport.o(.text.R_IOPORT_PortRead)
    R_IOPORT_PortWrite                       0x00001af5   Thumb Code    32  r_ioport.o(.text.R_IOPORT_PortWrite)
    R_SCI_UART_Abort                         0x00001b15   Thumb Code    34  r_sci_uart.o(.text.R_SCI_UART_Abort)
    R_SCI_UART_BaudSet                       0x00001b37   Thumb Code   104  r_sci_uart.o(.text.R_SCI_UART_BaudSet)
    R_SCI_UART_CallbackSet                   0x00001b9f   Thumb Code    14  r_sci_uart.o(.text.R_SCI_UART_CallbackSet)
    R_SCI_UART_Close                         0x00001bad   Thumb Code   166  r_sci_uart.o(.text.R_SCI_UART_Close)
    R_SCI_UART_InfoGet                       0x00001c53   Thumb Code    12  r_sci_uart.o(.text.R_SCI_UART_InfoGet)
    R_SCI_UART_Open                          0x00001c5f   Thumb Code   826  r_sci_uart.o(.text.R_SCI_UART_Open)
    R_SCI_UART_Read                          0x00001f99   Thumb Code    10  r_sci_uart.o(.text.R_SCI_UART_Read)
    R_SCI_UART_ReadStop                      0x00001fa3   Thumb Code    14  r_sci_uart.o(.text.R_SCI_UART_ReadStop)
    R_SCI_UART_Write                         0x00001fb1   Thumb Code    74  r_sci_uart.o(.text.R_SCI_UART_Write)
    Reset_Handler                            0x00001ffd   Thumb Code    10  startup.o(.text.Reset_Handler)
    SysTick_Handler                          0x00002007   Thumb Code    24  hal_entry.o(.text.SysTick_Handler)
    SystemCoreClockUpdate                    0x0000201f   Thumb Code    44  bsp_clocks.o(.text.SystemCoreClockUpdate)
    SystemInit                               0x0000204d   Thumb Code   240  system.o(.text.SystemInit)
    __aeabi_assert                           0x0000213d   Thumb Code     6  bsp_common.o(.text.__aeabi_assert)
    adc_scan_end_isr                         0x00002143   Thumb Code     6  r_adc.o(.text.adc_scan_end_isr)
    agencylogHexDump                         0x00002149   Thumb Code    32  log.o(.text.agencylogHexDump)
    agencylogSetLevel                        0x00002169   Thumb Code    88  log.o(.text.agencylogSetLevel)
    bsp_clock_init                           0x000021c1   Thumb Code   298  bsp_clocks.o(.text.bsp_clock_init)
    bsp_init                                 0x000022eb   Thumb Code     2  bsp_common.o(.text.bsp_init_internal)
    bsp_init_internal                        0x000022eb   Thumb Code     2  bsp_common.o(.text.bsp_init_internal)
    bsp_irq_cfg                              0x000022ed   Thumb Code   138  bsp_irq.o(.text.bsp_irq_cfg)
    bsp_prv_software_delay_loop              0x00002377   Thumb Code     8  bsp_delay.o(.text.bsp_prv_software_delay_loop)
    button_attach                            0x00002459   Thumb Code     8  multi_button.o(.text.button_attach)
    button_init                              0x00002461   Thumb Code    44  multi_button.o(.text.button_init)
    button_start                             0x0000248d   Thumb Code    40  multi_button.o(.text.button_start)
    button_ticks                             0x000024b5   Thumb Code   474  multi_button.o(.text.button_ticks)
    cmd_hex2dec                              0x00002691   Thumb Code    84  shell_cmds.o(.text.cmd_hex2dec)
    cmd_rd                                   0x00002721   Thumb Code   356  shell_cmds.o(.text.cmd_rd)
    cmd_time                                 0x00002929   Thumb Code   312  shell_cmds.o(.text.cmd_time)
    cmd_wr                                   0x00002ae5   Thumb Code   256  shell_cmds.o(.text.cmd_wr)
    get_adc_scan_status                      0x00002c75   Thumb Code    12  r_adc.o(.text.get_adc_scan_status)
    gpt_capture_compare_a_isr                0x00002cef   Thumb Code     6  r_gpt.o(.text.gpt_capture_compare_a_isr)
    gpt_capture_compare_b_isr                0x00002cf5   Thumb Code     6  r_gpt.o(.text.gpt_capture_compare_b_isr)
    gpt_counter_overflow_isr                 0x00002cfb   Thumb Code   172  r_gpt.o(.text.gpt_counter_overflow_isr)
    hal_entry                                0x00002da9   Thumb Code  2024  hal_entry.o(.text.hal_entry)
    logHexDump                               0x00003625   Thumb Code   308  log.o(.text.logHexDump)
    logRegister                              0x00003795   Thumb Code    54  log.o(.text.logRegister)
    logSwitchLevel                           0x000037cd   Thumb Code    48  log.o(.text.logSwitchLevel)
    logWrite                                 0x00003811   Thumb Code    60  log.o(.text.logWrite)
    lwrb_get_full                            0x000038ad   Thumb Code    30  lwrb.o(.text.lwrb_get_full)
    lwrb_init                                0x000038cb   Thumb Code    36  lwrb.o(.text.lwrb_init)
    lwrb_read                                0x000038ef   Thumb Code    34  lwrb.o(.text.lwrb_read)
    lwrb_read_ex                             0x00003911   Thumb Code   164  lwrb.o(.text.lwrb_read_ex)
    lwrb_write                               0x000039b5   Thumb Code    34  lwrb.o(.text.lwrb_write)
    lwrb_write_ex                            0x000039d7   Thumb Code   168  lwrb.o(.text.lwrb_write_ex)
    main                                     0x00003a7f   Thumb Code    10  main.o(.text.main)
    read_button_GPIO                         0x00003dc5   Thumb Code    44  hal_entry.o(.text.read_button_GPIO)
    reset_adc_scan_state                     0x00003dfd   Thumb Code    14  r_adc.o(.text.reset_adc_scan_state)
    sci_uart_eri_isr                         0x00003e0b   Thumb Code   106  r_sci_uart.o(.text.sci_uart_eri_isr)
    sci_uart_rxi_isr                         0x00003e75   Thumb Code   136  r_sci_uart.o(.text.sci_uart_rxi_isr)
    sci_uart_tei_isr                         0x00003efd   Thumb Code    74  r_sci_uart.o(.text.sci_uart_tei_isr)
    sci_uart_txi_isr                         0x00003f47   Thumb Code   138  r_sci_uart.o(.text.sci_uart_txi_isr)
    shellBackspace                           0x00003fd1   Thumb Code     6  shell.o(.text.shellBackspace)
    shellCheckPermission                     0x00003fd7   Thumb Code    56  shell.o(.text.shellCheckPermission)
    shellClear                               0x00004011   Thumb Code    52  shell.o(.text.shellClear)
    shellClearCommandLine                    0x00004045   Thumb Code    76  shell.o(.text.shellClearCommandLine)
    shellCmds                                0x00004091   Thumb Code    40  shell.o(.text.shellCmds)
    shellCompanionAdd                        0x000040b9   Thumb Code     6  shell_companion.o(.text.shellCompanionAdd)
    shellCompanionGet                        0x000040c1   Thumb Code    24  shell_companion.o(.text.shellCompanionGet)
    shellDelete                              0x000040d9   Thumb Code     8  shell.o(.text.shellDelete)
    shellDeleteByte                          0x000040e1   Thumb Code   240  shell.o(.text.shellDeleteByte)
    shellDown                                0x000041d1   Thumb Code     8  shell.o(.text.shellDown)
    shellEnter                               0x000041d9   Thumb Code    20  shell.o(.text.shellEnter)
    shellExec                                0x000041ed   Thumb Code   328  shell.o(.text.shellExec)
    shellExtParsePara                        0x00004391   Thumb Code   450  shell_ext.o(.text.shellExtParsePara)
    shellExtRun                              0x00004555   Thumb Code   230  shell_ext.o(.text.shellExtRun)
    shellGetCurrent                          0x00004699   Thumb Code    38  shell.o(.text.shellGetCurrent)
    shellGetVarValue                         0x000046c1   Thumb Code    60  shell.o(.text.shellGetVarValue)
    shellHandler                             0x000046fd   Thumb Code   248  shell.o(.text.shellHandler)
    shellHelp                                0x000047f5   Thumb Code   216  shell.o(.text.shellHelp)
    shellInit                                0x000049bd   Thumb Code   158  shell.o(.text.shellInit)
    shellInsertByte                          0x00004a5d   Thumb Code   274  shell.o(.text.shellInsertByte)
    shellKeys                                0x00004b71   Thumb Code    40  shell.o(.text.shellKeys)
    shellLeft                                0x00004b99   Thumb Code    36  shell.o(.text.shellLeft)
    shellListCommand                         0x00004bbd   Thumb Code    76  shell.o(.text.shellListCommand)
    shellListItem                            0x00004c1d   Thumb Code   300  shell.o(.text.shellListItem)
    shellListKey                             0x00004d75   Thumb Code    76  shell.o(.text.shellListKey)
    shellListUser                            0x00004dd1   Thumb Code    76  shell.o(.text.shellListUser)
    shellListVar                             0x00004e2d   Thumb Code    80  shell.o(.text.shellListVar)
    shellPrint                               0x00004e8d   Thumb Code    58  shell.o(.text.shellPrint)
    shellRight                               0x00004ec7   Thumb Code    38  shell.o(.text.shellRight)
    shellRunCommand                          0x00004eed   Thumb Code   200  shell.o(.text.shellRunCommand)
    shellSeekCommand                         0x00004fb5   Thumb Code   116  shell.o(.text.shellSeekCommand)
    shellSetUser                             0x00005029   Thumb Code   128  shell.o(.text.shellSetUser)
    shellSetVar                              0x000050a9   Thumb Code   140  shell.o(.text.shellSetVar)
    shellSetVarValue                         0x00005155   Thumb Code   144  shell.o(.text.shellSetVarValue)
    shellSplit                               0x00005369   Thumb Code   240  shell.o(.text.shellSplit)
    shellTab                                 0x00005459   Thumb Code   410  shell.o(.text.shellTab)
    shellToDec                               0x000055f5   Thumb Code   102  shell.o(.text.shellToDec)
    shellUp                                  0x0000565b   Thumb Code     6  shell.o(.text.shellUp)
    shellUsers                               0x00005661   Thumb Code    40  shell.o(.text.shellUsers)
    shellVars                                0x00005689   Thumb Code    40  shell.o(.text.shellVars)
    shellWriteEndLine                        0x000056b1   Thumb Code   140  shell.o(.text.shellWriteEndLine)
    uart9_wait_for_tx                        0x000058e1   Thumb Code    20  r_sci_uart.o(.text.uart9_wait_for_tx)
    uartLogWrite                             0x000058f5   Thumb Code    26  shell_port_1.o(.text.uartLogWrite)
    userShellInit                            0x0000590f   Thumb Code    56  shell_port_1.o(.text.userShellInit)
    userShellWrite                           0x00005947   Thumb Code    36  shell_port_1.o(.text.userShellWrite)
    user_adc_callback                        0x0000596b   Thumb Code    14  r_adc.o(.text.user_adc_callback)
    user_timer0_callback                     0x00005979   Thumb Code    50  hal_entry.o(.text.user_timer0_callback)
    user_timer5_callback                     0x000059ab   Thumb Code   194  hal_entry.o(.text.user_timer5_callback)
    user_uart9_callback                      0x00005a6d   Thumb Code    58  r_sci_uart.o(.text.user_uart9_callback)
    __0snprintf                              0x00005aa9   Thumb Code    48  printfa.o(i.__0snprintf)
    __1snprintf                              0x00005aa9   Thumb Code     0  printfa.o(i.__0snprintf)
    __2snprintf                              0x00005aa9   Thumb Code     0  printfa.o(i.__0snprintf)
    __c89snprintf                            0x00005aa9   Thumb Code     0  printfa.o(i.__0snprintf)
    snprintf                                 0x00005aa9   Thumb Code     0  printfa.o(i.__0snprintf)
    __0sprintf                               0x00005add   Thumb Code    34  printfa.o(i.__0sprintf)
    __1sprintf                               0x00005add   Thumb Code     0  printfa.o(i.__0sprintf)
    __2sprintf                               0x00005add   Thumb Code     0  printfa.o(i.__0sprintf)
    __c89sprintf                             0x00005add   Thumb Code     0  printfa.o(i.__0sprintf)
    sprintf                                  0x00005add   Thumb Code     0  printfa.o(i.__0sprintf)
    __0vsnprintf                             0x00005b05   Thumb Code    46  printfa.o(i.__0vsnprintf)
    __1vsnprintf                             0x00005b05   Thumb Code     0  printfa.o(i.__0vsnprintf)
    __2vsnprintf                             0x00005b05   Thumb Code     0  printfa.o(i.__0vsnprintf)
    __c89vsnprintf                           0x00005b05   Thumb Code     0  printfa.o(i.__0vsnprintf)
    vsnprintf                                0x00005b05   Thumb Code     0  printfa.o(i.__0vsnprintf)
    fputc                                    0x0000640b   Thumb Code    18  fputc.o(i.fputc)
    puts                                     0x0000641d   Thumb Code    30  puts.o(i.puts)
    __ctype_categories                       0x00006440   Data          64  ctype_c.o(.constdata)
    g_adc0                                   0x00006488   Data          16  hal_data.o(.rodata.g_adc0)
    g_adc0_cfg                               0x00006498   Data          48  hal_data.o(.rodata.g_adc0_cfg)
    g_adc0_cfg_extend                        0x000064c8   Data          40  hal_data.o(.rodata.g_adc0_cfg_extend)
    g_adc0_channel_cfg                       0x000064f0   Data          24  hal_data.o(.rodata.g_adc0_channel_cfg)
    g_adc_on_adc                             0x00006508   Data          52  r_adc.o(.rodata.g_adc_on_adc)
    g_bsp_pin_cfg                            0x0000653c   Data          12  pin_data.o(.rodata.g_bsp_pin_cfg)
    g_bsp_pin_cfg_data                       0x00006548   Data         128  pin_data.o(.rodata.g_bsp_pin_cfg_data)
    g_dac0                                   0x000065c8   Data          12  hal_data.o(.rodata.g_dac0)
    g_dac0_cfg                               0x000065d4   Data           8  hal_data.o(.rodata.g_dac0_cfg)
    g_dac0_ext_cfg                           0x000065dc   Data          12  hal_data.o(.rodata.g_dac0_ext_cfg)
    g_dac_on_dac                             0x000065e8   Data          20  r_dac.o(.rodata.g_dac_on_dac)
    g_interrupt_event_link_select            0x000065fc   Data          36  vector_data.o(.rodata.g_interrupt_event_link_select)
    g_ioport                                 0x00006620   Data          12  common_data.o(.rodata.g_ioport)
    g_ioport_on_ioport                       0x0000662c   Data          52  r_ioport.o(.rodata.g_ioport_on_ioport)
    g_timer0                                 0x00006660   Data          12  hal_data.o(.rodata.g_timer0)
    g_timer0_cfg                             0x0000666c   Data          36  hal_data.o(.rodata.g_timer0_cfg)
    g_timer0_extend                          0x00006690   Data          84  hal_data.o(.rodata.g_timer0_extend)
    g_timer2                                 0x000066e4   Data          12  hal_data.o(.rodata.g_timer2)
    g_timer2_cfg                             0x000066f0   Data          36  hal_data.o(.rodata.g_timer2_cfg)
    g_timer2_extend                          0x00006714   Data          84  hal_data.o(.rodata.g_timer2_extend)
    g_timer5                                 0x00006768   Data          12  hal_data.o(.rodata.g_timer5)
    g_timer5_cfg                             0x00006774   Data          36  hal_data.o(.rodata.g_timer5_cfg)
    g_timer5_extend                          0x00006798   Data          84  hal_data.o(.rodata.g_timer5_extend)
    g_timer_on_gpt                           0x000067ec   Data          52  r_gpt.o(.rodata.g_timer_on_gpt)
    g_uart9                                  0x00006820   Data          12  hal_data.o(.rodata.g_uart9)
    g_uart9_cfg                              0x0000682c   Data          68  hal_data.o(.rodata.g_uart9_cfg)
    g_uart9_cfg_extend                       0x00006870   Data          44  hal_data.o(.rodata.g_uart9_cfg_extend)
    g_uart_on_sci                            0x0000689c   Data          36  r_sci_uart.o(.rodata.g_uart_on_sci)
    gp_start_of_nonsecure_callable_flash     0x000068c0   Data           4  bsp_security.o(.rodata.gp_start_of_nonsecure_callable_flash)
    gp_start_of_nonsecure_callable_ram       0x000068c4   Data           4  bsp_security.o(.rodata.gp_start_of_nonsecure_callable_ram)
    gp_start_of_nonsecure_data_flash         0x000068c8   Data           4  bsp_security.o(.rodata.gp_start_of_nonsecure_data_flash)
    gp_start_of_nonsecure_flash              0x000068cc   Data           4  bsp_security.o(.rodata.gp_start_of_nonsecure_flash)
    gp_start_of_nonsecure_ram                0x000068d0   Data           4  bsp_security.o(.rodata.gp_start_of_nonsecure_ram)
    gp_start_of_secure_data_flash            0x000068d4   Data           4  bsp_security.o(.rodata.gp_start_of_secure_data_flash)
    gp_start_of_secure_flash                 0x000068d8   Data           4  bsp_security.o(.rodata.gp_start_of_secure_flash)
    gp_start_of_secure_ram                   0x000068dc   Data           4  bsp_security.o(.rodata.gp_start_of_secure_ram)
    shellCmdDefaultUser                      0x000068e0   Data          13  shell.o(.rodata.shellCmdDefaultUser)
    shellCmdclear                            0x000068ed   Data           6  shell.o(.rodata.shellCmdclear)
    shellCmdcmds                             0x000068f3   Data           5  shell.o(.rodata.shellCmdcmds)
    shellCmdgettemperature                   0x000068f8   Data          15  hal_entry.o(.rodata.shellCmdgettemperature)
    shellCmdhelp                             0x00006907   Data           5  shell.o(.rodata.shellCmdhelp)
    shellCmdhex2dec                          0x0000690c   Data           8  shell_cmds.o(.rodata.shellCmdhex2dec)
    shellCmdhexdump                          0x00006914   Data           8  log.o(.rodata.shellCmdhexdump)
    shellCmdkeys                             0x0000691c   Data           5  shell.o(.rodata.shellCmdkeys)
    shellCmdlogSetLevel                      0x00006921   Data          12  log.o(.rodata.shellCmdlogSetLevel)
    shellCmdrd                               0x0000692d   Data           3  shell_cmds.o(.rodata.shellCmdrd)
    shellCmdsetVar                           0x00006930   Data           7  shell.o(.rodata.shellCmdsetVar)
    shellCmdtimecal                          0x00006937   Data           8  shell_cmds.o(.rodata.shellCmdtimecal)
    shellCmdusers                            0x0000693f   Data           6  shell.o(.rodata.shellCmdusers)
    shellCmdvarPwm                           0x00006945   Data           7  hal_entry.o(.rodata.shellCmdvarPwm)
    shellCmdvars                             0x0000694c   Data           5  shell.o(.rodata.shellCmdvars)
    shellCmdwr                               0x00006951   Data           3  shell_cmds.o(.rodata.shellCmdwr)
    shellDesDefaultUser                      0x00006954   Data          13  shell.o(.rodata.shellDesDefaultUser)
    shellDesc0x04000000                      0x00006961   Data          17  log.o(.rodata.shellDesc0x04000000)
    shellDesc0x08000000                      0x00006972   Data          10  shell.o(.rodata.shellDesc0x08000000)
    shellDesc0x09000000                      0x0000697c   Data           4  shell.o(.rodata.shellDesc0x09000000)
    shellDesc0x0A000000                      0x00006980   Data           6  shell.o(.rodata.shellDesc0x0A000000)
    shellDesc0x0D000000                      0x00006986   Data           6  shell.o(.rodata.shellDesc0x0D000000)
    shellDesc0x1B5B337E                      0x0000698c   Data           7  shell.o(.rodata.shellDesc0x1B5B337E)
    shellDesc0x1B5B4100                      0x00006993   Data           3  shell.o(.rodata.shellDesc0x1B5B4100)
    shellDesc0x1B5B4200                      0x00006996   Data           5  shell.o(.rodata.shellDesc0x1B5B4200)
    shellDesc0x1B5B4300                      0x0000699b   Data           6  shell.o(.rodata.shellDesc0x1B5B4300)
    shellDesc0x1B5B4400                      0x000069a1   Data           5  shell.o(.rodata.shellDesc0x1B5B4400)
    shellDesc0x7F000000                      0x000069a6   Data          10  shell.o(.rodata.shellDesc0x7F000000)
    shellDescclear                           0x000069b0   Data          14  shell.o(.rodata.shellDescclear)
    shellDesccmds                            0x000069be   Data          13  shell.o(.rodata.shellDesccmds)
    shellDescgettemperature                  0x000069cb   Data           5  hal_entry.o(.rodata.shellDescgettemperature)
    shellDeschelp                            0x000069d0   Data          30  shell.o(.rodata.shellDeschelp)
    shellDeschex2dec                         0x000069ee   Data           5  shell_cmds.o(.rodata.shellDeschex2dec)
    shellDeschexdump                         0x000069f3   Data          32  log.o(.rodata.shellDeschexdump)
    shellDesckeys                            0x00006a13   Data          13  shell.o(.rodata.shellDesckeys)
    shellDesclogSetLevel                     0x00006a20   Data          36  log.o(.rodata.shellDesclogSetLevel)
    shellDescrd                              0x00006a44   Data           5  shell_cmds.o(.rodata.shellDescrd)
    shellDescsetVar                          0x00006a49   Data           8  shell.o(.rodata.shellDescsetVar)
    shellDesctimecal                         0x00006a51   Data           5  shell_cmds.o(.rodata.shellDesctimecal)
    shellDescusers                           0x00006a56   Data          14  shell.o(.rodata.shellDescusers)
    shellDescvarPwm                          0x00006a64   Data           5  hal_entry.o(.rodata.shellDescvarPwm)
    shellDescvars                            0x00006a69   Data          13  shell.o(.rodata.shellDescvars)
    shellDescwr                              0x00006a76   Data           5  shell_cmds.o(.rodata.shellDescwr)
    shellPasswordDefaultUser                 0x00006a7b   Data           1  shell.o(.rodata.shellPasswordDefaultUser)
    sindata                                  0x00006a7c   Data          64  hal_entry.o(.rodata.sindata)
    shellCommand$$Base                       0x000072ba   Number         0  hal_entry.o(shellCommand)
    shellVargettemperature                   0x000072ba   Data          16  hal_entry.o(shellCommand)
    shellVarvarPwm                           0x000072ca   Data          16  hal_entry.o(shellCommand)
    shellUserDefault                         0x000072da   Data          16  shell.o(shellCommand)
    shellCommandsetVar                       0x000072ea   Data          16  shell.o(shellCommand)
    shellKey0x1B5B4100                       0x000072fa   Data          16  shell.o(shellCommand)
    shellKey0x1B5B4200                       0x0000730a   Data          16  shell.o(shellCommand)
    shellKey0x1B5B4300                       0x0000731a   Data          16  shell.o(shellCommand)
    shellKey0x1B5B4400                       0x0000732a   Data          16  shell.o(shellCommand)
    shellKey0x09000000                       0x0000733a   Data          16  shell.o(shellCommand)
    shellKey0x08000000                       0x0000734a   Data          16  shell.o(shellCommand)
    shellKey0x7F000000                       0x0000735a   Data          16  shell.o(shellCommand)
    shellKey0x1B5B337E                       0x0000736a   Data          16  shell.o(shellCommand)
    shellKey0x0A000000                       0x0000737a   Data          16  shell.o(shellCommand)
    shellKey0x0D000000                       0x0000738a   Data          16  shell.o(shellCommand)
    shellCommandhelp                         0x0000739a   Data          16  shell.o(shellCommand)
    shellCommandusers                        0x000073aa   Data          16  shell.o(shellCommand)
    shellCommandcmds                         0x000073ba   Data          16  shell.o(shellCommand)
    shellCommandvars                         0x000073ca   Data          16  shell.o(shellCommand)
    shellCommandkeys                         0x000073da   Data          16  shell.o(shellCommand)
    shellCommandclear                        0x000073ea   Data          16  shell.o(shellCommand)
    shellCommandrd                           0x000073fa   Data          16  shell_cmds.o(shellCommand)
    shellCommandwr                           0x0000740a   Data          16  shell_cmds.o(shellCommand)
    shellCommandhex2dec                      0x0000741a   Data          16  shell_cmds.o(shellCommand)
    shellCommandtimecal                      0x0000742a   Data          16  shell_cmds.o(shellCommand)
    shellCommandlogSetLevel                  0x0000743a   Data          16  log.o(shellCommand)
    shellCommandhexdump                      0x0000744a   Data          16  log.o(shellCommand)
    shellKey0x04000000                       0x0000745a   Data          16  log.o(shellCommand)
    shellCommand$$Limit                      0x0000746a   Number         0  log.o(shellCommand)
    Load$$DATA$$Base                         0x0000746c   Number         0  anon$$obj.o ABSOLUTE
    Image$$__tz_FLASH_C$$Base                0x0000a000   Number         0  anon$$obj.o ABSOLUTE
    Image$$__tz_FLASH_N$$Base                0x00010000   Number         0  anon$$obj.o ABSOLUTE
    Image$$__tz_DATA_FLASH_N$$Base           0x08000000   Number         0  anon$$obj.o ABSOLUTE
    Image$$__tz_DATA_FLASH_S$$Base           0x08000000   Number         0  anon$$obj.o ABSOLUTE
    Image$$DATA$$Base                        0x20000000   Number         0  anon$$obj.o ABSOLUTE
    Image$$__tz_RAM_S$$Base                  0x20000000   Number         0  anon$$obj.o ABSOLUTE
    __stdout                                 0x20000000   Data           4  stdout.o(.data)
    g_uart9_baud_setting                     0x20000004   Data           4  hal_data.o(.data.g_uart9_baud_setting)
    gpt2_pwma_duty                           0x20000008   Data           1  hal_entry.o(.data.gpt2_pwma_duty)
    pairedChars                              0x20000009   Data           2  shell.o(.data.pairedChars)
    uartLog                                  0x2000000c   Data          16  shell_port_1.o(.data.uartLog)
    Image$$BSS$$ZI$$Base                     0x20000020   Number         0  anon$$obj.o ABSOLUTE
    SysTickms                                0x20000020   Data           8  hal_entry.o(.bss.SysTickms)
    SystemCoreClock                          0x20000028   Data           4  system.o(.bss.SystemCoreClock)
    adc_val                                  0x2000002c   Data          16  hal_entry.o(.bss.adc_val)
    btn                                      0x2000003c   Data         132  hal_entry.o(.bss.btn)
    buff                                     0x200000c0   Data          24  hal_entry.o(.bss.buff)
    buff_data                                0x200000d8   Data         256  hal_entry.o(.bss.buff_data)
    g_adc0_ctrl                              0x200001d8   Data          36  hal_data.o(.bss.g_adc0_ctrl)
    g_bsp_group_irq_sources                  0x200001fc   Data          56  bsp_group_irq.o(.bss.g_bsp_group_irq_sources)
    g_dac0_ctrl                              0x20000234   Data          16  hal_data.o(.bss.g_dac0_ctrl)
    g_ioport_ctrl                            0x20000244   Data           8  common_data.o(.bss.g_ioport_ctrl)
    g_protect_counters                       0x2000024c   Data           8  bsp_register_protection.o(.bss.g_protect_counters)
    g_protect_pfswe_counter                  0x20000254   Data           4  bsp_io.o(.bss.g_protect_pfswe_counter)
    g_timer0_ctrl                            0x20000258   Data          32  hal_data.o(.bss.g_timer0_ctrl)
    g_timer2_ctrl                            0x20000278   Data          32  hal_data.o(.bss.g_timer2_ctrl)
    g_timer5_ctrl                            0x20000298   Data          32  hal_data.o(.bss.g_timer5_ctrl)
    g_uart9_ctrl                             0x200002b8   Data          48  hal_data.o(.bss.g_uart9_ctrl)
    gi_temperature                           0x200002ec   Data           4  hal_entry.o(.bss.gi_temperature)
    gp_renesas_isr_context                   0x200002f0   Data          36  bsp_irq.o(.bss.gp_renesas_isr_context)
    info                                     0x20000318   Data          12  hal_entry.o(.bss.info)
    logList                                  0x20000424   Data          20  log.o(.bss.logList)
    period                                   0x20000438   Data           4  hal_entry.o(.bss.period)
    pwm_duty                                 0x2000043c   Data           4  hal_entry.o(.bss.pwm_duty)
    pwm_freq                                 0x20000440   Data           4  hal_entry.o(.bss.pwm_freq)
    pwm_high_level_time                      0x20000444   Data           4  hal_entry.o(.bss.pwm_high_level_time)
    pwm_period                               0x20000448   Data           4  hal_entry.o(.bss.pwm_period)
    scan_complete_flag                       0x2000044c   Data           1  r_adc.o(.bss.scan_complete_flag)
    shell                                    0x20000450   Data         112  shell_port_1.o(.bss.shell)
    shellBuffer                              0x200004c0   Data         256  shell_port_1.o(.bss.shellBuffer)
    temperature                              0x200005e4   Data           4  hal_entry.o(.bss.temperature)
    Image$$__tz_RAM_C$$Base                  0x20020000   Number         0  anon$$obj.o ABSOLUTE
    Image$$__tz_RAM_N$$Base                  0x20020000   Number         0  anon$$obj.o ABSOLUTE



==============================================================================

Memory Map of the image

  Image Entry point : 0x00001ffd

  Load Region LOAD_REGION_FLASH (Base: 0x00000000, Size: 0x00007490, Max: 0x00080000, ABSOLUTE)

    Execution Region __tz_FLASH_S (Exec base: 0x00000000, Load base: 0x00000000, Size: 0x00000000, Max: 0x00000000, ABSOLUTE)

    Exec Addr    Load Addr    Size         Type   Attr      Idx    E Section Name        Object

    0x00000000        -       0x00000000   Zero   RW            1    __tz_FLASH_S.bss    anon$$obj.o


    Execution Region VECTORS (Exec base: 0x00000000, Load base: 0x00000000, Size: 0x00000064, Max: 0xffffffff, ABSOLUTE, FIXED)

    Exec Addr    Load Addr    Size         Type   Attr      Idx    E Section Name        Object

    0x00000000   0x00000000   0x00000040   Data   RO          452    .fixed_vectors      startup.o
    0x00000040   0x00000040   0x00000024   Data   RO          765    .application_vectors  vector_data.o


    Execution Region MCUBOOT_SCE9_KEY (Exec base: 0x00000064, Load base: 0x00000064, Size: 0x00000000, Max: 0xffffffff, ABSOLUTE, FIXED)

    **** No section assigned to this execution region ****


    Execution Region INIT_ARRAY (Exec base: 0x00000064, Load base: 0x00000064, Size: 0x00000000, Max: 0xffffffff, ABSOLUTE, FIXED)

    **** No section assigned to this execution region ****


    Execution Region USB_DESC_FS (Exec base: 0x00000064, Load base: 0x00000064, Size: 0x00000000, Max: 0xffffffff, ABSOLUTE, FIXED)

    **** No section assigned to this execution region ****


    Execution Region RO_CODE_DATA (Exec base: 0x00000064, Load base: 0x00000064, Size: 0x00007408, Max: 0xffffffff, ABSOLUTE, FIXED)

    Exec Addr    Load Addr    Size         Type   Attr      Idx    E Section Name        Object

    0x00000064   0x00000064   0x00000062   Code   RO          911    .text               mc_w.l(uldiv.o)
    0x000000c6   0x000000c6   0x00000024   Code   RO          915    .text               mc_w.l(memcpya.o)
    0x000000ea   0x000000ea   0x00000024   Code   RO          917    .text               mc_w.l(memseta.o)
    0x0000010e   0x0000010e   0x0000000e   Code   RO          919    .text               mc_w.l(strlen.o)
    0x0000011c   0x0000011c   0x0000001c   Code   RO          921    .text               mc_w.l(strcmp.o)
    0x00000138   0x00000138   0x0000001e   Code   RO          923    .text               mc_w.l(strncmp.o)
    0x00000156   0x00000156   0x00000002   PAD
    0x00000158   0x00000158   0x00000038   Code   RO         1188    .text               mc_w.l(__0sscanf.o)
    0x00000190   0x00000190   0x0000014c   Code   RO         1190    .text               mc_w.l(_scanf_int.o)
    0x000002dc   0x000002dc   0x0000002c   Code   RO         1206    .text               mc_w.l(uidiv.o)
    0x00000308   0x00000308   0x0000001e   Code   RO         1208    .text               mc_w.l(llshl.o)
    0x00000326   0x00000326   0x00000020   Code   RO         1210    .text               mc_w.l(llushr.o)
    0x00000346   0x00000346   0x0000001c   Code   RO         1212    .text               mc_w.l(_chval.o)
    0x00000362   0x00000362   0x00000002   PAD
    0x00000364   0x00000364   0x00000028   Code   RO         1214    .text               mc_w.l(scanf_char.o)
    0x0000038c   0x0000038c   0x00000040   Code   RO         1216    .text               mc_w.l(_sgetc.o)
    0x000003cc   0x000003cc   0x00000000   Code   RO         1218    .text               mc_w.l(iusefp.o)
    0x000003cc   0x000003cc   0x0000014e   Code   RO         1219    .text               mf_w.l(dadd.o)
    0x0000051a   0x0000051a   0x000000e4   Code   RO         1221    .text               mf_w.l(dmul.o)
    0x000005fe   0x000005fe   0x000000de   Code   RO         1223    .text               mf_w.l(ddiv.o)
    0x000006dc   0x000006dc   0x00000030   Code   RO         1225    .text               mf_w.l(dfixul.o)
    0x0000070c   0x0000070c   0x00000030   Code   RO         1227    .text               mf_w.l(cdrcmple.o)
    0x0000073c   0x0000073c   0x00000000   Code   RO         1229    .text               mc_w.l(semi.o)
    0x0000073c   0x0000073c   0x00000024   Code   RO         1230    .text               mc_w.l(llsshr.o)
    0x00000760   0x00000760   0x0000000a   Code   RO         1232    .text               mc_w.l(isspace_c.o)
    0x0000076a   0x0000076a   0x00000002   PAD
    0x0000076c   0x0000076c   0x0000032c   Code   RO         1234    .text               mc_w.l(_scanf.o)
    0x00000a98   0x00000a98   0x00000000   Code   RO         1236    .text               mc_w.l(iusesemip.o)
    0x00000a98   0x00000a98   0x000000ba   Code   RO         1237    .text               mf_w.l(depilogue.o)
    0x00000b52   0x00000b52   0x00000002   PAD
    0x00000b54   0x00000b54   0x00000028   Code   RO         1239    .text               mc_w.l(ctype_c.o)
    0x00000b7c   0x00000b7c   0x00000074   Code   RO           48    .text.Callback_btn_Handler  hal_entry.o
    0x00000bf0   0x00000bf0   0x00000004   Code   RO          449    .text.Default_Handler  startup.o
    0x00000bf4   0x00000bf4   0x00000044   Code   RO          536    .text.NMI_Handler   bsp_group_irq.o
    0x00000c38   0x00000c38   0x00000004   Code   RO          788    .text.R_ADC_Calibrate  r_adc.o
    0x00000c3c   0x00000c3c   0x0000000e   Code   RO          792    .text.R_ADC_CallbackSet  r_adc.o
    0x00000c4a   0x00000c4a   0x000000e4   Code   RO          794    .text.R_ADC_Close   r_adc.o
    0x00000d2e   0x00000d2e   0x00000002   PAD
    0x00000d30   0x00000d30   0x0000006c   Code   RO          796    .text.R_ADC_InfoGet  r_adc.o
    0x00000d9c   0x00000d9c   0x00000004   Code   RO          790    .text.R_ADC_OffsetSet  r_adc.o
    0x00000da0   0x00000da0   0x0000010e   Code   RO          772    .text.R_ADC_Open    r_adc.o
    0x00000eae   0x00000eae   0x0000000e   Code   RO          784    .text.R_ADC_Read    r_adc.o
    0x00000ebc   0x00000ebc   0x00000018   Code   RO          786    .text.R_ADC_Read32  r_adc.o
    0x00000ed4   0x00000ed4   0x000001d4   Code   RO          774    .text.R_ADC_ScanCfg  r_adc.o
    0x000010a8   0x000010a8   0x00000004   Code   RO          778    .text.R_ADC_ScanGroupStart  r_adc.o
    0x000010ac   0x000010ac   0x0000000a   Code   RO          776    .text.R_ADC_ScanStart  r_adc.o
    0x000010b6   0x000010b6   0x0000000a   Code   RO          780    .text.R_ADC_ScanStop  r_adc.o
    0x000010c0   0x000010c0   0x0000000c   Code   RO          782    .text.R_ADC_StatusGet  r_adc.o
    0x000010cc   0x000010cc   0x0000007a   Code   RO          494    .text.R_BSP_Init_RTC  bsp_clocks.o
    0x00001146   0x00001146   0x0000004e   Code   RO          568    .text.R_BSP_RegisterProtectDisable  bsp_register_protection.o
    0x00001194   0x00001194   0x00000052   Code   RO          566    .text.R_BSP_RegisterProtectEnable  bsp_register_protection.o
    0x000011e6   0x000011e6   0x00000048   Code   RO          522    .text.R_BSP_SoftwareDelay  bsp_delay.o
    0x0000122e   0x0000122e   0x0000000e   Code   RO          492    .text.R_BSP_SourceClockHzGet  bsp_clocks.o
    0x0000123c   0x0000123c   0x00000002   Code   RO          488    .text.R_BSP_SubClockStabilizeWaitAfterReset  bsp_clocks.o
    0x0000123e   0x0000123e   0x0000001a   Code   RO           58    .text.R_BSP_WarmStart  hal_entry.o
    0x00001258   0x00001258   0x0000003a   Code   RO          830    .text.R_DAC_Close   r_dac.o
    0x00001292   0x00001292   0x000000be   Code   RO          828    .text.R_DAC_Open    r_dac.o
    0x00001350   0x00001350   0x000000be   Code   RO          834    .text.R_DAC_Start   r_dac.o
    0x0000140e   0x0000140e   0x00000028   Code   RO          836    .text.R_DAC_Stop    r_dac.o
    0x00001436   0x00001436   0x0000000c   Code   RO          832    .text.R_DAC_Write   r_dac.o
    0x00001442   0x00001442   0x0000000e   Code   RO          869    .text.R_GPT_CallbackSet  r_gpt.o
    0x00001450   0x00001450   0x00000094   Code   RO          871    .text.R_GPT_Close   r_gpt.o
    0x000014e4   0x000014e4   0x0000000e   Code   RO          863    .text.R_GPT_CompareMatchSet  r_gpt.o
    0x000014f2   0x000014f2   0x0000001e   Code   RO          857    .text.R_GPT_Disable  r_gpt.o
    0x00001510   0x00001510   0x000000ac   Code   RO          861    .text.R_GPT_DutyCycleSet  r_gpt.o
    0x000015bc   0x000015bc   0x00000038   Code   RO          855    .text.R_GPT_Enable  r_gpt.o
    0x000015f4   0x000015f4   0x0000003c   Code   RO          865    .text.R_GPT_InfoGet  r_gpt.o
    0x00001630   0x00001630   0x00000240   Code   RO          847    .text.R_GPT_Open    r_gpt.o
    0x00001870   0x00001870   0x00000038   Code   RO          859    .text.R_GPT_PeriodSet  r_gpt.o
    0x000018a8   0x000018a8   0x0000000a   Code   RO          853    .text.R_GPT_Reset   r_gpt.o
    0x000018b2   0x000018b2   0x0000000a   Code   RO          849    .text.R_GPT_Start   r_gpt.o
    0x000018bc   0x000018bc   0x00000012   Code   RO          867    .text.R_GPT_StatusGet  r_gpt.o
    0x000018ce   0x000018ce   0x0000000a   Code   RO          851    .text.R_GPT_Stop    r_gpt.o
    0x000018d8   0x000018d8   0x0000000a   Code   RO          619    .text.R_IOPORT_Close  r_ioport.o
    0x000018e2   0x000018e2   0x00000016   Code   RO          617    .text.R_IOPORT_Open  r_ioport.o
    0x000018f8   0x000018f8   0x000000b2   Code   RO          623    .text.R_IOPORT_PinCfg  r_ioport.o
    0x000019aa   0x000019aa   0x00000028   Code   RO          625    .text.R_IOPORT_PinEventInputRead  r_ioport.o
    0x000019d2   0x000019d2   0x00000052   Code   RO          627    .text.R_IOPORT_PinEventOutputWrite  r_ioport.o
    0x00001a24   0x00001a24   0x00000022   Code   RO          629    .text.R_IOPORT_PinRead  r_ioport.o
    0x00001a46   0x00001a46   0x00000028   Code   RO          631    .text.R_IOPORT_PinWrite  r_ioport.o
    0x00001a6e   0x00001a6e   0x0000000c   Code   RO          621    .text.R_IOPORT_PinsCfg  r_ioport.o
    0x00001a7a   0x00001a7a   0x0000002c   Code   RO          633    .text.R_IOPORT_PortDirectionSet  r_ioport.o
    0x00001aa6   0x00001aa6   0x00000018   Code   RO          635    .text.R_IOPORT_PortEventInputRead  r_ioport.o
    0x00001abe   0x00001abe   0x00000020   Code   RO          637    .text.R_IOPORT_PortEventOutputWrite  r_ioport.o
    0x00001ade   0x00001ade   0x00000016   Code   RO          639    .text.R_IOPORT_PortRead  r_ioport.o
    0x00001af4   0x00001af4   0x00000020   Code   RO          641    .text.R_IOPORT_PortWrite  r_ioport.o
    0x00001b14   0x00001b14   0x00000022   Code   RO          672    .text.R_SCI_UART_Abort  r_sci_uart.o
    0x00001b36   0x00001b36   0x00000068   Code   RO          668    .text.R_SCI_UART_BaudSet  r_sci_uart.o
    0x00001b9e   0x00001b9e   0x0000000e   Code   RO          674    .text.R_SCI_UART_CallbackSet  r_sci_uart.o
    0x00001bac   0x00001bac   0x000000a6   Code   RO          676    .text.R_SCI_UART_Close  r_sci_uart.o
    0x00001c52   0x00001c52   0x0000000c   Code   RO          670    .text.R_SCI_UART_InfoGet  r_sci_uart.o
    0x00001c5e   0x00001c5e   0x0000033a   Code   RO          662    .text.R_SCI_UART_Open  r_sci_uart.o
    0x00001f98   0x00001f98   0x0000000a   Code   RO          664    .text.R_SCI_UART_Read  r_sci_uart.o
    0x00001fa2   0x00001fa2   0x0000000e   Code   RO          678    .text.R_SCI_UART_ReadStop  r_sci_uart.o
    0x00001fb0   0x00001fb0   0x0000004a   Code   RO          666    .text.R_SCI_UART_Write  r_sci_uart.o
    0x00001ffa   0x00001ffa   0x00000002   PAD
    0x00001ffc   0x00001ffc   0x0000000a   Code   RO          447  * .text.Reset_Handler  startup.o
    0x00002006   0x00002006   0x00000018   Code   RO           44    .text.SysTick_Handler  hal_entry.o
    0x0000201e   0x0000201e   0x0000002c   Code   RO          478    .text.SystemCoreClockUpdate  bsp_clocks.o
    0x0000204a   0x0000204a   0x00000002   PAD
    0x0000204c   0x0000204c   0x000000f0   Code   RO          461    .text.SystemInit    system.o
    0x0000213c   0x0000213c   0x00000006   Code   RO          509    .text.__aeabi_assert  bsp_common.o
    0x00002142   0x00002142   0x00000006   Code   RO          802    .text.adc_scan_end_isr  r_adc.o
    0x00002148   0x00002148   0x00000020   Code   RO          352    .text.agencylogHexDump  log.o
    0x00002168   0x00002168   0x00000058   Code   RO          346    .text.agencylogSetLevel  log.o
    0x000021c0   0x000021c0   0x0000012a   Code   RO          484    .text.bsp_clock_init  bsp_clocks.o
    0x000022ea   0x000022ea   0x00000002   Code   RO          505    .text.bsp_init_internal  bsp_common.o
    0x000022ec   0x000022ec   0x0000008a   Code   RO          554    .text.bsp_irq_cfg   bsp_irq.o
    0x00002376   0x00002376   0x00000008   Code   RO          524    .text.bsp_prv_software_delay_loop  bsp_delay.o
    0x0000237e   0x0000237e   0x00000002   PAD
    0x00002380   0x00002380   0x000000d8   Code   RO          645    .text.bsp_vbatt_init  r_ioport.o
    0x00002458   0x00002458   0x00000008   Code   RO          428    .text.button_attach  multi_button.o
    0x00002460   0x00002460   0x0000002c   Code   RO          426    .text.button_init   multi_button.o
    0x0000248c   0x0000248c   0x00000028   Code   RO          432    .text.button_start  multi_button.o
    0x000024b4   0x000024b4   0x000001da   Code   RO          436    .text.button_ticks  multi_button.o
    0x0000268e   0x0000268e   0x00000002   PAD
    0x00002690   0x00002690   0x00000090   Code   RO          312    .text.cmd_hex2dec   shell_cmds.o
    0x00002720   0x00002720   0x00000208   Code   RO          308    .text.cmd_rd        shell_cmds.o
    0x00002928   0x00002928   0x000001bc   Code   RO          314    .text.cmd_time      shell_cmds.o
    0x00002ae4   0x00002ae4   0x00000190   Code   RO          310    .text.cmd_wr        shell_cmds.o
    0x00002c74   0x00002c74   0x0000000c   Code   RO          814    .text.get_adc_scan_status  r_adc.o
    0x00002c80   0x00002c80   0x0000006e   Code   RO          873    .text.gpt_calculate_duty_cycle  r_gpt.o
    0x00002cee   0x00002cee   0x00000006   Code   RO          889    .text.gpt_capture_compare_a_isr  r_gpt.o
    0x00002cf4   0x00002cf4   0x00000006   Code   RO          893    .text.gpt_capture_compare_b_isr  r_gpt.o
    0x00002cfa   0x00002cfa   0x000000ac   Code   RO          887    .text.gpt_counter_overflow_isr  r_gpt.o
    0x00002da6   0x00002da6   0x00000002   PAD
    0x00002da8   0x00002da8   0x0000087c   Code   RO           56    .text.hal_entry     hal_entry.o
    0x00003624   0x00003624   0x00000170   Code   RO          350    .text.logHexDump    log.o
    0x00003794   0x00003794   0x00000036   Code   RO          338    .text.logRegister   log.o
    0x000037ca   0x000037ca   0x00000002   PAD
    0x000037cc   0x000037cc   0x00000044   Code   RO          354    .text.logSwitchLevel  log.o
    0x00003810   0x00003810   0x0000003c   Code   RO          344    .text.logWrite      log.o
    0x0000384c   0x0000384c   0x00000060   Code   RO          348    .text.logWriteBuffer  log.o
    0x000038ac   0x000038ac   0x0000001e   Code   RO          397    .text.lwrb_get_full  lwrb.o
    0x000038ca   0x000038ca   0x00000024   Code   RO          375    .text.lwrb_init     lwrb.o
    0x000038ee   0x000038ee   0x00000022   Code   RO          393    .text.lwrb_read     lwrb.o
    0x00003910   0x00003910   0x000000a4   Code   RO          395    .text.lwrb_read_ex  lwrb.o
    0x000039b4   0x000039b4   0x00000022   Code   RO          387    .text.lwrb_write    lwrb.o
    0x000039d6   0x000039d6   0x000000a8   Code   RO          389    .text.lwrb_write_ex  lwrb.o
    0x00003a7e   0x00003a7e   0x0000000a   Code   RO          749    .text.main          main.o
    0x00003a88   0x00003a88   0x00000058   Code   RO          798    .text.r_adc_irq_enable  r_adc.o
    0x00003ae0   0x00003ae0   0x000000b0   Code   RO          804    .text.r_adc_scan_end_common_isr  r_adc.o
    0x00003b90   0x00003b90   0x000000d6   Code   RO          891    .text.r_gpt_ccmp_common_isr  r_gpt.o
    0x00003c66   0x00003c66   0x00000058   Code   RO          895    .text.r_gpt_enable_irq  r_gpt.o
    0x00003cbe   0x00003cbe   0x00000002   PAD
    0x00003cc0   0x00003cc0   0x000000c4   Code   RO          643    .text.r_ioport_pins_config  r_ioport.o
    0x00003d84   0x00003d84   0x00000040   Code   RO          684    .text.r_sci_uart_call_callback  r_sci_uart.o
    0x00003dc4   0x00003dc4   0x00000038   Code   RO           46    .text.read_button_GPIO  hal_entry.o
    0x00003dfc   0x00003dfc   0x0000000e   Code   RO          816    .text.reset_adc_scan_state  r_adc.o
    0x00003e0a   0x00003e0a   0x0000006a   Code   RO          690    .text.sci_uart_eri_isr  r_sci_uart.o
    0x00003e74   0x00003e74   0x00000088   Code   RO          686    .text.sci_uart_rxi_isr  r_sci_uart.o
    0x00003efc   0x00003efc   0x0000004a   Code   RO          688    .text.sci_uart_tei_isr  r_sci_uart.o
    0x00003f46   0x00003f46   0x0000008a   Code   RO          682    .text.sci_uart_txi_isr  r_sci_uart.o
    0x00003fd0   0x00003fd0   0x00000006   Code   RO          172    .text.shellBackspace  shell.o
    0x00003fd6   0x00003fd6   0x00000038   Code   RO          114    .text.shellCheckPermission  shell.o
    0x0000400e   0x0000400e   0x00000002   PAD
    0x00004010   0x00004010   0x00000034   Code   RO          194    .text.shellClear    shell.o
    0x00004044   0x00004044   0x0000004c   Code   RO          136    .text.shellClearCommandLine  shell.o
    0x00004090   0x00004090   0x00000028   Code   RO          188    .text.shellCmds     shell.o
    0x000040b8   0x000040b8   0x00000006   Code   RO          257    .text.shellCompanionAdd  shell_companion.o
    0x000040be   0x000040be   0x00000002   PAD
    0x000040c0   0x000040c0   0x00000018   Code   RO          261    .text.shellCompanionGet  shell_companion.o
    0x000040d8   0x000040d8   0x00000008   Code   RO          174    .text.shellDelete   shell.o
    0x000040e0   0x000040e0   0x000000f0   Code   RO          140    .text.shellDeleteByte  shell.o
    0x000041d0   0x000041d0   0x00000008   Code   RO          164    .text.shellDown     shell.o
    0x000041d8   0x000041d8   0x00000014   Code   RO          176    .text.shellEnter    shell.o
    0x000041ec   0x000041ec   0x0000015c   Code   RO          158    .text.shellExec     shell.o
    0x00004348   0x00004348   0x00000046   Code   RO          273    .text.shellExtParseChar  shell_ext.o
    0x0000438e   0x0000438e   0x00000002   PAD
    0x00004390   0x00004390   0x000001c2   Code   RO          271    .text.shellExtParsePara  shell_ext.o
    0x00004552   0x00004552   0x00000002   PAD
    0x00004554   0x00004554   0x000000e6   Code   RO          275    .text.shellExtRun   shell_ext.o
    0x0000463a   0x0000463a   0x00000002   PAD
    0x0000463c   0x0000463c   0x0000005a   Code   RO          122    .text.shellGetCommandName  shell.o
    0x00004696   0x00004696   0x00000002   PAD
    0x00004698   0x00004698   0x00000026   Code   RO          108    .text.shellGetCurrent  shell.o
    0x000046be   0x000046be   0x00000002   PAD
    0x000046c0   0x000046c0   0x0000003c   Code   RO          144    .text.shellGetVarValue  shell.o
    0x000046fc   0x000046fc   0x000000f8   Code   RO          180    .text.shellHandler  shell.o
    0x000047f4   0x000047f4   0x000000ec   Code   RO          178    .text.shellHelp     shell.o
    0x000048e0   0x000048e0   0x000000da   Code   RO          162    .text.shellHistory  shell.o
    0x000049ba   0x000049ba   0x00000002   PAD
    0x000049bc   0x000049bc   0x0000009e   Code   RO           98    .text.shellInit     shell.o
    0x00004a5a   0x00004a5a   0x00000002   PAD
    0x00004a5c   0x00004a5c   0x00000112   Code   RO          138    .text.shellInsertByte  shell.o
    0x00004b6e   0x00004b6e   0x00000002   PAD
    0x00004b70   0x00004b70   0x00000028   Code   RO          192    .text.shellKeys     shell.o
    0x00004b98   0x00004b98   0x00000024   Code   RO          168    .text.shellLeft     shell.o
    0x00004bbc   0x00004bbc   0x00000060   Code   RO          124    .text.shellListCommand  shell.o
    0x00004c1c   0x00004c1c   0x00000158   Code   RO          120    .text.shellListItem  shell.o
    0x00004d74   0x00004d74   0x0000005c   Code   RO          130    .text.shellListKey  shell.o
    0x00004dd0   0x00004dd0   0x0000005c   Code   RO          128    .text.shellListUser  shell.o
    0x00004e2c   0x00004e2c   0x00000060   Code   RO          126    .text.shellListVar  shell.o
    0x00004e8c   0x00004e8c   0x0000003a   Code   RO          112    .text.shellPrint    shell.o
    0x00004ec6   0x00004ec6   0x00000026   Code   RO          166    .text.shellRight    shell.o
    0x00004eec   0x00004eec   0x000000c8   Code   RO          152    .text.shellRunCommand  shell.o
    0x00004fb4   0x00004fb4   0x00000074   Code   RO          102    .text.shellSeekCommand  shell.o
    0x00005028   0x00005028   0x00000080   Code   RO          100    .text.shellSetUser  shell.o
    0x000050a8   0x000050a8   0x000000ac   Code   RO          150    .text.shellSetVar   shell.o
    0x00005154   0x00005154   0x000000c0   Code   RO          146    .text.shellSetVarValue  shell.o
    0x00005214   0x00005214   0x00000154   Code   RO          148    .text.shellShowVar  shell.o
    0x00005368   0x00005368   0x000000f0   Code   RO          142    .text.shellSplit    shell.o
    0x00005458   0x00005458   0x0000019a   Code   RO          170    .text.shellTab      shell.o
    0x000055f2   0x000055f2   0x00000002   PAD
    0x000055f4   0x000055f4   0x00000066   Code   RO          118    .text.shellToDec    shell.o
    0x0000565a   0x0000565a   0x00000006   Code   RO          160    .text.shellUp       shell.o
    0x00005660   0x00005660   0x00000028   Code   RO          186    .text.shellUsers    shell.o
    0x00005688   0x00005688   0x00000028   Code   RO          190    .text.shellVars     shell.o
    0x000056b0   0x000056b0   0x00000094   Code   RO          182    .text.shellWriteEndLine  shell.o
    0x00005744   0x00005744   0x000000c4   Code   RO          104    .text.shellWritePrompt  shell.o
    0x00005808   0x00005808   0x000000d8   Code   RO          154    .text.shellWriteReturnValue  shell.o
    0x000058e0   0x000058e0   0x00000014   Code   RO          658    .text.uart9_wait_for_tx  r_sci_uart.o
    0x000058f4   0x000058f4   0x0000001a   Code   RO          293    .text.uartLogWrite  shell_port_1.o
    0x0000590e   0x0000590e   0x00000038   Code   RO          295    .text.userShellInit  shell_port_1.o
    0x00005946   0x00005946   0x00000024   Code   RO          285    .text.userShellWrite  shell_port_1.o
    0x0000596a   0x0000596a   0x0000000e   Code   RO          810    .text.user_adc_callback  r_adc.o
    0x00005978   0x00005978   0x00000032   Code   RO           60    .text.user_timer0_callback  hal_entry.o
    0x000059aa   0x000059aa   0x000000c2   Code   RO           62    .text.user_timer5_callback  hal_entry.o
    0x00005a6c   0x00005a6c   0x0000003a   Code   RO          656    .text.user_uart9_callback  r_sci_uart.o
    0x00005aa6   0x00005aa6   0x00000002   PAD
    0x00005aa8   0x00005aa8   0x00000034   Code   RO         1161    i.__0snprintf       mc_w.l(printfa.o)
    0x00005adc   0x00005adc   0x00000028   Code   RO         1162    i.__0sprintf        mc_w.l(printfa.o)
    0x00005b04   0x00005b04   0x00000034   Code   RO         1165    i.__0vsnprintf      mc_w.l(printfa.o)
    0x00005b38   0x00005b38   0x00000184   Code   RO         1167    i._fp_digits        mc_w.l(printfa.o)
    0x00005cbc   0x00005cbc   0x000006dc   Code   RO         1168    i._printf_core      mc_w.l(printfa.o)
    0x00006398   0x00006398   0x00000024   Code   RO         1169    i._printf_post_padding  mc_w.l(printfa.o)
    0x000063bc   0x000063bc   0x0000002e   Code   RO         1170    i._printf_pre_padding  mc_w.l(printfa.o)
    0x000063ea   0x000063ea   0x00000016   Code   RO         1171    i._snputc           mc_w.l(printfa.o)
    0x00006400   0x00006400   0x0000000a   Code   RO         1172    i._sputc            mc_w.l(printfa.o)
    0x0000640a   0x0000640a   0x00000012   Code   RO         1192    i.fputc             mc_w.l(fputc.o)
    0x0000641c   0x0000641c   0x00000024   Code   RO          907    i.puts              mc_w.l(puts.o)
    0x00006440   0x00006440   0x00000040   Data   RO         1240    .constdata          mc_w.l(ctype_c.o)
    0x00006480   0x00006480   0x00000008   Data   RO          571    .rodata.cst8        bsp_register_protection.o
    0x00006488   0x00006488   0x00000010   Data   RO          737    .rodata.g_adc0      hal_data.o
    0x00006498   0x00006498   0x00000030   Data   RO          734    .rodata.g_adc0_cfg  hal_data.o
    0x000064c8   0x000064c8   0x00000028   Data   RO          733    .rodata.g_adc0_cfg_extend  hal_data.o
    0x000064f0   0x000064f0   0x00000018   Data   RO          735    .rodata.g_adc0_channel_cfg  hal_data.o
    0x00006508   0x00006508   0x00000034   Data   RO          818    .rodata.g_adc_on_adc  r_adc.o
    0x0000653c   0x0000653c   0x0000000c   Data   RO          759    .rodata.g_bsp_pin_cfg  pin_data.o
    0x00006548   0x00006548   0x00000080   Data   RO          758    .rodata.g_bsp_pin_cfg_data  pin_data.o
    0x000065c8   0x000065c8   0x0000000c   Data   RO          732    .rodata.g_dac0      hal_data.o
    0x000065d4   0x000065d4   0x00000008   Data   RO          730    .rodata.g_dac0_cfg  hal_data.o
    0x000065dc   0x000065dc   0x0000000c   Data   RO          729    .rodata.g_dac0_ext_cfg  hal_data.o
    0x000065e8   0x000065e8   0x00000014   Data   RO          838    .rodata.g_dac_on_dac  r_dac.o
    0x000065fc   0x000065fc   0x00000024   Data   RO          766    .rodata.g_interrupt_event_link_select  vector_data.o
    0x00006620   0x00006620   0x0000000c   Data   RO          708    .rodata.g_ioport    common_data.o
    0x0000662c   0x0000662c   0x00000034   Data   RO          647    .rodata.g_ioport_on_ioport  r_ioport.o
    0x00006660   0x00006660   0x0000000c   Data   RO          728    .rodata.g_timer0    hal_data.o
    0x0000666c   0x0000666c   0x00000024   Data   RO          726    .rodata.g_timer0_cfg  hal_data.o
    0x00006690   0x00006690   0x00000054   Data   RO          725    .rodata.g_timer0_extend  hal_data.o
    0x000066e4   0x000066e4   0x0000000c   Data   RO          724    .rodata.g_timer2    hal_data.o
    0x000066f0   0x000066f0   0x00000024   Data   RO          722    .rodata.g_timer2_cfg  hal_data.o
    0x00006714   0x00006714   0x00000054   Data   RO          721    .rodata.g_timer2_extend  hal_data.o
    0x00006768   0x00006768   0x0000000c   Data   RO          720    .rodata.g_timer5    hal_data.o
    0x00006774   0x00006774   0x00000024   Data   RO          718    .rodata.g_timer5_cfg  hal_data.o
    0x00006798   0x00006798   0x00000054   Data   RO          717    .rodata.g_timer5_extend  hal_data.o
    0x000067ec   0x000067ec   0x00000034   Data   RO          897    .rodata.g_timer_on_gpt  r_gpt.o
    0x00006820   0x00006820   0x0000000c   Data   RO          742    .rodata.g_uart9     hal_data.o
    0x0000682c   0x0000682c   0x00000044   Data   RO          740    .rodata.g_uart9_cfg  hal_data.o
    0x00006870   0x00006870   0x0000002c   Data   RO          739    .rodata.g_uart9_cfg_extend  hal_data.o
    0x0000689c   0x0000689c   0x00000024   Data   RO          694    .rodata.g_uart_on_sci  r_sci_uart.o
    0x000068c0   0x000068c0   0x00000004   Data   RO          605    .rodata.gp_start_of_nonsecure_callable_flash  bsp_security.o
    0x000068c4   0x000068c4   0x00000004   Data   RO          608    .rodata.gp_start_of_nonsecure_callable_ram  bsp_security.o
    0x000068c8   0x000068c8   0x00000004   Data   RO          610    .rodata.gp_start_of_nonsecure_data_flash  bsp_security.o
    0x000068cc   0x000068cc   0x00000004   Data   RO          604    .rodata.gp_start_of_nonsecure_flash  bsp_security.o
    0x000068d0   0x000068d0   0x00000004   Data   RO          607    .rodata.gp_start_of_nonsecure_ram  bsp_security.o
    0x000068d4   0x000068d4   0x00000004   Data   RO          611    .rodata.gp_start_of_secure_data_flash  bsp_security.o
    0x000068d8   0x000068d8   0x00000004   Data   RO          606    .rodata.gp_start_of_secure_flash  bsp_security.o
    0x000068dc   0x000068dc   0x00000004   Data   RO          609    .rodata.gp_start_of_secure_ram  bsp_security.o
    0x000068e0   0x000068e0   0x0000000d   Data   RO          198    .rodata.shellCmdDefaultUser  shell.o
    0x000068ed   0x000068ed   0x00000006   Data   RO          243    .rodata.shellCmdclear  shell.o
    0x000068f3   0x000068f3   0x00000005   Data   RO          234    .rodata.shellCmdcmds  shell.o
    0x000068f8   0x000068f8   0x0000000f   Data   RO           70    .rodata.shellCmdgettemperature  hal_entry.o
    0x00006907   0x00006907   0x00000005   Data   RO          228    .rodata.shellCmdhelp  shell.o
    0x0000690c   0x0000690c   0x00000008   Data   RO          323    .rodata.shellCmdhex2dec  shell_cmds.o
    0x00006914   0x00006914   0x00000008   Data   RO          362    .rodata.shellCmdhexdump  log.o
    0x0000691c   0x0000691c   0x00000005   Data   RO          240    .rodata.shellCmdkeys  shell.o
    0x00006921   0x00006921   0x0000000c   Data   RO          358    .rodata.shellCmdlogSetLevel  log.o
    0x0000692d   0x0000692d   0x00000003   Data   RO          317    .rodata.shellCmdrd  shell_cmds.o
    0x00006930   0x00006930   0x00000007   Data   RO          205    .rodata.shellCmdsetVar  shell.o
    0x00006937   0x00006937   0x00000008   Data   RO          326    .rodata.shellCmdtimecal  shell_cmds.o
    0x0000693f   0x0000693f   0x00000006   Data   RO          231    .rodata.shellCmdusers  shell.o
    0x00006945   0x00006945   0x00000007   Data   RO           74    .rodata.shellCmdvarPwm  hal_entry.o
    0x0000694c   0x0000694c   0x00000005   Data   RO          237    .rodata.shellCmdvars  shell.o
    0x00006951   0x00006951   0x00000003   Data   RO          320    .rodata.shellCmdwr  shell_cmds.o
    0x00006954   0x00006954   0x0000000d   Data   RO          200    .rodata.shellDesDefaultUser  shell.o
    0x00006961   0x00006961   0x00000011   Data   RO          365    .rodata.shellDesc0x04000000  log.o
    0x00006972   0x00006972   0x0000000a   Data   RO          218    .rodata.shellDesc0x08000000  shell.o
    0x0000697c   0x0000697c   0x00000004   Data   RO          216    .rodata.shellDesc0x09000000  shell.o
    0x00006980   0x00006980   0x00000006   Data   RO          224    .rodata.shellDesc0x0A000000  shell.o
    0x00006986   0x00006986   0x00000006   Data   RO          226    .rodata.shellDesc0x0D000000  shell.o
    0x0000698c   0x0000698c   0x00000007   Data   RO          222    .rodata.shellDesc0x1B5B337E  shell.o
    0x00006993   0x00006993   0x00000003   Data   RO          208    .rodata.shellDesc0x1B5B4100  shell.o
    0x00006996   0x00006996   0x00000005   Data   RO          210    .rodata.shellDesc0x1B5B4200  shell.o
    0x0000699b   0x0000699b   0x00000006   Data   RO          212    .rodata.shellDesc0x1B5B4300  shell.o
    0x000069a1   0x000069a1   0x00000005   Data   RO          214    .rodata.shellDesc0x1B5B4400  shell.o
    0x000069a6   0x000069a6   0x0000000a   Data   RO          220    .rodata.shellDesc0x7F000000  shell.o
    0x000069b0   0x000069b0   0x0000000e   Data   RO          244    .rodata.shellDescclear  shell.o
    0x000069be   0x000069be   0x0000000d   Data   RO          235    .rodata.shellDesccmds  shell.o
    0x000069cb   0x000069cb   0x00000005   Data   RO           71    .rodata.shellDescgettemperature  hal_entry.o
    0x000069d0   0x000069d0   0x0000001e   Data   RO          229    .rodata.shellDeschelp  shell.o
    0x000069ee   0x000069ee   0x00000005   Data   RO          324    .rodata.shellDeschex2dec  shell_cmds.o
    0x000069f3   0x000069f3   0x00000020   Data   RO          363    .rodata.shellDeschexdump  log.o
    0x00006a13   0x00006a13   0x0000000d   Data   RO          241    .rodata.shellDesckeys  shell.o
    0x00006a20   0x00006a20   0x00000024   Data   RO          359    .rodata.shellDesclogSetLevel  log.o
    0x00006a44   0x00006a44   0x00000005   Data   RO          318    .rodata.shellDescrd  shell_cmds.o
    0x00006a49   0x00006a49   0x00000008   Data   RO          206    .rodata.shellDescsetVar  shell.o
    0x00006a51   0x00006a51   0x00000005   Data   RO          327    .rodata.shellDesctimecal  shell_cmds.o
    0x00006a56   0x00006a56   0x0000000e   Data   RO          232    .rodata.shellDescusers  shell.o
    0x00006a64   0x00006a64   0x00000005   Data   RO           75    .rodata.shellDescvarPwm  hal_entry.o
    0x00006a69   0x00006a69   0x0000000d   Data   RO          238    .rodata.shellDescvars  shell.o
    0x00006a76   0x00006a76   0x00000005   Data   RO          321    .rodata.shellDescwr  shell_cmds.o
    0x00006a7b   0x00006a7b   0x00000001   Data   RO          199    .rodata.shellPasswordDefaultUser  shell.o
    0x00006a7c   0x00006a7c   0x00000040   Data   RO           64    .rodata.sindata     hal_entry.o
    0x00006abc   0x00006abc   0x000003b0   Data   RO           67    .rodata.str1.1      hal_entry.o
    0x00006e6c   0x00006e6c   0x00000262   Data   RO          204    .rodata.str1.1      shell.o
    0x000070ce   0x000070ce   0x000000dc   Data   RO          316    .rodata.str1.1      shell_cmds.o
    0x000071aa   0x000071aa   0x000000b6   Data   RO          357    .rodata.str1.1      log.o
    0x00007260   0x00007260   0x0000000c   Data   RO          247    .rodata.str1.4      shell.o
    0x0000726c   0x0000726c   0x00000004   Data   RO          511    .version            bsp_common.o
    0x00007270   0x00007270   0x00000006   Data   RO          512    .version            bsp_common.o
    0x00007276   0x00007276   0x00000044   Data   RO          513    .version            bsp_common.o
    0x000072ba   0x000072ba   0x00000010   Data   RO           72    shellCommand        hal_entry.o
    0x000072ca   0x000072ca   0x00000010   Data   RO           76    shellCommand        hal_entry.o
    0x000072da   0x000072da   0x00000010   Data   RO          201    shellCommand        shell.o
    0x000072ea   0x000072ea   0x00000010   Data   RO          207    shellCommand        shell.o
    0x000072fa   0x000072fa   0x00000010   Data   RO          209    shellCommand        shell.o
    0x0000730a   0x0000730a   0x00000010   Data   RO          211    shellCommand        shell.o
    0x0000731a   0x0000731a   0x00000010   Data   RO          213    shellCommand        shell.o
    0x0000732a   0x0000732a   0x00000010   Data   RO          215    shellCommand        shell.o
    0x0000733a   0x0000733a   0x00000010   Data   RO          217    shellCommand        shell.o
    0x0000734a   0x0000734a   0x00000010   Data   RO          219    shellCommand        shell.o
    0x0000735a   0x0000735a   0x00000010   Data   RO          221    shellCommand        shell.o
    0x0000736a   0x0000736a   0x00000010   Data   RO          223    shellCommand        shell.o
    0x0000737a   0x0000737a   0x00000010   Data   RO          225    shellCommand        shell.o
    0x0000738a   0x0000738a   0x00000010   Data   RO          227    shellCommand        shell.o
    0x0000739a   0x0000739a   0x00000010   Data   RO          230    shellCommand        shell.o
    0x000073aa   0x000073aa   0x00000010   Data   RO          233    shellCommand        shell.o
    0x000073ba   0x000073ba   0x00000010   Data   RO          236    shellCommand        shell.o
    0x000073ca   0x000073ca   0x00000010   Data   RO          239    shellCommand        shell.o
    0x000073da   0x000073da   0x00000010   Data   RO          242    shellCommand        shell.o
    0x000073ea   0x000073ea   0x00000010   Data   RO          245    shellCommand        shell.o
    0x000073fa   0x000073fa   0x00000010   Data   RO          319    shellCommand        shell_cmds.o
    0x0000740a   0x0000740a   0x00000010   Data   RO          322    shellCommand        shell_cmds.o
    0x0000741a   0x0000741a   0x00000010   Data   RO          325    shellCommand        shell_cmds.o
    0x0000742a   0x0000742a   0x00000010   Data   RO          328    shellCommand        shell_cmds.o
    0x0000743a   0x0000743a   0x00000010   Data   RO          360    shellCommand        log.o
    0x0000744a   0x0000744a   0x00000010   Data   RO          364    shellCommand        log.o
    0x0000745a   0x0000745a   0x00000010   Data   RO          366    shellCommand        log.o


    Execution Region __tz_RAM_S (Exec base: 0x20000000, Load base: 0x0000746c, Size: 0x00000000, Max: 0x00000000, ABSOLUTE)

    Exec Addr    Load Addr    Size         Type   Attr      Idx    E Section Name        Object

    0x20000000        -       0x00000000   Zero   RW            2    __tz_RAM_S.bss      anon$$obj.o


    Execution Region DTC_VECTOR_TABLE (Exec base: 0x20000000, Load base: 0x0000746c, Size: 0x00000000, Max: 0x00020000, ABSOLUTE, UNINIT)

    **** No section assigned to this execution region ****


    Execution Region DATA (Exec base: 0x20000000, Load base: 0x0000746c, Size: 0x00000020, Max: 0xffffffff, ABSOLUTE)

    Exec Addr    Load Addr    Size         Type   Attr      Idx    E Section Name        Object

    0x20000000   0x0000746c   0x00000004   Data   RW         1196    .data               mc_w.l(stdout.o)
    0x20000004   0x00007470   0x00000004   Data   RW          738    .data.g_uart9_baud_setting  hal_data.o
    0x20000008   0x00007474   0x00000001   Data   RW           73    .data.gpt2_pwma_duty  hal_entry.o
    0x20000009   0x00007475   0x00000002   Data   RW          202    .data.pairedChars   shell.o
    0x2000000b   0x00007477   0x00000001   PAD
    0x2000000c   0x00007478   0x00000010   Data   RW          297    .data.uartLog       shell_port_1.o
    0x2000001c   0x00007488   0x00000004   Data   RW           86    .data.user_timer0_callback.level_led3  hal_entry.o


    Execution Region BSS (Exec base: 0x20000020, Load base: 0x0000748c, Size: 0x000005d4, Max: 0xffffffff, ABSOLUTE)

    Exec Addr    Load Addr    Size         Type   Attr      Idx    E Section Name        Object

    0x20000020        -       0x00000008   Zero   RW           66    .bss.SysTickms      hal_entry.o
    0x20000028        -       0x00000004   Zero   RW          465    .bss.SystemCoreClock  system.o
    0x2000002c        -       0x00000010   Zero   RW           81    .bss.adc_val        hal_entry.o
    0x2000003c        -       0x00000084   Zero   RW           80    .bss.btn            hal_entry.o
    0x200000c0        -       0x00000018   Zero   RW           65    .bss.buff           hal_entry.o
    0x200000d8        -       0x00000100   Zero   RW           77    .bss.buff_data      hal_entry.o
    0x200001d8        -       0x00000024   Zero   RW          736    .bss.g_adc0_ctrl    hal_data.o
    0x200001fc        -       0x00000038   Zero   RW          538    .bss.g_bsp_group_irq_sources  bsp_group_irq.o
    0x20000234        -       0x00000010   Zero   RW          731    .bss.g_dac0_ctrl    hal_data.o
    0x20000244        -       0x00000008   Zero   RW          707    .bss.g_ioport_ctrl  common_data.o
    0x2000024c        -       0x00000008   Zero   RW          570    .bss.g_protect_counters  bsp_register_protection.o
    0x20000254        -       0x00000004   Zero   RW          548    .bss.g_protect_pfswe_counter  bsp_io.o
    0x20000258        -       0x00000020   Zero   RW          727    .bss.g_timer0_ctrl  hal_data.o
    0x20000278        -       0x00000020   Zero   RW          723    .bss.g_timer2_ctrl  hal_data.o
    0x20000298        -       0x00000020   Zero   RW          719    .bss.g_timer5_ctrl  hal_data.o
    0x200002b8        -       0x00000030   Zero   RW          741    .bss.g_uart9_ctrl   hal_data.o
    0x200002e8        -       0x00000001   Zero   RW          693    .bss.g_uart9_rx_complete  r_sci_uart.o
    0x200002e9        -       0x00000001   Zero   RW          692    .bss.g_uart9_tx_complete  r_sci_uart.o
    0x200002ea   0x0000748c   0x00000002   PAD
    0x200002ec        -       0x00000004   Zero   RW           69    .bss.gi_temperature  hal_entry.o
    0x200002f0        -       0x00000024   Zero   RW          557    .bss.gp_renesas_isr_context  bsp_irq.o
    0x20000314        -       0x00000004   Zero   RW          438    .bss.head_handle    multi_button.o
    0x20000318        -       0x0000000c   Zero   RW           78    .bss.info           hal_entry.o
    0x20000324        -       0x00000100   Zero   RW          361    .bss.logBuffer      log.o
    0x20000424        -       0x00000014   Zero   RW          356    .bss.logList        log.o
    0x20000438        -       0x00000004   Zero   RW           79    .bss.period         hal_entry.o
    0x2000043c        -       0x00000004   Zero   RW           85    .bss.pwm_duty       hal_entry.o
    0x20000440        -       0x00000004   Zero   RW           83    .bss.pwm_freq       hal_entry.o
    0x20000444        -       0x00000004   Zero   RW           84    .bss.pwm_high_level_time  hal_entry.o
    0x20000448        -       0x00000004   Zero   RW           82    .bss.pwm_period     hal_entry.o
    0x2000044c        -       0x00000001   Zero   RW          819    .bss.scan_complete_flag  r_adc.o
    0x2000044d   0x0000748c   0x00000003   PAD
    0x20000450        -       0x00000070   Zero   RW          298    .bss.shell          shell_port_1.o
    0x200004c0        -       0x00000100   Zero   RW          299    .bss.shellBuffer    shell_port_1.o
    0x200005c0        -       0x00000009   Zero   RW          246    .bss.shellGetCommandName.buffer  shell.o
    0x200005c9   0x0000748c   0x00000003   PAD
    0x200005cc        -       0x00000014   Zero   RW          203    .bss.shellList      shell.o
    0x200005e0        -       0x00000004   Zero   RW          329    .bss.shell_get_ts_ns.cyc  shell_cmds.o
    0x200005e4        -       0x00000004   Zero   RW           68    .bss.temperature    hal_entry.o
    0x200005e8        -       0x00000004   Zero   RW           87    .bss.user_timer5_callback.a_time  hal_entry.o
    0x200005ec        -       0x00000001   Zero   RW           89    .bss.user_timer5_callback.one_period_flag  hal_entry.o
    0x200005ed   0x0000748c   0x00000003   PAD
    0x200005f0        -       0x00000004   Zero   RW           88    .bss.user_timer5_callback.overflow_times  hal_entry.o


    Execution Region NOINIT (Exec base: 0x200005f4, Load base: 0x0000748c, Size: 0x0000001c, Max: 0xffffffff, ABSOLUTE, UNINIT)

    Exec Addr    Load Addr    Size         Type   Attr      Idx    E Section Name        Object

    0x200005f4        -       0x0000001c   Zero   RW          496    .bss.noinit         bsp_clocks.o


    Execution Region ARM_LIB_HEAP (Exec base: 0x20000610, Load base: 0x00007490, Size: 0x00002000, Max: 0xffffffff, ABSOLUTE, UNINIT)

    Exec Addr    Load Addr    Size         Type   Attr      Idx    E Section Name        Object

    0x20000610        -       0x00002000   Zero   RW          453    .bss.heap           startup.o


    Execution Region ARM_LIB_STACK (Exec base: 0x20002610, Load base: 0x00007490, Size: 0x00000000, Max: 0x00000000, ABSOLUTE, UNINIT)

    Exec Addr    Load Addr    Size         Type   Attr      Idx    E Section Name        Object

    0x20002610        -       0x00000000   Zero   RW            3    ARM_LIB_STACK.bss   anon$$obj.o


    Execution Region STACK (Exec base: 0x20002610, Load base: 0x00007490, Size: 0x00000400, Max: 0xffffffff, ABSOLUTE, UNINIT)

    Exec Addr    Load Addr    Size         Type   Attr      Idx    E Section Name        Object

    0x20002610        -       0x00000400   Zero   RW          451    .bss.stack          startup.o


    Execution Region RAM_END (Exec base: 0x20002a10, Load base: 0x00007490, Size: 0x00000004, Max: 0x00000004, ABSOLUTE)

    Exec Addr    Load Addr    Size         Type   Attr      Idx    E Section Name        Object

    0x20002a10        -       0x00000004   Zero   RW            4    RAM_END.bss         anon$$obj.o


    Execution Region __tz_RAM_C (Exec base: 0x20020000, Load base: 0x00007490, Size: 0x00000000, Max: 0x00000000, ABSOLUTE)

    Exec Addr    Load Addr    Size         Type   Attr      Idx    E Section Name        Object

    0x20020000        -       0x00000000   Zero   RW            5    __tz_RAM_C.bss      anon$$obj.o


    Execution Region __tz_RAM_N (Exec base: 0x20020000, Load base: 0x00007490, Size: 0x00000000, Max: 0x00000000, ABSOLUTE)

    Exec Addr    Load Addr    Size         Type   Attr      Idx    E Section Name        Object

    0x20020000        -       0x00000000   Zero   RW            6    __tz_RAM_N.bss      anon$$obj.o


    Execution Region RAM_LIMIT (Exec base: 0x20020000, Load base: 0x00007490, Size: 0x00000004, Max: 0x00000004, ABSOLUTE)

    Exec Addr    Load Addr    Size         Type   Attr      Idx    E Section Name        Object

    0x20020000        -       0x00000004   Zero   RW            7    RAM_LIMIT.bss       anon$$obj.o


    Execution Region OSPI_DEVICE_0_NO_LOAD (Exec base: 0x80020000, Load base: 0x00007490, Size: 0x00000000, Max: 0xffffffff, ABSOLUTE, UNINIT)

    **** No section assigned to this execution region ****


    Execution Region OSPI_DEVICE_1_NO_LOAD (Exec base: 0x80030000, Load base: 0x00007490, Size: 0x00000000, Max: 0xffffffff, ABSOLUTE, UNINIT)

    **** No section assigned to this execution region ****



  Load Region LOAD_REGION_NSC_FLASH (Base: 0x0000a000, Size: 0x00000000, Max: 0xffffffff, ABSOLUTE)

    Execution Region __tz_FLASH_C (Exec base: 0x0000a000, Load base: 0x0000a000, Size: 0x00000000, Max: 0x00000000, ABSOLUTE)

    Exec Addr    Load Addr    Size         Type   Attr      Idx    E Section Name        Object

    0x0000a000        -       0x00000000   Zero   RW            8    __tz_FLASH_C.bss    anon$$obj.o


    Execution Region EXEC_NSCR (Exec base: 0x0000a000, Load base: 0x0000a000, Size: 0x00000000, Max: 0xffffffff, ABSOLUTE, FIXED)

    **** No section assigned to this execution region ****


    Execution Region __tz_FLASH_N (Exec base: 0x00010000, Load base: 0x0000a000, Size: 0x00000000, Max: 0x00000000, ABSOLUTE)

    Exec Addr    Load Addr    Size         Type   Attr      Idx    E Section Name        Object

    0x00010000        -       0x00000000   Zero   RW            9    __tz_FLASH_N.bss    anon$$obj.o



  Load Region LOAD_REGION_ID_CODE (Base: 0x00000000, Size: 0x00000000, Max: 0x00000004, ABSOLUTE)

    Execution Region __tz_ID_CODE_S (Exec base: 0x00000000, Load base: 0x00000000, Size: 0x00000000, Max: 0x00000000, ABSOLUTE)

    Exec Addr    Load Addr    Size         Type   Attr      Idx    E Section Name        Object

    0x00000000        -       0x00000000   Zero   RW           10    __tz_ID_CODE_S.bss  anon$$obj.o


    Execution Region __tz_ID_CODE_N (Exec base: 0x00000000, Load base: 0x00000000, Size: 0x00000000, Max: 0x00000000, ABSOLUTE)

    Exec Addr    Load Addr    Size         Type   Attr      Idx    E Section Name        Object

    0x00000000        -       0x00000000   Zero   RW           11    __tz_ID_CODE_N.bss  anon$$obj.o



  Load Region LOAD_REGION_OPTION_SETTING (Base: 0x0100a100, Size: 0x00000080, Max: 0x00000100, ABSOLUTE)

    Execution Region __tz_OPTION_SETTING_S (Exec base: 0x0100a100, Load base: 0x0100a100, Size: 0x00000000, Max: 0x00000000, ABSOLUTE)

    Exec Addr    Load Addr    Size         Type   Attr      Idx    E Section Name        Object

    0x0100a100        -       0x00000000   Zero   RW           12    __tz_OPTION_SETTING_S.bss  anon$$obj.o


    Execution Region OFS0 (Exec base: 0x0100a100, Load base: 0x0100a100, Size: 0x00000004, Max: 0xffffffff, ABSOLUTE, FIXED)

    Exec Addr    Load Addr    Size         Type   Attr      Idx    E Section Name        Object

    0x0100a100   0x0100a100   0x00000004   Data   RO          580    .option_setting_ofs0  bsp_rom_registers.o


    Execution Region UNUSED_0 (Exec base: 0x0100a104, Load base: 0x0100a104, Size: 0x00000000, Max: 0x00000000, ABSOLUTE, FIXED)

    Exec Addr    Load Addr    Size         Type   Attr      Idx    E Section Name        Object

    0x0100a104        -       0x00000000   Zero   RW           13    UNUSED_0.bss        anon$$obj.o


    Execution Region OFS2 (Exec base: 0x0100a104, Load base: 0x0100a104, Size: 0x00000000, Max: 0xffffffff, ABSOLUTE, FIXED)

    **** No section assigned to this execution region ****


    Execution Region UNUSED_1 (Exec base: 0x0100a104, Load base: 0x0100a104, Size: 0x0000000c, Max: 0x0000000c, ABSOLUTE, FIXED)

    Exec Addr    Load Addr    Size         Type   Attr      Idx    E Section Name        Object

    0x0100a104        -       0x0000000c   Zero   RW           14    UNUSED_1.bss        anon$$obj.o


    Execution Region DUALSEL (Exec base: 0x0100a110, Load base: 0x0100a110, Size: 0x00000000, Max: 0xffffffff, ABSOLUTE, FIXED)

    **** No section assigned to this execution region ****


    Execution Region UNUSED_2 (Exec base: 0x0100a110, Load base: 0x0100a110, Size: 0x00000024, Max: 0x00000024, ABSOLUTE, FIXED)

    Exec Addr    Load Addr    Size         Type   Attr      Idx    E Section Name        Object

    0x0100a110        -       0x00000024   Zero   RW           15    UNUSED_2.bss        anon$$obj.o


    Execution Region SAS (Exec base: 0x0100a134, Load base: 0x0100a134, Size: 0x00000004, Max: 0xffffffff, ABSOLUTE, FIXED)

    Exec Addr    Load Addr    Size         Type   Attr      Idx    E Section Name        Object

    0x0100a134   0x0100a134   0x00000004   Data   RO          581    .option_setting_sas  bsp_rom_registers.o


    Execution Region UNUSED_3 (Exec base: 0x0100a138, Load base: 0x0100a138, Size: 0x00000048, Max: 0x00000048, ABSOLUTE, FIXED)

    Exec Addr    Load Addr    Size         Type   Attr      Idx    E Section Name        Object

    0x0100a138        -       0x00000048   Zero   RW           16    UNUSED_3.bss        anon$$obj.o


    Execution Region __tz_OPTION_SETTING_N (Exec base: 0x0100a180, Load base: 0x0100a180, Size: 0x00000000, Max: 0x00000000, ABSOLUTE)

    Exec Addr    Load Addr    Size         Type   Attr      Idx    E Section Name        Object

    0x0100a180        -       0x00000000   Zero   RW           17    __tz_OPTION_SETTING_N.bss  anon$$obj.o



  Load Region LOAD_REGION_OPTION_SETTING_S (Base: 0x0100a200, Size: 0x00000100, Max: 0x00000100, ABSOLUTE)

    Execution Region __tz_OPTION_SETTING_S_S (Exec base: 0x0100a200, Load base: 0x0100a200, Size: 0x00000000, Max: 0x00000000, ABSOLUTE)

    Exec Addr    Load Addr    Size         Type   Attr      Idx    E Section Name        Object

    0x0100a200        -       0x00000000   Zero   RW           18    __tz_OPTION_SETTING_S_S.bss  anon$$obj.o


    Execution Region OFS1_SEC (Exec base: 0x0100a200, Load base: 0x0100a200, Size: 0x00000004, Max: 0xffffffff, ABSOLUTE, FIXED)

    Exec Addr    Load Addr    Size         Type   Attr      Idx    E Section Name        Object

    0x0100a200   0x0100a200   0x00000004   Data   RO          582    .option_setting_ofs1_sec  bsp_rom_registers.o


    Execution Region UNUSED_7 (Exec base: 0x0100a204, Load base: 0x0100a204, Size: 0x00000000, Max: 0x00000000, ABSOLUTE, FIXED)

    Exec Addr    Load Addr    Size         Type   Attr      Idx    E Section Name        Object

    0x0100a204        -       0x00000000   Zero   RW           19    UNUSED_7.bss        anon$$obj.o


    Execution Region OFS3_SEC (Exec base: 0x0100a204, Load base: 0x0100a204, Size: 0x00000000, Max: 0xffffffff, ABSOLUTE, FIXED)

    **** No section assigned to this execution region ****


    Execution Region UNUSED_8 (Exec base: 0x0100a204, Load base: 0x0100a204, Size: 0x0000000c, Max: 0x0000000c, ABSOLUTE, FIXED)

    Exec Addr    Load Addr    Size         Type   Attr      Idx    E Section Name        Object

    0x0100a204        -       0x0000000c   Zero   RW           20    UNUSED_8.bss        anon$$obj.o


    Execution Region BANKSEL_SEC (Exec base: 0x0100a210, Load base: 0x0100a210, Size: 0x00000004, Max: 0xffffffff, ABSOLUTE, FIXED)

    Exec Addr    Load Addr    Size         Type   Attr      Idx    E Section Name        Object

    0x0100a210   0x0100a210   0x00000004   Data   RO          583    .option_setting_banksel_sec  bsp_rom_registers.o


    Execution Region UNUSED_9 (Exec base: 0x0100a214, Load base: 0x0100a214, Size: 0x0000002c, Max: 0x0000002c, ABSOLUTE, FIXED)

    Exec Addr    Load Addr    Size         Type   Attr      Idx    E Section Name        Object

    0x0100a214        -       0x0000002c   Zero   RW           21    UNUSED_9.bss        anon$$obj.o


    Execution Region BPS_SEC (Exec base: 0x0100a240, Load base: 0x0100a240, Size: 0x00000010, Max: 0xffffffff, ABSOLUTE, FIXED)

    Exec Addr    Load Addr    Size         Type   Attr      Idx    E Section Name        Object

    0x0100a240   0x0100a240   0x00000004   Data   RO          584    .option_setting_bps_sec0  bsp_rom_registers.o
    0x0100a244   0x0100a244   0x00000004   Data   RO          585    .option_setting_bps_sec1  bsp_rom_registers.o
    0x0100a248   0x0100a248   0x00000004   Data   RO          586    .option_setting_bps_sec2  bsp_rom_registers.o
    0x0100a24c   0x0100a24c   0x00000004   Data   RO          587    .option_setting_bps_sec3  bsp_rom_registers.o


    Execution Region UNUSED_10 (Exec base: 0x0100a250, Load base: 0x0100a250, Size: 0x00000010, Max: 0x00000010, ABSOLUTE, FIXED)

    Exec Addr    Load Addr    Size         Type   Attr      Idx    E Section Name        Object

    0x0100a250        -       0x00000010   Zero   RW           22    UNUSED_10.bss       anon$$obj.o


    Execution Region PBPS_SEC (Exec base: 0x0100a260, Load base: 0x0100a260, Size: 0x00000010, Max: 0xffffffff, ABSOLUTE, FIXED)

    Exec Addr    Load Addr    Size         Type   Attr      Idx    E Section Name        Object

    0x0100a260   0x0100a260   0x00000004   Data   RO          588    .option_setting_pbps_sec0  bsp_rom_registers.o
    0x0100a264   0x0100a264   0x00000004   Data   RO          589    .option_setting_pbps_sec1  bsp_rom_registers.o
    0x0100a268   0x0100a268   0x00000004   Data   RO          590    .option_setting_pbps_sec2  bsp_rom_registers.o
    0x0100a26c   0x0100a26c   0x00000004   Data   RO          591    .option_setting_pbps_sec3  bsp_rom_registers.o


    Execution Region UNUSED_11 (Exec base: 0x0100a270, Load base: 0x0100a270, Size: 0x00000010, Max: 0x00000010, ABSOLUTE, FIXED)

    Exec Addr    Load Addr    Size         Type   Attr      Idx    E Section Name        Object

    0x0100a270        -       0x00000010   Zero   RW           23    UNUSED_11.bss       anon$$obj.o


    Execution Region OFS1_SEL (Exec base: 0x0100a280, Load base: 0x0100a280, Size: 0x00000004, Max: 0xffffffff, ABSOLUTE, FIXED)

    Exec Addr    Load Addr    Size         Type   Attr      Idx    E Section Name        Object

    0x0100a280   0x0100a280   0x00000004   Data   RO          592    .option_setting_ofs1_sel  bsp_rom_registers.o


    Execution Region UNUSED_12 (Exec base: 0x0100a284, Load base: 0x0100a284, Size: 0x00000000, Max: 0x00000000, ABSOLUTE, FIXED)

    Exec Addr    Load Addr    Size         Type   Attr      Idx    E Section Name        Object

    0x0100a284        -       0x00000000   Zero   RW           24    UNUSED_12.bss       anon$$obj.o


    Execution Region OFS3_SEL (Exec base: 0x0100a284, Load base: 0x0100a284, Size: 0x00000000, Max: 0xffffffff, ABSOLUTE, FIXED)

    **** No section assigned to this execution region ****


    Execution Region UNUSED_13 (Exec base: 0x0100a284, Load base: 0x0100a284, Size: 0x0000000c, Max: 0x0000000c, ABSOLUTE, FIXED)

    Exec Addr    Load Addr    Size         Type   Attr      Idx    E Section Name        Object

    0x0100a284        -       0x0000000c   Zero   RW           25    UNUSED_13.bss       anon$$obj.o


    Execution Region BANKSEL_SEL (Exec base: 0x0100a290, Load base: 0x0100a290, Size: 0x00000000, Max: 0xffffffff, ABSOLUTE, FIXED)

    **** No section assigned to this execution region ****


    Execution Region UNUSED_14 (Exec base: 0x0100a290, Load base: 0x0100a290, Size: 0x00000030, Max: 0x00000030, ABSOLUTE, FIXED)

    Exec Addr    Load Addr    Size         Type   Attr      Idx    E Section Name        Object

    0x0100a290        -       0x00000030   Zero   RW           26    UNUSED_14.bss       anon$$obj.o


    Execution Region BPS_SEL (Exec base: 0x0100a2c0, Load base: 0x0100a2c0, Size: 0x00000010, Max: 0xffffffff, ABSOLUTE, FIXED)

    Exec Addr    Load Addr    Size         Type   Attr      Idx    E Section Name        Object

    0x0100a2c0   0x0100a2c0   0x00000004   Data   RO          593    .option_setting_bps_sel0  bsp_rom_registers.o
    0x0100a2c4   0x0100a2c4   0x00000004   Data   RO          594    .option_setting_bps_sel1  bsp_rom_registers.o
    0x0100a2c8   0x0100a2c8   0x00000004   Data   RO          595    .option_setting_bps_sel2  bsp_rom_registers.o
    0x0100a2cc   0x0100a2cc   0x00000004   Data   RO          596    .option_setting_bps_sel3  bsp_rom_registers.o


    Execution Region UNUSED_15 (Exec base: 0x0100a2d0, Load base: 0x0100a2d0, Size: 0x00000030, Max: 0x00000030, ABSOLUTE, FIXED)

    Exec Addr    Load Addr    Size         Type   Attr      Idx    E Section Name        Object

    0x0100a2d0        -       0x00000030   Zero   RW           27    UNUSED_15.bss       anon$$obj.o


    Execution Region __tz_OPTION_SETTING_S_N (Exec base: 0x0100a300, Load base: 0x0100a300, Size: 0x00000000, Max: 0x00000000, ABSOLUTE)

    Exec Addr    Load Addr    Size         Type   Attr      Idx    E Section Name        Object

    0x0100a300        -       0x00000000   Zero   RW           28    __tz_OPTION_SETTING_S_N.bss  anon$$obj.o



  Load Region LOAD_REGION_DATA_FLASH (Base: 0x08000000, Size: 0x00000000, Max: 0x00002000, ABSOLUTE)

    Execution Region __tz_DATA_FLASH_S (Exec base: 0x08000000, Load base: 0x08000000, Size: 0x00000000, Max: 0x00000000, ABSOLUTE)

    Exec Addr    Load Addr    Size         Type   Attr      Idx    E Section Name        Object

    0x08000000        -       0x00000000   Zero   RW           29    __tz_DATA_FLASH_S.bss  anon$$obj.o


    Execution Region DATA_FLASH (Exec base: 0x08000000, Load base: 0x08000000, Size: 0x00000000, Max: 0xffffffff, ABSOLUTE)

    **** No section assigned to this execution region ****


    Execution Region __tz_DATA_FLASH_N (Exec base: 0x08000000, Load base: 0x08000000, Size: 0x00000000, Max: 0x00000000, ABSOLUTE)

    Exec Addr    Load Addr    Size         Type   Attr      Idx    E Section Name        Object

    0x08000000        -       0x00000000   Zero   RW           30    __tz_DATA_FLASH_N.bss  anon$$obj.o



  Load Region LOAD_REGION_QSPI_FLASH (Base: 0x60000000, Size: 0x00000000, Max: 0x04000000, ABSOLUTE)

    Execution Region __tz_QSPI_FLASH_S (Exec base: 0x60000000, Load base: 0x60000000, Size: 0x00000000, Max: 0x00000000, ABSOLUTE)

    Exec Addr    Load Addr    Size         Type   Attr      Idx    E Section Name        Object

    0x60000000        -       0x00000000   Zero   RW           31    __tz_QSPI_FLASH_S.bss  anon$$obj.o


    Execution Region QSPI_FLASH (Exec base: 0x60000000, Load base: 0x60000000, Size: 0x00000000, Max: 0xffffffff, ABSOLUTE, FIXED)

    **** No section assigned to this execution region ****


    Execution Region __tz_QSPI_FLASH_N (Exec base: 0x60000000, Load base: 0x60000000, Size: 0x00000000, Max: 0x00000000, ABSOLUTE)

    Exec Addr    Load Addr    Size         Type   Attr      Idx    E Section Name        Object

    0x60000000        -       0x00000000   Zero   RW           32    __tz_QSPI_FLASH_N.bss  anon$$obj.o



  Load Region LOAD_REGION_OSPI_DEVICE_0 (Base: 0x80020000, Size: 0x00000000, Max: 0x00000000, ABSOLUTE)

    Execution Region __tz_OSPI_DEVICE_0_S (Exec base: 0x80020000, Load base: 0x80020000, Size: 0x00000000, Max: 0x00000000, ABSOLUTE)

    Exec Addr    Load Addr    Size         Type   Attr      Idx    E Section Name        Object

    0x80020000        -       0x00000000   Zero   RW           33    __tz_OSPI_DEVICE_0_S.bss  anon$$obj.o


    Execution Region OSPI_DEVICE_0 (Exec base: 0x80020000, Load base: 0x80020000, Size: 0x00000000, Max: 0xffffffff, ABSOLUTE, FIXED)

    **** No section assigned to this execution region ****


    Execution Region __tz_OSPI_DEVICE_0_N (Exec base: 0x80020000, Load base: 0x80020000, Size: 0x00000000, Max: 0x00000000, ABSOLUTE)

    Exec Addr    Load Addr    Size         Type   Attr      Idx    E Section Name        Object

    0x80020000        -       0x00000000   Zero   RW           34    __tz_OSPI_DEVICE_0_N.bss  anon$$obj.o



  Load Region LOAD_REGION_OSPI_DEVICE_1 (Base: 0x80030000, Size: 0x00000000, Max: 0x00000000, ABSOLUTE)

    Execution Region __tz_OSPI_DEVICE_1_S (Exec base: 0x80030000, Load base: 0x80030000, Size: 0x00000000, Max: 0x00000000, ABSOLUTE)

    Exec Addr    Load Addr    Size         Type   Attr      Idx    E Section Name        Object

    0x80030000        -       0x00000000   Zero   RW           35    __tz_OSPI_DEVICE_1_S.bss  anon$$obj.o


    Execution Region OSPI_DEVICE_1 (Exec base: 0x80030000, Load base: 0x80030000, Size: 0x00000000, Max: 0xffffffff, ABSOLUTE, FIXED)

    **** No section assigned to this execution region ****


    Execution Region __tz_OSPI_DEVICE_1_N (Exec base: 0x80030000, Load base: 0x80030000, Size: 0x00000000, Max: 0x00000000, ABSOLUTE)

    Exec Addr    Load Addr    Size         Type   Attr      Idx    E Section Name        Object

    0x80030000        -       0x00000000   Zero   RW           36    __tz_OSPI_DEVICE_1_N.bss  anon$$obj.o



  Load Region LOAD_REGION_SDRAM (Base: 0x80010000, Size: 0x00000000, Max: 0x00000000, ABSOLUTE)

    Execution Region __tz_SDRAM_S (Exec base: 0x80010000, Load base: 0x80010000, Size: 0x00000000, Max: 0x00000000, ABSOLUTE)

    Exec Addr    Load Addr    Size         Type   Attr      Idx    E Section Name        Object

    0x80010000        -       0x00000000   Zero   RW           37    __tz_SDRAM_S.bss    anon$$obj.o


    Execution Region SDRAM (Exec base: 0x80010000, Load base: 0x80010000, Size: 0x00000000, Max: 0xffffffff, ABSOLUTE, FIXED)

    **** No section assigned to this execution region ****


    Execution Region __tz_SDRAM_N (Exec base: 0x80010000, Load base: 0x80010000, Size: 0x00000000, Max: 0x00000000, ABSOLUTE)

    Exec Addr    Load Addr    Size         Type   Attr      Idx    E Section Name        Object

    0x80010000        -       0x00000000   Zero   RW           38    __tz_SDRAM_N.bss    anon$$obj.o



  Load Region LOAD_REGION_SHELL_COMMAND (Base: 0x0007e000, Size: 0x00000000, Max: 0x00002000, ABSOLUTE)

    Execution Region SHELL_COMMAND (Exec base: 0x0007e000, Load base: 0x0007e000, Size: 0x00000000, Max: 0xffffffff, ABSOLUTE, FIXED)

    **** No section assigned to this execution region ****


==============================================================================

Image component sizes


      Code (inc. data)   RO Data    RW Data    ZI Data      Debug   Object Name

       480          0          0          0         28      34203   bsp_clocks.o
         8          0         78          0          0       9808   bsp_common.o
        80          0          0          0          0       1571   bsp_delay.o
        68          0          0          0         56      14093   bsp_group_irq.o
         0          0          0          0          4        463   bsp_io.o
       138          0          0          0         36      16509   bsp_irq.o
       160          0          8          0          8      22665   bsp_register_protection.o
         0          0         68          0          0       1052   bsp_rom_registers.o
         0          0         32          0          0        824   bsp_security.o
         0          0         12          0          8      17603   common_data.o
         0          0        680          4        196      87080   hal_data.o
      2638        212       1072          5        485      39699   hal_entry.o
       766         80        335          0        276       7395   log.o
       466          0          0          0          0      10795   lwrb.o
        10          0          0          0          0        390   main.o
       566          6          0          0          4       3428   multi_button.o
         0          0        140          0          0       7998   pin_data.o
      1480          0         52          0          1      81948   r_adc.o
       490          0         20          0          0      19112   r_dac.o
      1770          0         52          0          0      78221   r_gpt.o
       984         12         52          0          0      58257   r_ioport.o
      1850          0         36          0          2      75724   r_sci_uart.o
      5614        304       1143          2         29      38545   shell.o
      1508        500        326          0          4       7516   shell_cmds.o
        30          0          0          0          0       3425   shell_companion.o
       750          8          0          0          0       7493   shell_ext.o
       118          0          0         16        368       4089   shell_port_1.o
        14          0         64          0       9216        927   startup.o
       240          0          0          0          4       6665   system.o
         0          0         72          0          0       7622   vector_data.o

    ----------------------------------------------------------------------
     20268       1122       4244         28      11060     665120   Object Totals
         0          0          0          0        324          0   (incl. Generated)
        40          0          2          1         11          0   (incl. Padding)

    ----------------------------------------------------------------------

      Code (inc. data)   RO Data    RW Data    ZI Data      Debug   Library Member Name

        56          8          0          0          0         84   __0sscanf.o
        28          0          0          0          0         68   _chval.o
       812          4          0          0          0        112   _scanf.o
       332          0          0          0          0         96   _scanf_int.o
        64          0          0          0          0         84   _sgetc.o
        40          6         64          0          0         68   ctype_c.o
        18          0          0          0          0         80   fputc.o
        10          0          0          0          0         68   isspace_c.o
         0          0          0          0          0          0   iusefp.o
         0          0          0          0          0          0   iusesemip.o
        30          0          0          0          0         68   llshl.o
        36          0          0          0          0         68   llsshr.o
        32          0          0          0          0         68   llushr.o
        36          0          0          0          0         68   memcpya.o
        36          0          0          0          0        108   memseta.o
      2402         96          0          0          0        756   printfa.o
        36          6          0          0          0         80   puts.o
        40          8          0          0          0         84   scanf_char.o
         0          0          0          0          0          0   semi.o
         0          0          0          4          0          0   stdout.o
        28          0          0          0          0         76   strcmp.o
        14          0          0          0          0         68   strlen.o
        30          0          0          0          0         80   strncmp.o
        44          0          0          0          0         80   uidiv.o
        98          0          0          0          0         92   uldiv.o
        48          0          0          0          0         68   cdrcmple.o
       334          0          0          0          0        148   dadd.o
       222          0          0          0          0        100   ddiv.o
       186          0          0          0          0        176   depilogue.o
        48          0          0          0          0         68   dfixul.o
       228          0          0          0          0         96   dmul.o

    ----------------------------------------------------------------------
      5296        128         64          4          0       3012   Library Totals
         8          0          0          0          0          0   (incl. Padding)

    ----------------------------------------------------------------------

      Code (inc. data)   RO Data    RW Data    ZI Data      Debug   Library Name

      4222        128         64          4          0       2356   mc_w.l
      1066          0          0          0          0        656   mf_w.l

    ----------------------------------------------------------------------
      5296        128         64          4          0       3012   Library Totals

    ----------------------------------------------------------------------

==============================================================================


      Code (inc. data)   RO Data    RW Data    ZI Data      Debug   

     25564       1250       4308         32      11060     666028   Grand Totals
     25564       1250       4308         32      11060     666028   ELF Image Totals
     25564       1250       4308         32          0          0   ROM Totals

==============================================================================

    Total RO  Size (Code + RO Data)                29872 (  29.17kB)
    Total RW  Size (RW Data + ZI Data)             11092 (  10.83kB)
    Total ROM Size (Code + RO Data + RW Data)      29904 (  29.20kB)

==============================================================================

